:020000040800F2
:100000000000022059B105085D990008755C0208DE
:1000100009B2050809B2050809B205080000000088
:100020000000000000000000000000008DB000088B
:100030008FB000080000000091B00008F51401081E
:1000400009B2050809B2050809B2050809B2050890
:1000500009B2050809B205086BFE00086FFE00082A
:1000600009B2050873FE000877FE00084DA00008DD
:1000700061A0000875A0000889A000089DA00008E4
:10008000B1A00008C5A0000809B2050800000000E2
:100090000000000000000000000000007BFE0008DF
:1000A000859F0008AD9F0008D59F00086F9F00083E
:1000B000FD9F000811A0000825A0000809B205084E
:1000C00009B2050809B2050809B2050809B2050810
:1000D00009B20508A19A0008AD9A000800000000C6
:1000E0007FFE000809B2050893B000080000000078
:1000F000000000000000000000000000D9A000087F
:100100000000000009B2050839A0000809B205087E
:1001100000000000000000000000000000000000DF
:10012000EDA0000801A1000815A1000829A1000800
:100130003DA10008000000000000000000000000D9
:10014000000000000000000000000000E5B0000812
:1001500051A1000865A1000879A1000809B20508AD
:1001600009B2050809B205080000000000000000FF
:10017000000000000000000000000000000000007F
:100180000000000009B205080000000000000000A7
:0801900009B2050809B20508D7
:1001980081C90181008408B10000000080C9018183
:1001A800008408B10000000080C90181B0AB08B12B
:1001B80000000000C9010181B0B0AC80000000005F
:1001C800C9060181B0B0AF85000000003F1A018167
:1001D800B0AF81C90000000008B10181B0B000844F
:1001E8000000000008B10181B0B0008400000000E8
:1001F800B0B805000084028018B9050001000000AD
:1002080080BA050000840280ECBA050001000000F5
:10021800ECBA05007CFFFF7FA0BB050080FFFF7FD5
:10022800E0BB050084FFFF7FC8BC0500B0B0AE800E
:100238006CBE0500B0A80180B4BF050078FFFF7F41
:10024800D4C50500B0AA058030C80500010000002B
:1002580030C805006CFFFF7F9CD30500010000003B
:1002680030D6050068FFFF7F9CDC05000100000018
:1002780024DD0500B0A8018034DD05000100000080
:1002880064DD0500B00D848074DD05000100000008
:1002980098DD050044FFFF7FA4DD050048FFFF7FD0
:1002A800B0DD0500AF08B180E8E0050001000000FE
:1002B800F4E00500A908B180A0E2050001000000F3
:1002C80074180600A908B1809C18060001000000F7
:1002D80068190600B0A90280FC190600B0B0A88011
:1002E8004C1A060001000000541A0600B0B0AA809B
:1002F800881A0600AE71B2804C1B0600AB3F3880EE
:10030800AC1B060001000000B41B0600B0B0AA80B8
:10031800F01B060001000000901C0600AA0DB28028
:100328000C1D0600B0AF0880AC1F060001000000DD
:10033800BC1F0600AD3F0280382206000100000005
:1003480068220600B0AD04800C25060001000000FC
:10035800B85001200201000002001400D85001200A
:100368000202000002001400F8500120020A0000F6
:1003780002001400185101200206000002001400B7
:1003880038510120020700000200140058510120D2
:100398000203000004001400785101200208000044
:1003A8000400140098510120010B000000007700A0
:1003B800B8510120010C000000007600D85101203E
:1003C8000110000000007600F8510120010D010025
:1003D800000077001852012001120000000076008A
:1003E800385201200114000000001E00585201205C
:1003F800011A000000000D0078520120011B0000C6
:1004080000000E0098520120011C000000001E0090
:10041800B85201200117000000000C00D85201203A
:100428000118000000000E00F85201200128010008
:1004380000001800185301200120000000004800A7
:1004480038530120012100000000490058530120C1
:100458000122000000004A00785301200123000017
:1004680000004B00985301200124000000004C00BC
:10047800B85301200125000000004D00D853012089
:100488000126000000004E00F8530120012700005B
:1004980000004F0018540120012B00000000290023
:1004A80038540120012C0100000029005854012073
:1004B800012D01000000700078540120012E010078
:1004C8000000520098540120012F0100000028006C
:1004D800B85401200130010000002800D854012040
:1004E8000234040000012C00F854012001330000FC
:1004F80000003C00185501200136000000002000D3
:10800000D0E907239A422FBFD01AC0688018C01A3F
:108010007047D0E9092300699A4238BF1218D31A71
:108020000138C01A7047D0E90902131A5842584162
:108030007047036A41690246C85CD16801338B42CC
:1080400028BF002313627047436A8269D154436A90
:1080500002690133934228BF0023426B4362D36815
:1080600043F08003D3607047436B188810F0100012
:108070001EBF1A889B8801207047436B99891A8814
:10808000890610B592B2044607D5900605D5E26A76
:1080900022B39888216B80B29047636B99891A88C4
:1080A000090692B20FD510060DD5D4E909128A42FD
:1080B00022D0A169895C998021690132B2FBF1F07B
:1080C00001FB1022A262998A1A88C90592B204D5CE
:1080D000D20744BF4FF6F7721A8010BD9B88E26941
:1080E0006169DBB28B54E369E2680133B3FBF2F1FF
:1080F00002FB1133E361D0E7DA6822F08002DA6034
:10810000E1E7036941681F2B30B54FF0200285BFBE
:10811000A3F120054C680C68AA4098BF9A402242FF
:108120001ED0826900201074D0688468206820F016
:10813000010020605468206865790A4C828934F80F
:10814000154092B21F2B22EA0402828188BF203B95
:108150004FF020028BBF9A4002FA03F3CA608B6093
:1081600030BD00BF542B06080E4BDA68D20310D482
:10817000DA68D1060FD4DA68D2050ED4DA6812F0C4
:10818000E00F0CD1DB6813F0020F14BF08200920A8
:108190007047012070470620704702207047072073
:1081A000704700BF003C024007B509238DF8073037
:1081B000FFF7DAFF8DF807009DF80730012BF7D0A5
:1081C0009DF8070003B05DF804FB838A028B9BB225
:1081D00043EA024331EA03030CBF01200020704749
:1081E00082B0002301930093012300900193019B2F
:1081F00063B1009A21F07F4314320092009A126812
:108200001A4214BF0120002002B07047009A1832B1
:10821000F3E77047704701207047034BD3E9000331
:10822000C01AC0F30A007047F8180020054AD2E9C6
:1082300000138B42FDD0D1180133C3F30A03087A2F
:1082400053607047F8180020044BD3F8080820B199
:10825000D3F80808431F584258417047F8180020C7
:10826000012380F849307047044BD3E90003C01A5A
:10827000C0F30A00C0F50060704700BFF818002086
:1082800010B5D0F8E83504461B699847032384F8F5
:108290001231002010BD08B590F8123180F813316A
:1082A000042380F81231D0F8E835DB6898470020C5
:1082B00008BD08B5D0F8E435DB6903B19847002064
:1082C00008BD08B5D0F8E4351B6A9847002008BD02
:1082D00008B5D0F8E4355B6A9847002008BD30B592
:1082E0000138002423460134055D002DFAD1DBB2AC
:1082F00001335B0013800B7003234B70022310F8D3
:10830000014F04B930BD5A1CD2B2CC5402338D5443
:10831000DBB2F4E710B5074C2068FF2808D0064907
:10832000D1F80C2801F5016100F070F8FF232360FB
:10833000002010BD00000020F81800204323014851
:108340000B80704704000020122301480B80704707
:1083500047000020042301480B807047590000208B
:1083600008B50A4602490348FFF7B9FF084608BDA9
:10837000102100202CCA060808B50A460249034805
:10838000FFF7ADFF084608BD102100203FCA0608D0
:1083900008B50A4602490348FFF7A1FF084608BD91
:1083A0001021002044CA060808B50A4602490348BD
:1083B000FFF795FF084608BD102100204ECA0608A9
:1083C00008B50A4602490348FFF789FF084608BD79
:1083D0001021002059CA060870477047704770473F
:1083E00070477047044B00200522C3F80828C3F8E3
:1083F0001809C3F81C097047F8180020024B002028
:10840000C3F80808704700BFF8180020212838B5C5
:108410000C461BD022282BD0202815D1A1B1072A29
:1084200012D11A4DD5F81C3913B1096800209847AC
:108430002368C5F82039237985F82439637985F8CC
:108440002539A37985F82639002038BD0029FBD0CD
:10845000072AF9D10D4BD3F820290A6093F8242973
:108460000A7193F825294A7193F826398B71EBE745
:108470000029E9D0022AE7D1044BD3F81839002BA0
:10848000E2D0098800209847DEE700BFF8180020F6
:1084900030B50E4CD4E900329A1AC2F30A020A44EB
:1084A000B2F5006F10D801440022814203D102B11D
:1084B0002360002030BDE21810F8015B1572013313
:1084C000C3F30A030122F0E70220F3E7F8180020C3
:1084D000034BD3F8280908B103691847704700BF58
:1084E000F8180020034B93F85009003818BF0120FA
:1084F000704700BFF8180020034B93F85009032879
:1085000094BF002001207047F818002000487047F1
:108510004C220020837B042B0DD0074BD3F89820EE
:108520000132C3F89820426004228273D3F89C2061
:108530000132C3F89C207047C45F0020202301480B
:108540000B8070475D000020122301480B807047AC
:108550007D000020042301480B8070478F0000201D
:108560000A4608B5044920B90448FFF7B8FE024896
:1085700008BD0348F9E700BF7C22002067CA06084F
:108580007FCA060808B50A4602490348FFF7A7FE56
:10859000084608BD7C22002097CA060808B50A468E
:1085A00002490348FFF79BFE084608BD7C220020D5
:1085B000AACA060808B50A4602490348FFF78FFE13
:1085C000084608BD7C220020B5CA0608002370B505
:1085D0004D1C1E46040FB0F1204F34BF30343734E9
:1085E00001F8134005F813600133DCB2A2424FEAF0
:1085F0000010EFD870BD1A2310B50B80094BD3F8CB
:10860000E807D3F8EC2780180AD0D3F8EA470649E0
:108610000822FFF7DBFF042210312046FFF7D6FFC8
:10862000024810BD00F0FF1F9500002093000020BD
:1086300008B5FFF74DFF80F00100404240B208BD91
:10864000002070470020704770477047D0ED007AD7
:10865000D0ED036A30EE677AE6EE877AB0EE670A0D
:10866000C0ED007A7047D0ED017AF5EE407AF1EE78
:1086700010FA09D1DFED0F7A60EEA70AB7EE007AA3
:10868000C7EE207AC0ED017AD0ED017A80ED021AB2
:1086900071EE277AC1EE276AD0ED007AC0ED036A49
:1086A00030EE677AE6EE877AB0EE670AC0ED007AC0
:1086B000704700BFDB0FC940D0ED017AD0ED036AEF
:1086C00030EE670AE6EE807A90ED000AC0ED017A9E
:1086D000B0EE677AD0ED027A37EE677AE6EE877A07
:1086E000C0ED027A77EEC07AA6EEA70A80ED000A06
:1086F000704790ED056AD0ED017AD0ED006AD0EDBB
:10870000025A90ED045A66EE277AB0EE407AE6EE11
:10871000807AD0ED066A80ED057AE5EEA67AD0ED96
:10872000076AD0ED035A80ED066AE5EEE67AD0EDF1
:10873000085AC0ED086AE5EE657AB0EE670AC0ED4A
:10874000077A7047D0ED006AD0ED057AE6EE807AC0
:10875000B0EE407AB0EE670AD0ED037AD0ED016A50
:1087600067EEC07AE6EE877AD0ED066A76EEA77AF3
:10877000D0ED026AC0ED057AD0ED047A67EEC07ADA
:10878000E6EE877AC0ED067A704703685A1C0260ED
:108790001970704703690133012B036106D100236F
:1087A00080ED010A80ED000A8360704790ED006A59
:1087B00007EE903A70EE466AF8EEE77A86EEA77A10
:1087C00077EE067A90ED027AC0ED017A30EE670A14
:1087D000C0ED007AA6EE807A80ED037A80ED027A11
:1087E000704703685A1C026019707047007970471F
:1087F0000079C0F3401070470079400970472DE9B7
:10880000F041476906468846002F59D10368C3F3F3
:108810000D0515B3D8F800803568FFF7C5FC0928A9
:1088200040F08780444C236923F44073236123691B
:1088300043F400732361236943F001032361C5F806
:108840000080FFF7B1FC2369092823F001032361AD
:108850006FD133680433336032E0384A934229D30E
:1088600002F58042934224D302F5804293422AD3F8
:10887000334A934229D902F58032934227D902F52F
:108880000032934225D902F50032934223D902F5F2
:108890000032934221D902F5003293421FD902F5EA
:1088A000802293421DD9B3F1016F1CD305200BF038
:1088B000A7F80825FFF778FC092816D04FF0FF37F6
:1088C0003846BDE8F0811025F4E71825F2E72025A9
:1088D000F0E72825EEE73025ECE73825EAE74025E4
:1088E000E8E74825E6E75825E4E7134C236923F435
:1088F00040732361236943F400732361236923F0E8
:10890000F803236123691D4345F0020525612369AE
:1089100043F480332361FFF747FC236923F002030C
:1089200023612369092823F0F80323613FF472AF20
:10893000C4E76FF00107C3E7003C024000400008B5
:10894000FFFF000803682DE9F04104464068134426
:1089500083421AD80D468E1804F10C074FF0000818
:10896000B54202D16069BDE8F08123695A1C2261D9
:10897000234415F8011B1973042AF1D13946204606
:10898000FFF73DFFC4E90480EAE74FF0FF30EAE774
:108990002DE9F347038A8689B6B205460C461E4088
:1089A0004FF0004901F14C0701F1340816B902B04B
:1089B000BDE8F087B6FA86F329FA03F2D24391B202
:1089C000298216401B3B002C40D0042BEED8DFE858
:1089D00003F039342E280300E368D5F82CA02BB11E
:1089E0009B681BB11FFA8AF1201D9847636A33B157
:1089F0009B6823B11FFA8AF104F11C009847E36BCE
:108A00002BB19B681BB11FFA8AF140469847636DF2
:108A1000002BCBD09B68002BC8D01FFA8AF13846B8
:108A200003E0E368696B5B68201D9847BEE7636AF3
:108A3000A96B5B6804F11C00F7E7E36BE96B5B680B
:108A40004046F2E7636D296C5B68E8E7042B06D8C3
:108A5000DFE803F00D0B09070300EB6A0193019BAC
:108A6000A4E76B6BFAE7AB6BF8E7EB6BF6E72B6C05
:108A7000F4E790F84820531C0244DBB280F84830F9
:108A800082F8341090F849200AB1132B01D951F023
:108A9000D6B97047002280F8492051F0D0B970B59E
:108AA000124D95F8833A002BFBD104464618B44288
:108AB00004D1002070BD01200AF016FCD5F8843ADC
:108AC000D5F8882A0133C3F30A039342F3D0D5F8CB
:108AD000843A14F8012B2B4483F88C2AD5F8843A75
:108AE0000133C3F30A03C5F8843AE0E7F81800201D
:108AF00038B50C461146FFF7A7FB48B1054D002AD3
:108B0000D5F8943104DD2046FFF7C9FFD5F894313C
:108B100038BD00BFF0290020F0B590F8CF5590F88F
:108B2000CE1590F8D12590F8D03590F8CC7590F806
:108B3000CDC501EB05218DB203EB022390F8D315CF
:108B400090F8D22585B002EB012207F01F06012123
:108B500092B29BB28E4204468DF808708DF809C01F
:108B6000ADF80A50ADF80C30ADF80E20C0F8402139
:108B700080F8111100F00C81022E00F01D81002EF2
:108B800040F09B81BCF1090F5ED8DFE81CF0B60015
:108B9000F4005D00C8005D0057000A005D00A900F8
:108BA00076002E0A022EADF806200BD0032E25D01B
:108BB000012E49D1D0F8EC351B68A0780DF10601E3
:108BC000984709E0D0F8E43580789B6A0DF10601FA
:108BD00098474670C4F8F005BDF80620002A47D033
:108BE000BDF80E30002B43D09A4228BF1A46ADF88C
:108BF00006200146204650F037FC39E0E9B205294D
:108C000022D8DFE801F003070B0F1317D0F8EC357B
:108C10005B68D2E7D0F8EC359B68CEE7D0F8EC354E
:108C2000DB68CAE7D0F8EC351B69C6E7D0F8EC354D
:108C30005B69C2E7D0F8EC359B69BEE71A4303D104
:108C400090F81231032B03D1204650F039FB0FE08E
:108C5000016905F07F0680F814610B6865F30A125C
:108C60001A430A6050F014FC2EB1022384F812312A
:108C7000002005B0F0BD0123F8E7E9B2904D0129CD
:108C800085F89811E0D890F81231022B0FD0032B01
:108C9000DAD1C1B9022380F81231D0F8E43580F876
:108CA00010115B689847204650F0F2FBE0E700297E
:108CB000F9D00121032380F8101180F812312046E9
:108CC00050F0C0FAEFE790F810110129EBD0D0F87E
:108CD000E4355B68984795F8981184F81011EEE731
:108CE000012AB1D190F81231022B04D0032BABD161
:108CF00000F588717EE773497CE790F81231023BFA
:108D0000012BA1D86E4B0022C3F8A021D0F8182166
:108D100012B10222C3F8A0216B4902226AE7012D99
:108D200008D1C0F81851D4F8E43502A99B68204650
:108D30009847B8E7022D9BD1DAB2002A98D1026990
:108D40001B0A023B5268032B03D8DFE803F00C0E2A
:108D50001012012363F30612594BC3F8A421012317
:108D600084F816319FE70223F4E70323F2E7042394
:108D7000F0E70523EEE790F81231023B012B3FF6B6
:108D800063AF012D7FF474AF0023C0F81831CAE738
:108D900090F81221032A7FF457AFDBB2012B3FF684
:108DA00053AFD0F8E43502A99B689847BDF80E3060
:108DB000002B7FF45DAF76E707F06007202FD9B274
:108DC00005D1D0F8E43502A99B68984750E7BCF17B
:108DD000010F31D0BCF1030F1ED0BCF1000F7FF4A6
:108DE00047AF90F81221022A5AD0032A7FF42CAF01
:108DF00013F0800F4FF02802314B59D001F07F0162
:108E000002FB010191F81E21002A4FD00122C3F874
:108E1000A8212E490222EDE690F81231022B3FD014
:108E2000032B7FF411AF002D7FF47DAF4A063FF492
:108E30007AAF50F013FA76E790F81221022A2FD079
:108E4000032A7FF401AF002D7FF412AF11F07F00F1
:108E50003FF429AF5BB2002B4FF02802B5BF02FBF5
:108E6000004102FB014101F58E7101F55D710022A7
:108E7000DB0F08708A704B7004EB8000C9786BB10F
:108E80008269136802396FF3555301298CBFC3F30C
:108E90000071012161F31C73136044E7426DF0E738
:108EA0004B063FF4E5AE50F0D9F9E1E60022AEE71B
:108EB00002FB010191F87623A6E707F08001F2E7B3
:108EC000F02900208C2B0020902B0020982B0020D4
:108ED00010B5044671BB90F81131032B1BD1D0F8AB
:108EE0009023D0F87C339A4217D9C178012908BF62
:108EF000D0F88013A2EB030204BFC918C0F8801396
:108F0000934228BF1346C0F890239BB2D0F8802329
:108F1000002150F06DFB002010BDD0F8E4351B6936
:108F200023B190F81221032A00D19847204650F02F
:108F3000AFFAF0E7D0F8E4359B69002BEBD090F85E
:108F40001221032AE7D19847E5E770B50A7812F0B5
:108F5000600406460D462AD0202C2FD1CC884B78B1
:108F6000FCB112060CD51F4922461846FFF74EFAEF
:108F7000EA881C49304650F077FA0024204670BD3C
:108F8000194A1360194A0323C2F80C4880F81131BA
:108F9000C0E9E444234602F50162002150F028FBB9
:108FA000EBE7022211441846FFF730FAE6E74B7868
:108FB0000A2B08D00B2B0BD0062BDFD1304650F0FC
:108FC0007FF90224DAE70A49012250F04DFAD5E789
:108FD0008B781BB9074BC3F8AC41CFE750F070F961
:108FE000CCE700BF0821002000000020F818002076
:108FF0009C2B0020F029002010B5282303FB010141
:10900000074AB1F88C1304461046FFF741FA204690
:10901000034A4023012150F0EBFA002010BD00BFAD
:10902000A02B002070B50F4DD5F8F831044643B1A0
:1090300095F8FC2195F81032134302D1012150F02C
:109040000DF98121204650F009F995F81032022BD4
:1090500007D12046044ABDE870401F23012150F08B
:10906000C7BA70BDF0290020E02B0020002310B506
:1090700019460446402250F05AF9402280212046E9
:10908000002350F054F9012384F81231D4F8E83564
:10909000A0785B689847002010BD38B54022044690
:1090A0000223812150F043F920460223402201216E
:1090B00050F03DF9204603230822822150F037F971
:1090C000084B0222002583F84B2083F84C50FFF711
:1090D00089F901212046044A402350F089FA2846A4
:1090E00038BD00BF00000020A02B002010B581215A
:1090F000044650F0F3F82046012150F0EFF82046E6
:10910000822150F0EBF8FFF779F9002010BD10B57F
:109110008121044650F0E2F82046012150F0DEF8AB
:10912000024B002083F8110210BD00BFF02900207F
:1091300070B5234D95F8832A012A03462FD1214E7D
:10914000D6F8144214B985F8834A24E0402C24D878
:109150000ABF0222A4B285F8832AD5F8881A1A4ACF
:109160000A44C3E9542240F201110022A3F8441139
:10917000C3E9564203F5A271184650F0A0F9D5F89C
:10918000883A2344C3F30A03C5F8883AD6F8143260
:109190001B1BC6F81432002070BD4024DDE7022AF4
:1091A000F9D1002440F20112C0E95444C0E9564408
:1091B000A0F8442100F5A27150F081F9C3E700BF87
:1091C000F8180020F02900208423002070B52B4ED1
:1091D000D6F818320F2B03F1010203D0C6F818227B
:1091E000002070BD264D0023C6F8183295F8833A4A
:1091F000002BF5D1D5F8882AD5F8843A9A42EFD0D9
:10920000D5F8882AD5F8843A9A4295BFD5F8844A89
:10921000D5F8884AD5F8883AC4F5006498BFE41AAE
:10922000402CC6F8144221D9012385F8833A402402
:10923000D5F8882A134B1344C0E9543340F2011285
:109240000023C0E95643A0F8442100F5A27150F074
:1092500036F9D5F8883A2344C3F30A03C5F8883AA7
:10926000D6F814321B1BC6F81432B9E70EBF02231E
:109270000123A4B285F8833ADAE700BFF029002081
:10928000F818002084230020064BD3F880391A797F
:10929000022A05D19A68920702D558694FF02EBD6F
:1092A000704700BFF818002010B50A4CD4F88009A8
:1092B00006F0B6FC58B9D4F880090379022B08D11E
:1092C00083689B0705D5BDE8104008F041B900BF91
:1092D000ECE710BDF818002073B50A4E441C0025B9
:1092E000D6F88009012300220DF1070150F0EBFDB3
:1092F0009DF80700FF2802D10135A542F0D102B048
:1093000070BD00BFF818002037B504460820019151
:10931000FFF7E2FFFF2813D0FE2813D10A4D019B6F
:10932000D5F880090022214650F0CDFD0022D5F865
:1093300080090223114650F0C6FD002003B030BD65
:109340000120FBE70220F9E7F818002037B5124D9D
:109350004FF6FF530024D5F88009ADF8043001AA78
:1093600002232146C5F84C4950F0ADFD0120FFF71E
:10937000B3FFFF2805D1042385F85039022003B03C
:1093800030BD092385F85039044BD3F89431C5F822
:1093900040392046F3E700BFF8180020F0290020EC
:1093A00013B540F040038DF800300B0E8DF80130FE
:1093B0000B0C8DF802300B0A8DF803309523044610
:1093C0008DF804108DF8053050F0A2FD00B964B995
:1093D00007480623D0F880096A46002150F073FD43
:1093E0000820FFF779FF02B010BDFF20FBE700BFA8
:1093F000F81800202DE9F041194C1E4694F8503918
:10940000042B0546884617461CD1FFF73DFF94F80C
:10941000463903BB69021120FFF7C2FFE8B90523F3
:1094200084F850390F4BC4F82C89D3F89431C4F820
:109430003059C4F83879C4F83C69C4F8403901207F
:10944000BDE8F081082B01D00020F9E7FFF77EFF8F
:109450000228F9D1D9E72946DDE7FFF725FFF3E731
:10946000F8180020F029002038B500220D233421FF
:10947000022006F033FF234CC4F8800910B984F8A9
:10948000500938BD002106F051FA012009F02CFFE7
:10949000D4F880391C4D586906F0FCFCD4F88039AA
:1094A0001A4893F91030142202FB03000022D0F86E
:1094B000B0000A23114650F0DBFCD4F8800906F016
:1094C000AFFB50B9124B84F84409D3F89431C4F877
:1094D0004039012384F85039D3E7013DEDD1D4F868
:1094E0008009022106F022FAD4F8800906F0F1F989
:1094F00094F84439C4F88059013384F8505984F8F9
:109500004439BEE7F8180020A186010000000020C1
:10951000F029002038B5134C0023A07BE0B125686A
:109520008D4219D1104C03F581751AB904EB05145D
:10953000A27138BD04F1180101EB43239A4209D10D
:10954000831E5842584104EB05144FF089FD012356
:10955000A371EEE70020F6E70133082B04F11004B5
:10956000DBD1E6E7DC5F0020C44F0020174838B5A8
:10957000002380F8A03000F1180425688D421ED128
:10958000A57B032D1BD1124C03F581754AB904EB61
:1095900005140423A371D0F89C300133C0F89C302B
:1095A00038BD04F1180000EB4320131A584258410B
:1095B00004EB05144FF054FD0123A371F0E70133D0
:1095C000082B04F11004D8D1EAE700BFC45F0020E3
:1095D000C44F002070B50446144EFFF798FD204696
:1095E0000223402281214FF0A2FE40220121204689
:1095F00002234FF09CFE0025D6F81C3286F811524B
:109600001B6886F8105228469847E06850F03AFAEE
:10961000E068012150F04CFA20461F2306F5F8724D
:1096200001214FF0E5FF284670BD00BFF029002062
:109630002DE9F84F0E460121084617461D4606F053
:10964000CFFFDFF844800024A54206DC0021012082
:1096500006F0C6FF0020BDE8F88F06EB442A04EBB5
:109660000709D8F8283903B9FEE7D3F804B0002376
:109670001A4651464846D8470028F2D0FEF728FF40
:109680000028FBD00134DFE7F81800202DE9F84F5F
:109690000E460121084615461F4606F0A1FFDFF8D9
:1096A00048A00024A74218DD06EB442905EB040876
:1096B00001E0FEF70DFFDAF8283943B1D3F80CB01A
:1096C00000231A4649464046D8470028F1D1FEF704
:1096D000FFFE0028FBD00134E4E70021012006F062
:1096E0007FFF0020BDE8F88FF8180020024BD3F868
:1096F000200207F054BE00BFF02900200068F022CD
:10970000FF2107F053BFCA4341EA02120068D2B2F8
:10971000D22107F04BBF0068B422FF2107F046BFFB
:109720000A460068A52107F041BF5521F8E7006807
:109730009622FF2107F03ABF0A460068872107F00A
:1097400035BFC90101F080020068782107F02EBF03
:1097500038B50446154600680A46E12107F026FFA1
:1097600030B120682A46FF21BDE8384008F014BE19
:1097700038BD0A46E121EBE70A46C321E8E738B5E0
:10978000021D0D46F0210446FFF7E2FF08B12379E0
:109790002B7038BDF8B504460E461546071D2068E7
:1097A0003A46FF2108F0F8FD30B116B12379DB0706
:1097B000F5D40DB123792B70F8BD00220121E9E722
:1097C00010B50446FFF7A7FF18B12046BDE81040CA
:1097D000F3E710BD10B50446FFF7A2FF18B120460D
:1097E000BDE81040E9E710BD70B506460C468D187F
:1097F000AC4201D1012006E014F8011B3046FFF70E
:10980000E9FF0028F4D170BDCC21E3E738B5044668
:109810000D46FFF78CFF40B12046FFF7CEFF20B189
:1098200029462046BDE83840A3E7002038BD70B582
:1098300006460C468D18AC4201D1012006E02146B7
:109840003046FFF7E3FF01340028F4D170BD38B58E
:1098500005461446FFF770FF2846FFF7AEFF20B11C
:109860001CB12B79C3F34013237038BD10B50446E7
:10987000FFF7A6FF38B12046FFF7C6FF18B1204614
:10988000BDE8104099E7002010BD73B50546CDE94D
:109890000023FFF795FFA8B12846FFF746FF88B1E0
:1098A0002846FFF78AFF68B16E46082416F8011BA8
:1098B0002846FFF78FFF28B1013C14F0FF04F5D1D3
:1098C00002B070BD0020FBE7C90138B501F080018E
:1098D00004461546FFF735FF08B9002038BD0022C1
:1098E00001212046FFF756FF0028F6D023795B09B7
:1098F0002B70F3E710B5021D0446FF21006808F045
:109900004BFD18B12079C04300F0010010BD0F4994
:10991000D1F8883043F47003C1F888300C4B1A68D2
:10992000002042F001021A6098601A6822F08472E6
:1099300022F480321A60074A5A601A6822F48022A0
:109940001A60D860044B8B60704700BF00ED00E0E8
:109950000038024010300024000000087047002842
:10996000ACBF00F16040074B4FEA0111ACBF00F5FE
:10997000614000F00F00C9B2B4BF195480F8001361
:10998000704700BF14ED00E02DE9F0479846414BC9
:10999000914603EB800205469468002C78D028336A
:1099A000636004F13E03A36104F59F73E3614FF428
:1099B0008073C4E90433236894F83D00E160A36335
:1099C00006F0DCFA064694F8440294F83CA0271D01
:1099D00008B14CF053FF94F8450208B14CF04EFF2B
:1099E000D4F840321BB12C4A116B0B43136318F0AF
:1099F000080F2CD00135EDB21EB140F20673F38092
:109A0000357218F0100F94F846221AD00221304611
:109A100006F074FAD4F8481294F94702FFF79FFF52
:109A200094F9473294F84722002B07DB02F01F011C
:109A300001228A405B09194941F823203846BDE8D4
:109A4000F08718F0200F14BF12213221DFE719F040
:109A5000020F0CD06B1CDBB21EB140F20652F2803A
:109A6000337294F846220221304606F047FA19F084
:109A7000010FCFD0504606F081FA0135EDB218B192
:109A800040F20663C380057294F846220221BFE7C4
:109A90002746D3E7542B06080038024000E100E0D7
:109AA0000148FEF7EABA00BF040100200148FEF7B2
:109AB000E4BA00BF50030020024B586FC0F300709F
:109AC000704700BF003802407047064A002352F832
:109AD0003310814201D1D8B2704701330E2BF6D139
:109AE000FE207047AC2B0608704770B5002828D0C0
:109AF0004C684CB9426815685679AB8902229BB212
:109B0000B24023EA0203AB818A683AB943681D6810
:109B1000AB8923F001031B041B0CAB81816044B1B2
:109B20004468216864798D890223A3402B439BB24A
:109B30008B8132B143681A6893899BB243F0010369
:109B4000938170BD0B4B30B51A4600241D798542B8
:109B500008D1DD68294203D0142000FB042030BD69
:109B60000029F9D001340A2C03F11403EED10020AE
:109B7000F5E700BF9805002038B503681B681C682E
:109B8000254B03F5CC6393ED007A07EE902AB8EEEF
:109B9000477AF8EE677A013987EE270A8DB2DFED52
:109BA0001F7A30EE270A51F0FDFF1D4A2388013845
:109BB000944280B29BB212D002F5806294420ED0E1
:109BC000B4F1804F0BD0A2F58032944207D002F559
:109BD0008062944203D002F58062944202D123F065
:109BE00070039BB20F4A944206D002F58062944201
:109BF0001CBF23F440739BB22380094BE5629C4257
:109C0000208503D003F580639C4201D10023238685
:109C10000123A38238BD00BF000000200AD7233CE7
:109C200000000140001000402DE9F0434568A8798C
:109C300010F0040300F002020BD00020174680460B
:109C4000042406466B79032B49D8DFE803F0094A60
:109C500089C990464FF480701F461C460126F1E7E3
:109C60002D682B8C23F001031B041B0C2B84B5F8EF
:109C700020C0B5F804902B8B23F073031B041B0C3E
:109C800043F0600E2CF0020C6E4B4FEA0C4C4FEA86
:109C90001C4C48EA06069D421FFA89F94CEA060C5C
:109CA00003D003F580639D420AD14FF6F3730CEAAB
:109CB00003033B4329F4407943EA040C40EA0909D1
:109CC000A5F80490A5F818E06963A5F820C02B8BCF
:109CD00023F008031B041B0C43F008032B83BDE88F
:109CE000F0832D682B8C23F010031B041B0C2B849A
:109CF0002A8CB5F804E0B5F818C0524B2CF4E64CA9
:109D000022F020024FEA0C4C12044FEA1C4C120CB9
:109D100048EA06069D421FFA8EFE4CF4C04C42EA09
:109D2000061203D003F580639D420BD122F080021E
:109D300042EA071222F040022EF4406E42EA041278
:109D40004EEA800EA5F804E0A5F818C0A9632A849D
:109D50002B8B23F400631B041B0C43F40063BDE74F
:109D60002D682B8C23F480731B041B0C2B842A8CF2
:109D7000B5F804E0B5F81CC022F400732CF0730CA5
:109D8000304A4FEA0C4C1B044FEA1C4C1B0C48EAAF
:109D9000060695421FFA8EFE4CF0600C43EA06233D
:109DA00003D002F5806295420BD123F4006343EAAD
:109DB000072323F480632EF4405E43EA04234EEA33
:109DC000001EA5F804E0A5F81CC0E9632B84AB8B4A
:109DD00023F008031B041B0C43F00803AB837EE74E
:109DE0002C68238C23F480531B041B0C2384258CA8
:109DF000A288A38B25F400552D0448EA06062D0CF5
:109E000023F4E64345EA06350E4E1B041B0CB44210
:109E100092B243F4C04303D006F58066B44203D146
:109E200022F4804242EA8012A280A3832164258426
:109E3000A38B23F400631B041B0C43F40063A38374
:109E40004DE700BF0000014043685A79032A0FD84C
:109E5000DFE802F00205080B186834307047186814
:109E60003830704718683C30704718684030704789
:109E70000020704710B543681A685879084B0344AE
:109E8000012093F8C840138CA0409BB223EA000342
:109E90001384138CA140194389B2118410BD00BFF3
:109EA000542B0608F0B5EFF31184102383F31288C6
:109EB000C5684668AA68136823F001031360326816
:109EC0007779104E938936F817609BB223EA060320
:109ED00093812A696D681F2A4FF0200385BF203ABD
:109EE00093409340EB6098BFAB60E3B283F311887B
:109EF000C3689B6859601A6842F001021A60012326
:109F00000374F0BD542B06080268137D012B04BFB7
:109F10000223137592F82C100CBF4FF4007300232A
:109F2000012904BF022182F82C1092F8441008BFC6
:109F300043F48063012904BF022182F8441092F89F
:109F40005C1008BF43F4006301290DD1022182F89F
:109F50005C1043F480534268116800224A628A8987
:109F600092B213438B8101E0002BF4D17047034B75
:109F70000348D3F82412FEF70BBD00BFF0290020E0
:109F80000000014010B5064C0648D4F82412FEF734
:109F9000FFFCD4F844120448BDE81040FEF7F8BCBA
:109FA000F0290020000001400040014010B5064C9F
:109FB0000648D4F82412FEF7EBFCD4F84812044803
:109FC000BDE81040FEF7E4BCF0290020000001408D
:109FD0000044014010B5064C0648D4F82412FEF7A0
:109FE000D7FCD4F84C120448BDE81040FEF7D0BCB2
:109FF000F02900200000014000480140034B4FF0D1
:10A000008040D3F82812FEF7C3BC00BFF02900201F
:10A01000024B0348D3F82C12FEF7BABCF0290020FB
:10A0200000040040024B0348D3F83012FEF7B0BCE6
:10A03000F029002000080040024B0348D3F83412F6
:10A04000FEF7A6BCF0290020000C00400348D0F821
:10A05000703613B100F264601847704700000020AA
:10A060000348D0F8903613B100F284601847704767
:10A07000000000200348D0F8B03613B100F2A4600D
:10A0800018477047000000200348D0F8D03613B1BD
:10A0900000F2C46018477047000000200348D0F861
:10A0A000F03613B100F2E46018477047000000205A
:10A0B0000348D0F8103713B100F204701847704706
:10A0C000000000200348D0F8303713B100F22470AC
:10A0D00018477047000000200348D0F8503713B1EC
:10A0E00000F2447018477047000000200348D0F881
:10A0F000703713B100F264701847704700000020F9
:10A100000348D0F8903713B100F2847018477047B5
:10A11000000000200348D0F8B03713B100F2A4705B
:10A1200018477047000000200348D0F8D03713B11B
:10A1300000F2C47018477047000000200348D0F8B0
:10A14000F03713B100F2E4701847704700000020A8
:10A150000348D0F8103813B100F6040018477047D0
:10A16000000000200348D0F8303813B100F6240076
:10A1700018477047000000200348D0F8503813B14A
:10A1800000F644001847704700000020036823F0E1
:10A19000010303600023036043608360C3600361C5
:10A1A000212343612A4B984203D13D2243F8082CD6
:10A1B0007047284B984204D14FF4746243F8202C26
:10A1C0007047254B984204D14FF4741243F8382C51
:10A1D0007047224B984204D14FF0746243F8502CE0
:10A1E00070471F4B984203D11E4A43F8642C7047B6
:10A1F0001D4B984203D11D4A43F87C2C70471C4BE1
:10A20000984203D11B4A43F8942C70471A4B98424A
:10A2100004D14FF03D5243F8AC2C17E0174B984255
:10A22000C3D0174B9842C7D0164B9842CCD0164B90
:10A230009842D1D0154B9842D6D0154B9842DAD0DF
:10A24000144B9842DED0144B9842E2D0704700BFC6
:10A2500010600240286002404060024058600240A6
:10A26000706002403D00002088600240400F0020E6
:10A27000A060024000003D20B8600240106402402F
:10A280002864024040640240586402407064024006
:10A2900088640240A0640240B86402402DE9F041A5
:10A2A0000022012603250B6806FA02FC3CEA0303A0
:10A2B00031D10368540005FA04FE23EA0E0303605B
:10A2C0000B79D0F800806FEA0E0703FA04FE013B19
:10A2D0004EEA080E012BC0F800E011D883681F4039
:10A2E00087604B798768A3403B438360436823EAD8
:10A2F0000C0343608B79476893409BB23B434360B8
:10A30000C36805FA04F723EA0703C360CB79C7687B
:10A31000A3403B43C3600132102AC4D1BDE8F081A1
:10A32000204A936803F00C03042B10B520D0082BAF
:10A3300020D01D4B1B4C0360A3681C4AC3F30313BE
:10A34000134493F864180368CB404360A168C1F3D9
:10A350008221114491F8641823FA01F18160A16807
:10A36000C1F342310A4492F86428D340C36010BD5F
:10A370000F4BDFE75368516813F4800F01F03F0182
:10A38000536814BF0A4A084AB2FBF1F1054A526801
:10A39000C2F30142C3F3881301324B435200B3FBB3
:10A3A000F2F3C7E7003802400024F4000000002068
:10A3B00040787D01F0B5446B8668A38923F400538F
:10A3C0001B041B0CA3818279278A0546BFB21003A8
:10A3D00012F0040F4FEA022100F400506A7927F4CA
:10A3E000405740EA0700208214BF4FF4805C4FF0D2
:10A3F000000C12F0010F0CBF002304239207A28966
:10A4000022F4B05201F4806122F00C0248BF43F004
:10A41000080341EA0C0112040B43120C1A43A281F7
:10A42000A38A23F440731B041B0C85B0A3826846E7
:10A43000FFF776FF214B9C4203D003F580639C42DB
:10A440003AD1039BA2891921170401FB03F34FF0B2
:10A4500064014CBF7600B600B3FBF6F3B3FBF1F03A
:10A4600001FB10330201A08900044BBFDB001B017C
:10A47000323332334BBFB3FBF1F3B3FBF1F303F0F1
:10A48000070303F00F0313439BB223816A6BAB797D
:10A4900013F0080F938A0BBF23F008039BB21B0431
:10A4A00043F0080308BF1B0C938293899BB243F4CB
:10A4B0000053938105B0F0BD029BC3E7001001403B
:10A4C0002DE9F8431E46204B9DF820509DF824703E
:10A4D0009842894690462CD13B462A463146002078
:10A4E000FFF752FA04460020C4E90700C4E9090056
:10A4F000C4E90B986571A660A7712046FFF75AFF63
:10A50000EA0707D5636B4FF6DF721A80DA6842F00C
:10A510002002DA60626BAB0742BFD36843F080036E
:10A52000D36093899BB243F4005393812046BDE8E6
:10A53000F883064B984204D13B462A463146012017
:10A54000CEE70024F2E700BF0010014000440040C5
:10A5500081602FE741712DE72DE9F043654F07EB4F
:10A56000C00985B005464FEAC00899F8780805F09B
:10A5700005FD064699F8790805F000FD044699F8AE
:10A580007A084CF07BF96B1CDBB21EB140F60C1262
:10A59000F28033721CB140F60C22E2802372042256
:10A5A0003A21304605F0AAFC204604223A2105F063
:10A5B000A5FC07EB0803D3F874484F4B9C4263D1CA
:10A5C00003F5F2331A6A42F400121A621A6A22F48C
:10A5D00000121A62474497F87B38022B6ED0032B87
:10A5E0006ED0464E464A012B08BF1646A78827F074
:10A5F0003F0768463F04FFF793FE3F0C029A414B2A
:10A60000B2FBF3F398B20743A780218821F0010140
:10A610000904090C21803C498E4253D13B4BB2FBCB
:10A62000F3F2013092B2042A80B238BF04222084AF
:10A63000A28323889BB243F001032380238823F461
:10A64000816323F002031B041B0C43F4806323800B
:10A650004FF480432381238823F080031B041B0CC9
:10A66000238023889BB243F001032380284B03EB14
:10A670004513012283F86122002283F8605283F897
:10A68000622205B0BDE8F083224B9C4209D103F55C
:10A69000F0331A6A42F480021A621A6A22F48002C3
:10A6A00097E71D4B9C4295D103F5EE331A6A42F4AD
:10A6B00000021A621A6A22F400028AE7124E95E733
:10A6C000124E93E706EB4606B2FBF6F291B2C2F3E6
:10A6D0000B020AB941F0010141F400424FF49671B6
:10A6E0004B434FF47A71B3FBF1F301339BB22384F4
:10A6F0009EE700BF0000002000540040801A0600C2
:10A7000000350C0040420F00A0860100400D030000
:10A71000F029002000580040005C00402DE9F0477F
:10A72000B74D460105EB401908F002FD99F960228A
:10A73000B44B8846D10003EBC2020746D2F87448F6
:10A7400099F86222013A142A00F28380DFE812F0BD
:10A75000790089009F00B700C200CC00D500EA0054
:10A76000F5000A01150164017D01A301060217022B
:10A77000290232024302670215005F184FF0090AEE
:10A7800097F8780805F0FAFB044697F8790805F081
:10A79000F5FBB5F8C03201339BB207462046A5F859
:10A7A000C03205F077FB384605F074FB11212046D6
:10A7B00005F07AFB1121384605F076FB4FF065086D
:10A7C00003E00520002108F0F3FC204605F059FBCA
:10A7D00010B9B8F10108F4D1204605F060FB002162
:10A7E000052008F0E5FC204605F054FB052000217B
:10A7F00008F0DEFCBAF1010AE0D1204605F04FFB7B
:10A800000021052008F0D4FC384605F048FB002163
:10A81000052008F0CDFC204605F03CFB052000217A
:10A8200008F0C6FC384605F035FBAB1993F9600219
:10A83000431C01D0FFF790FEAB19002283F862227F
:10A8400007E0238813F4007340F02381AA1982F8EB
:10A850006232AB1993F86232002B7FF465AFBDE82A
:10A86000F087238823F400631B041B0C23802388B8
:10A870009BB243F48063238023889BB243F48073AC
:10A880002380AB19C3E99A78032283F862225E49D8
:10A890002046FDF79AFCAB19002855D093F8722298
:10A8A0005AB993F87322FF2A04D193F870220AB19F
:10A8B0000A22C3E7AB190422C0E70F22BEE7AB1997
:10A8C00093F8712202F0FE022282C3E99A780522EF
:10A8D00083F862224D492046FDF777FC002800F0FE
:10A8E0007081AB190622A9E7AB1993F87322228273
:10A8F000C3E99A78072283F8622245492046FDF78A
:10A9000064FC002800F05D81AB19D3F874223AB9D9
:10A91000228892B242F400722280C3E99A780EE152
:10A9200008228BE723889BB243F480732380AB1902
:10A93000C3E99A78092283F8622233492046FDF759
:10A9400044FCAB190028B3D1D3E99A0142F210724A
:10A95000381A68EB0101904271F10002FFF479AFFF
:10A9600015226BE7AB1993F8712242F001022282A3
:10A97000C3E99A780B2283F8622226492046FDF724
:10A9800024FC002800F01D81AA19D2F87432012B92
:10A990001AD1238823F480631B041B0C2380EFF35C
:10A9A0001181102383F31288238B23889BB243F4F5
:10A9B00000732380CBB283F311880C2382F86232B8
:10A9C000AB19C3E99A7844E7022B15D123889BB2CF
:10A9D00043F400632380EFF31181102383F3128883
:10A9E000238B238823F480631B041B0C2380CBB2AE
:10A9F00083F311880D23E1E7238B0E23DEE700BFED
:10AA0000F029002000000020010003008200070060
:10AA1000840007000200030086492046FDF7E0FBA2
:10AA2000AB19002890D0D3F87822511CC3F87812C3
:10AA3000218A1170D3F87422013AC3F874220122DA
:10AA4000C3E99A7883F87C22F8E67B492046FDF733
:10AA5000C7FBF0B1EFF31182102383F31288238830
:10AA60009BB243F400732380AB19D2B2D3F87812AF
:10AA7000481CC3F87802208A087082F31188D3F842
:10AA80007822511CC3F87812218A11706FF00102EC
:10AA9000D3E7AB1958E768492046FDF7A1FBAB198E
:10AAA00000283FF451AFD3F87422032A03F51A713A
:10AAB00030D1228822F480621204120C2280EFF33B
:10AAC0001180102282F31288D3F8782202F1010C4F
:10AAD000C3F878C2B4F810C082F800C0228892B2DD
:10AAE00042F400722280C2B282F31188D3F8782235
:10AAF000501CC3F87802208A1070D3F87422023AEE
:10AB0000C3F874220C2283F86222C3F86872C1F879
:10AB100004809EE6022A14D8228822F4806212045D
:10AB2000120C2280228892B242F400722280228A81
:10AB3000C3F86872002283F87C22C1F804800122E5
:10AB40007CE6D3F87822501CC3F87802208A107073
:10AB5000D3F87422013AC3F87422D6E7238823F489
:10AB600080631B041B0C2380AB1993F8712202F045
:10AB7000FE022282C3E99A78102283F862222F49CA
:10AB80002046FDF722FBE0B1AB1993F87322FF2AB0
:10AB900004D193F870220AB113224FE6AB191122A7
:10ABA0004CE6AB1993F873222282C3E99A781222F9
:10ABB00083F8622222492046FDF707FB08B1AB1952
:10ABC000EAE720492046FDF70BFBAB1900283FF4CC
:10ABD000BBAE142232E6AB1903F51A70D3F8742217
:10ABE00082B1D3F87812013A11F801CBA4F810C061
:10ABF000C3F87422C3F86872C3F87812C0F80480EE
:10AC000012221BE6228892B242F4007222800122B4
:10AC1000C3F8687283F87C22C0F804800EE62388AB
:10AC20009BB243F4007323804FF6FF33A382AB192A
:10AC300073E600BF4000001004000010820007000F
:10AC4000840007000004001038B5114C04EB4014D8
:10AC500094F86152D5B1C4F87432049BC4F87832C8
:10AC6000002384F87C320223490084F8732284F89C
:10AC7000623201229DF8143084F8711284F8722235
:10AC800084F87032FFF74AFD94F87C52284638BDAC
:10AC9000F029002038B5114C04EB401494F86152AF
:10ACA000CDB1C4F87432049BC4F878320223490051
:10ACB00084F8732284F8623200229DF8143084F8FC
:10ACC000711284F8722284F87C2284F87032FFF7C3
:10ACD00025FD94F87C52284638BD00BFF02900209D
:10ACE000F0B587B0002300930193744B1A6842F4C7
:10ACF00080321A601A6802F400320192009A01321E
:10AD00000092019A1AB9009AB2F5A04FF2D11B68CD
:10AD100013F4003318BF01230193019B012B40F072
:10AD2000B180664B66491A6C42F080521A640A6818
:10AD300042F440420A609A689A609A689A609A68F7
:10AD400042F480529A605F4A5A601A6842F08072F8
:10AD50001A601A689201FCD55B4A40F202711160D8
:10AD60009A6822F003029A609A6842F002029A609E
:10AD7000524A936803F00C03082BFAD19368534CA2
:10AD800003F00C03042B7FD0082B7FD0504BC4F86A
:10AD900060364A4B4F4D9A684F48C2F30312224423
:10ADA000002692F88C18D4F86026CA40C4F86026B1
:10ADB0004A4AEA605A6F4A4AAA605A6B22F08002F5
:10ADC0005A635A6F42F080725A67196B454A0A43B8
:10ADD0001A635A6B5A631A6C42F0875242F4F612A5
:10ADE00042F41F6242F00F021A64596C3E4A0A4351
:10ADF0005A6402A948F2FF73CDE902364FF6FF7795
:10AE0000FFF74CFA00F580600297FFF747FA00F56C
:10AE100080600297FFF742FA00F58060FFF73EFA84
:10AE200000F58060FFF73AFA0846FFF779FA029BCF
:10AE30002E4AB3FBF2F32E4AC2F8C432D5F8FC30E6
:10AE40002C4A43F08073C5F8FC302B4BC3F8B02F6D
:10AE50005E601A6842F001021A60D4F860364FF45E
:10AE60007A72B3FBF2F3013BB3F1807F08D24FF06B
:10AE7000E0225361F02385F82330072396611361A4
:10AE800007B0F0BD00BFFDE71C4B80E75368516879
:10AE900013F4800F01F03F01536814BF174A0C4AA6
:10AEA000B2FBF1F1054A5268C2F30142C3F38813C1
:10AEB00001324B435200B3FBF2F368E70038024023
:10AEC0000070004019304004003C024000000020A7
:10AED0000024F40000ED00E0000002400003FA0549
:10AEE000000000081F9067003357070040420F0022
:10AEF000F029002055CEACC5001000E040787D015F
:10AF000082B000230193054B0193019B03EB80006A
:10AF10000190019B196002B0704700BF50280040AB
:10AF200082B000230193054B0193019B03EB80004A
:10AF30000190019B186802B0704700BF5028004084
:10AF400010B51C2005F01AF81121044604F0ACFFDE
:10AF5000204604F0A4FFC82008F0C6F92046BDE84A
:10AF6000104004F097BF436D064A1A61C278012A67
:10AF700006D100F2CC5058611A684FF080221A6056
:10AF8000704700BF1800086038B5044600296FD12B
:10AF900090F81131022B2AD1D0F83821D0F82411A1
:10AFA0008A4232D9C378012B04BFD0F828315B180C
:10AFB000A2EB010208BFC0F828314FF48071D0F82D
:10AFC0002831C0F83821002592B2A0F81C11C0F831
:10AFD0002C31C0F83451C0F8302100F58E714EF09C
:10AFE000F1F92B462A46294620464EF001FB94F8FB
:10AFF0001631012B07D1244A2369D2F8A4215A60C3
:10B00000002384F81631002038BDD0F83C31B3FB62
:10B01000F1F501FB1535A5B9994212D8D0F84021B8
:10B0200093420ED24FF48073C0E94A55C0E94C55A3
:10B03000A0F81C3100F58E714EF0C4F9C4F84051EF
:10B04000CFE7D4F8E435DB682BB194F81221032A5A
:10B0500001D120469847052384F81131002320466A
:10B060001A4619464EF0C4FA2046FFF77CFFBEE7A9
:10B07000D0F8E4355B69002BC5D090F81221032A83
:10B08000C1D19847BFE700BFF02900207047704743
:10B09000704710B5114C94F8D232CBB14FF0E0228A
:10B0A000D2F8103D23F00603C2F8103DFEF72FFC46
:10B0B00094F8D23263B1D4F8D8329B68DB0707D555
:10B0C000D4F8D423136823F0030161F3070313605A
:10B0D000034B4FF480225A6110BD00BFF0290020BD
:10B0E000003C01402DE9F04F974CD4F8D4325A6916
:10B0F000D0078DB000F1A4825A699B691340019377
:10B1000000F09E82C3F307430293019B190311D5FC
:10B11000D4F8D832DFF83C929E69DB6904F5327BC3
:10B120001E40360C04F547774FF00008DA46002E33
:10B1300040F01681029B5A070FD5D4F8D832834EBF
:10B140009F69DB691F40BFB2A6F118054FF00009E7
:10B15000A6F53878002F40F04881019B9DF80470D7
:10B16000980741BF784BD3F8D43202225A61019B31
:10B17000002B1BDA744D95F8D2323BB1D5F8D423AD
:10B18000136823F0030161F307031360D5F8D82295
:10B190006F48536823F0010353606E4BD3F8B43803
:10B1A0009847D5F8D4324FF000425A61019B1905F7
:10B1B000C3F3072631D5644D00238DF81F3095F871
:10B1C000DA338DF81F30634B05F53270D3F8B038A1
:10B1D0009847D5F8D422D5F8D8324FF400619B684F
:10B1E000516195F8D222C2B1DA0716D595F8DD3350
:10B1F000012B12D19DF81F30032B0ED1D5F8D4337B
:10B200001A6842F001021A601A6842F003021A60DA
:10B21000514A136943F0060313613B070AD54A4DAF
:10B220004C4B05F53270D3F8A8389847D5F8D4328E
:10B2300008225A61FD0615D5434BD3F8D402826922
:10B2400022F010028261026AC2F34341022902F035
:10B250000F0500F08681062900F0AA81836943F07A
:10B2600010038361F00637D5374DD5F8D822D5F8CD
:10B27000D4025368002723F00103536039464EF08F
:10B2800017FCB84695F8C9023B4605F53875FF210D
:10B290008342C0F09B81D4F8D8322D484FF0FF3262
:10B2A0009A614FF00112DA610B2262F3070762F331
:10B2B00007085F61C3F810801A686FF30A121A60FA
:10B2C000FFF751FED4F8D43221484FF480525A612E
:10B2D000204BD3F8AC389847B10640F193811A4C13
:10B2E000D4F8D832D4F8E00299680268C1F3410179
:10B2F000022906BF032161F30A026FF30A0202600A
:10B300005A6842F480725A6008A8FFF709F8D4F826
:10B31000D412D4F8D802CB68099A6FF38D23CB608E
:10B3200085680E48C5F34105284490F8CC000328F1
:10B3300040F05381002284F8CA224FF40072A4F82E
:10B34000CC22092258E100BFF0290020D02C002097
:10B35000B82C00200000002000ED00E0542B06086F
:10B36000F2073BD55FFA88F104EB8103D3F81C3375
:10B370009D68D4F8D8325B691D40EB0720D594F85E
:10B38000CB023B680125A8429D6007D11869DBF814
:10B390007C33C0F312001B1ACBF88C33D9F89C38DD
:10B3A0005046984794F8CB32012B09D1B8F1000FE1
:10B3B00006D194F8D933052B02D15046FFF7D3FDBF
:10B3C000A80742BF3B6802259D60290706D5D9F82A
:10B3D000A438504698473B6808229A6008F1010853
:10B3E000760804370BF1280BA1E6FB0779D5D8F8CE
:10B3F000D8325FFA89FA1969586B08EB8A0220FA89
:10B400000AFBD2F8E0224FEACB1B92685FFA8BFB73
:10B410004BEA010B0BEA020B1BF0010F1ED05A6B1B
:10B42000A8484FF0010B0BFA09F122EA01025A6316
:10B430003368C3F808B0A44B5146D3F8A0389847F6
:10B4400098F8CB325B4509D1B9F1000F06D198F8D5
:10B45000D933042B02D19B48FFF785FD1BF0080F61
:10B460001EBF33684FF0080BC3F808B01BF0100F75
:10B470001EBF33684FF0100BC3F808B01BF0400F2D
:10B480001EBF33684FF0400BC3F808B01BF0020F2B
:10B490001EBF33684FF0020BC3F808B01BF0800FDB
:10B4A0001FD0D5E94C329B1AD5F82421D6F800E0FC
:10B4B00098F8CBB2DEF81800934228BF1346033346
:10B4C000D8F8D82203929B080AF1320A049308EBB9
:10B4D0008A0A049B80B2984203D9D5E94C0398426A
:10B4E00005D809F101097F080436283532E6C01A6B
:10B4F000D5F82431984228BF1846C31C9B080493F2
:10B50000BBF1000F1BD0D5F82811D5F83421014428
:10B51000C5F82811D5F8301102448A42DEF8180027
:10B52000C5F83421D5D1039B95F81C115A6B012322
:10B5300003FA01F1039B22EA01025A63C9E782B2CE
:10B54000DAF8D012D5F828C10332931005930A46D1
:10B550005946059B8B42D6D05CF8213013600131EF
:10B56000F7E747F6F07111423FF478AE282101FB6E
:10B570000531C2F30A12D71CD3F898E3D1F848C6B4
:10B58000BF1000218F420DD1282101FB0533D3F8D4
:10B5900048161144C3F84816D3F854160A44C3F8A1
:10B5A00054265BE6DEF800804CF821800131E9E7A3
:10B5B000D3F898130F68C3F894780968C3F89818FB
:10B5C000282101FB0533C2F30A12E5E755F8042BE5
:10B5D0009160AA6B013391605AE6012084F8CA0297
:10B5E0004020A4F8CC02A0F56400384CA0F56240DD
:10B5F0001044A04227D80E2262F38D23CB604FF473
:10B6000000534B61029BDA060BD5314C2E4B04F5EF
:10B610003270D3F8B8389847D4F8D4324FF4801247
:10B620005A61029B9B060BD5294C274B04F53270BF
:10B63000D3F8BC389847D4F8D4324FF400125A618A
:10B640000DB0BDE8F08F234CA2F57400A0F51050AA
:10B65000A04201D80D22CFE71F48204C1044A04241
:10B6600001D20C22C8E71E4CA2F18C70A0F5434019
:10B67000A04201D80B22BFE71A481B4C1044A0423D
:10B6800001D20A22B8E71948194C1044A042FFF42D
:10B6900058AE184CA2F1B770A0F55850A04201D294
:10B6A0000822A9E71448154C1044A04201D20722F1
:10B6B000A2E713481044134A904234BF06220522E1
:10B6C0009AE700BFB82C0020000000203F420F0086
:10B6D000F0290020DFC810002013FBFE20D6130045
:10B6E000FF69180000D3CEFE40771B00C05BB3FE9D
:10B6F000C091210040AC2700C01D6AFE40E133002C
:10B70000803C36FEE09C4100034BD3F87C0908B135
:10B7100004F0B7BB01207047F818002008B5FFF708
:10B72000F3FF0A4A18B9002382F8503908BD92F88D
:10B7300044390133DBB2072B82F84439F3D8044B88
:10B74000D3F89431C2F840390123EDE7F81800200E
:10B75000F02900202DE9FF47CC4CD4F880090028BF
:10B7600067D0CB4DCB4E04F66C1794F85039013BA3
:10B77000082B46D8DFE813F009006000EC00450014
:10B78000C4014B01A0014500FF01FDF77DFD002133
:10B790000846FDF705FE8046FDF786FDB8F1010F6E
:10B7A0002AD14FF0000984F84599FDF76DFD40F26C
:10B7B000AB110820FDF7F4FD05280AD184F845896E
:10B7C000FDF772FD94F84539A3B1022384F850398E
:10B7D000CBE70128F4D10423D4F880094A4669460E
:10B7E0004EF071FB9DF80330AB2B04BF022384F8AD
:10B7F0004539E5E784F85039D4F88009022104F08E
:10B8000095F894F85039013B022B09D8A04BD4F895
:10B810004029D3F894319B1AC82B01D9FFF77EFF3A
:10B8200094F85009042800F0B681A0F108035842AA
:10B83000584104B0BDE8F087FDF726FD94F845397E
:10B84000022B0CBF4FF080484FF00008002137203A
:10B85000FDF7A6FD41462920FDF7A2FD8046FDF734
:10B8600023FDB8F1000FC7D194F84539022B39D127
:10B87000FDF70AFD41463A20FDF792FD042381467B
:10B880004246D4F8800969464EF01DFBFDF70CFDD9
:10B89000B9F1000F02D0FFF741FF66E7009B1BBA2A
:10B8A000C3F3807384F84639FDF7EEFC00210920CC
:10B8B000FDF776FD98B910213846FDF725FD814644
:10B8C00068B901217F204AF041FE0128804606D157
:10B8D000022148464AF03AFE38B101282CD0FDF743
:10B8E000E3FC89E784F84689DEE704212C204AF04E
:10B8F0002DFE032182464E204AF028FE0C2181466F
:10B9000036204AF023FE09F10202411C01FA02F23C
:10B9100008FA0AF3A2FB03385B0A43EAC853C4F8E7
:10B920005439FDF7C1FCFDF7AFFC00210A20FDF7FB
:10B9300037FD50B9032349E716213A204AF006FEA5
:10B9400001308002C4F85409EBE7FDF7ADFCA2E733
:10B9500010216846FDF7D8FC00287FF44DAF9DF814
:10B96000003084F85A39BDF801305BBAA4F8583970
:10B970009DF8033084F85B399DF8043084F85C3915
:10B980009DF8053084F85D399DF8063084F85E39FD
:10B990009DF8073084F85F399DF808301A0903F0E4
:10B9A0000F0384F86539DDF8093084F864291BBA7F
:10B9B000C4F860399DF80D309DF80E201B01DBB2F4
:10B9C00043EA121303F5FA6302F00F02A4F8663992
:10B9D00084F86829FDF768FC94F846394BB1D4F82F
:10B9E0008009022103F0A2FF0023C4F84C3904238C
:10B9F000ECE6FDF749FC4FF400711020FDF7D0FC98
:10BA00008046FDF751FCB8F1000FE8D043E794F809
:10BA10003419D4F82C29D4F88009802302EBC11200
:10BA200000214EF050FA94F834390133DBB2042B84
:10BA300084F834397FF4E5AED4F880090223324625
:10BA400000214EF040FA0123D4F880090022694613
:10BA50004EF039FA9DF8003003F01F03052B1BD17F
:10BA6000072384F850390A4BD4F83859D3F8943165
:10BA7000C4F84039002D3FF4C4AED4F83C39D4F8B2
:10BA80002C29D4F830190120A847BAE6F81800206C
:10BA9000F0290020242C0608FFF740FED4F838894E
:10BAA000B8F1000F3FF461AED4F83C39D4F8301946
:10BAB00000220120C04758E64EF02AFA002861D043
:10BAC000002384F84439D4F84C39012B0BD9013BBD
:10BAD000C4F84C39D4F848390133C4F8483908233C
:10BAE00084F850398DE607D1FDF730FC02287FF449
:10BAF00088AEFDF7D9FB84E6042384F85039F8E7D3
:10BB0000D4F82C094FF40071FDF7FEFB01288046A4
:10BB100018D002281ED000287FF473AEFDF7C4FBB6
:10BB2000D4F8385984F84489042384F85039002D16
:10BB30003FF467AED4F83C39D4F82C29D4F8301946
:10BB40004046A1E7D4F84039D5F8942164339342B4
:10BB5000BFF457AEFDF7A8FBFFF7E0FDD4F8388936
:10BB6000B8F1000F3FF401AE0022D4F83C39D4F80C
:10BB7000301910469EE74EF0CBF918B1FDF794FB53
:10BB80000423ADE7D4F84039D5F89421FA33934231
:10BB9000FFF481AE35E601204BE62DE9F341294C57
:10BBA00005460E4690461F4694F85039042B0BD09C
:10BBB000082B07D1D4F84839AB4219D0FDF7C6FBA2
:10BBC0000228F1D001200EE0FDF75EFB94F8463923
:10BBD00063B969021820FDF7E3FB48B1FDF764FB88
:10BBE000FFF79CFD032002B0BDE8F0812946F1E794
:10BBF00094F85039D4F88009082B0CBFFC23FE239D
:10BC0000FF228DF804208DF8053001AA02230021BF
:10BC10004EF059F9D4F880098023324600214EF0C5
:10BC200052F9012384F834390623C4F82C69C4F886
:10BC30003059C4F83889C4F83C7984F85039002068
:10BC4000D1E700BFF818002070B51C4C94F85039AB
:10BC5000042B05460E4610D1FDF716FB00213720B8
:10BC6000FDF79EFB31461720FDF79AFB90B1FDF7DB
:10BC70001BFBFFF753FD032002E0082B01D001203E
:10BC800070BDD4F84839834214D0FDF75FFB022819
:10BC9000F5D1E1E794F8463973B969021920FDF747
:10BCA0007FFB0028E3D1082384F85039C4F84C699D
:10BCB000C4F848590220E3E72946EFE7F8180020C6
:10BCC000044B054A03F6C801D3F8C838C2F828194E
:10BCD000184700BF00000020F8180020002108B518
:10BCE000084604F07DFCFFF7EBFFFCF7F1FB0028B2
:10BCF000FBD00121002004F073FC002008BD034BA1
:10BD0000D3F8280908B1436918477047F81800208C
:10BD1000034BD3F8280908B183691847704700BF5F
:10BD2000F8180020034BD3F8280908B1C369184755
:10BD3000704700BFF818002038B50D461446FFF7CD
:10BD4000F1FF03682B604FF400732360002038BDBF
:10BD5000034B1B78032B0CBF80204FF4807070477F
:10BD6000C44F002008B50B4A68B1816811B10723A0
:10BD7000937008BDFFF7ECFFC2E90311C2E90100AF
:10BD800011750423F4E702F58051012381F8B431E1
:10BD90005370EEE7C44F002010B502784368022AC2
:10BDA0000B4A06D1D2E9800100EB410000EB5320A1
:10BDB00010BD0169D2F81802D2F8104218400239B9
:10BDC000D2F80C32400A04FB01001844F0E700BF2F
:10BDD000C45F0020074B1B78022B0BBF030AC0F384
:10BDE000D413C0B200F07F000CBF0B600B6010607A
:10BDF000704700BFC44F002090F91A305A1C0AD077
:10BE000003F58172124B03EB0213DA796FF3000230
:10BE1000DA71FF23837690F91B104B1C16D00C4A65
:10BE200001F5817102EB011302EB0112DB79D1798B
:10BE3000C3F34503012B86BF03F1FF3303F03F0338
:10BE4000002363F34601FF23D171C376704700BF1F
:10BE5000C44F002008B5FFF77BFF034BD3F8103227
:10BE60005843400208BD00BFC45F00200378022B86
:10BE700009D10D4BD3F820224368B3EB422F2CBFDE
:10BE8000012000207047006960B1084B1B78032B2C
:10BE90000EBF074B80B24FF6F773984294BF002055
:10BEA0000120704701207047C45F0020C44F00206C
:10BEB000F7FFFF0FF7B50D464168C1F308032B44A8
:10BEC000B3F5007F044603D22944616001202EE0CF
:10BED000FFF792FF0378022B01D16168F4E7164B5C
:10BEE000D3F81022B5EB422F4FEA422721DCD3F8DA
:10BEF000183246681E407342AB421ADCAB19BB4293
:10BF000010D30169007E01AA4DF07EF9012810D1FD
:10BF100023696361019B236163683B449B1BED1BA9
:10BF2000636035442046FFF7A1FF0028D5D003B059
:10BF3000F0BD0020FBE700BFC45F002070B50446E1
:10BF40000E461546FFF7B6FF20B10DB12046A847B3
:10BF5000012007E094F82800022320B9C4E90B5619
:10BF600084F8283070BD1846FCE7054A92F8B411F1
:10BF7000012309B982F8B431024A5370704700BFF7
:10BF8000C45F0020C44F002008B5074BC31A48BF48
:10BF900003F2FF13B3F5805F4FEA632003D3FFF78B
:10BFA000E4FF4FF0FF3008BDDC4F00202DE9F74FD4
:10BFB00012F0020B0191174600F0D180002840F0EA
:10BFC000CE80FFF7D2FF02266EE04FF0FF36DFF89B
:10BFD000C4C1DFF8ACA1B6463446B1460025DCF852
:10BFE00000109CF80E8088421BD1B8F1000F00F0C1
:10BFF0009880D2F89840624E0134C2F8984005F516
:10C0000081721201B4502C465D4D04F5817805EB28
:10C0100008129679042ED4D8DFE806F0315DB05DC1
:10C020006700B8F1000F26D0B8F1010F14D105F563
:10C0300081780AEB081898F8078018F0010F0BD1E7
:10C0400018F07E0F08D15FEAD81116D1DCF808800D
:10C05000C14501D9AE46C1460135082D0CF1100C81
:10C06000BDD1751C79D1611C5CD1BEF1FF3F00F0E0
:10C070008580744656E02E46EEE72C46ECE717F036
:10C08000010215D03F4BD3F82839002B76D03E491A
:10C090005F683E4A002301EB4421B84700286DD079
:10C0A00005EB08150223AB71304603B0BDE8F08FF5
:10C0B00005EB0810FE1090F807C0032B66F3C71CB1
:10C0C00080F807C02BD94FF6FF72934228BF134662
:10C0D00005EB08129380BBF1000F06D005EB0410AE
:10C0E00000F580501830FCF715FA7A0741BF05EBD0
:10C0F0000812D37943F00103D371FB0608D505EB91
:10C100000815EB79C3F34502013262F34603EB7184
:10C110001D4B019A03EB442313600126C4E7134629
:10C12000D6E72C46164E41F2180506EB041C4CF8D7
:10C130000500D2F898500135C2F8985041F21C021F
:10C140004CF8025004F581724FEA021C06EB021211
:10C1500046F80C500025556056E73446E2E70C4A95
:10C16000D2F80862002E3FF430AFD2E9834505FBD8
:10C170000644A042FFF429AFFFF7F7FE002693E73D
:10C18000C44F0020F8180020DC4F0020159500084F
:10C19000C45F0020DC5F00207FB50F4D01AA0C4674
:10C1A00002A9FFF717FE05F58053029ED3F800029F
:10C1B0000322002303A93044FFF7F8FE012808D129
:10C1C0002978039B019A02290CBF23F8124043F8F7
:10C1D000224004B070BD00BFC44F00202DE9F047DD
:10C1E0000D4686B0164604A903AA07462868FFF73D
:10C1F000F1FD364A0499D2F8003201EB0308039BA3
:10C20000013B9C19FFF7A4FD2B68E41A0444A2F536
:10C21000805AB4FBF0F408EB04092968B142A9EB99
:10C22000080303D3012006B0BDE8F087039A019309
:10C23000FFF78EFD9419641A8442019B28BF0446BF
:10C24000002A35D1A04294BF0A220B2205A94046FC
:10C25000FFF7ACFE0128E6D19AF800002A6805999C
:10C26000039B022802F101022DD1A34222D32B68A5
:10C27000039A9B1A2344012F2B6014D1B34212D18D
:10C2800002280BBF04F1004404F1804304F1FF34A1
:10C2900003F1FF330BBF4FF6FF734FF0FF3221F86E
:10C2A000143041F82320002308F101080393B4E778
:10C2B0000B22CBE721F8132001330132D5E741F8F7
:10C2C000232001330132A342F9D3D0E7C45F002019
:10C2D0002DE9F04F85B08346FFF73AFD0C46164630
:10C2E000814601AA206802A9FFF774FD0BF1FF3314
:10C2F000012B68D9019B63B94D46DFF8D080BBF1B3
:10C30000010F8CBF4FF0000B4FF0010BA8F5805AC6
:10C310001BE0FFF72AFE02202AE0D8F87821C2B1FC
:10C32000D8F89401884214D1D8F81032013A590251
:10C3300002EB4323B3FBF1F30344B3FBF5F205FB3C
:10C3400012320AB12B449B1A23602168B142E4D314
:10C3500029E0D8F80002029F0023092203A93844EB
:10C36000FFF724FE012806D00228D4D00028ECD103
:10C3700005B0BDE8F08F9AF800200399022A07D093
:10C38000032AC8D1019B51F8233023F0704302E007
:10C39000019B31F813302768B3FA83F35B095B45DF
:10C3A00004D1BE42E4D826600320E1E7019B2B4480
:10C3B0002F444B4527600193E0D3029B0133029346
:10C3C00000230193C1E7012597E700BFC45F002068
:10C3D00037B50446C0690D4698B10023032201A970
:10C3E000FFF7E4FD012806D1B4F92030002B0ADA6A
:10C3F000FFF7BBFD022003B030BDE5255554A26810
:10C400000BE00120F7E7019A012D4FEA431102EBFF
:10C410004313F4D0022DF0D0E268DA612278032AC7
:10C4200004D100221A775A779A77DA77626A5A83A8
:10C43000110C9982DFE770B5304D0446042694F85C
:10C440003430052B2CD8DFE803F003243139424B7C
:10C45000D5F8082204F1300102320120FFF738FF3D
:10C46000012807D00238C0B2012819D8052384F862
:10C470003430E4E7D5F81012E268236BC5F81432C3
:10C4800002EB4122E260E26A236102B963620123A6
:10C49000EDE7206B4FF0FF31FFF77EFE012801D062
:10C4A000002070BDE36A3BB10223E0E7D4E90B0151
:10C4B000FFF772FE0128F3D10323D8E700212046BD
:10C4C000FFF786FF0128EBD184F83460B7E794F8D2
:10C4D0002830082B02D1002384F828300120E0E71F
:10C4E00094F82830082B04BF002384F82830034B2D
:10C4F000012283F8B5210220D3E700BFC45F0020EA
:10C500002DE9F743DFF81891044694F83850032DCD
:10C5100000F28180DFE805F002106E772046FFF719
:10C520008AFF012802D184F83800EEE7022873D18F
:10C53000032384F83830E8E723786668022B18BFB5
:10C54000D9F81832204618BF1E40FFF725FCC6F365
:10C550004F260746361A0023022201A93846FFF764
:10C5600025FD06EB070801281FFA88F8054653D178
:10C5700001984FF40072002154F0C0FAE369FBB156
:10C580006368EBB9019B4FF020322E211A605A608C
:10C590001970C3F80720606A5883050C10201A62CE
:10C5A0005A6283F8201083F82110D872C3F827202C
:10C5B000E26B9D8222FA00F199865A8783F82B005C
:10C5C000D9F810124B1E984508D24FF4007120463E
:10C5D000FFF770FC4CF044FD0137BCE7C1EBC151E3
:10C5E000490201F500712046FFF764FC4CF038FD6C
:10C5F00002239EE7002384F82830236C0BB12046E9
:10C600009847012508E0236C002084F8280003B136
:10C610009847022500E00025284603B0BDE8F083D6
:10C62000C45F0020F8B52E4E044600F13007A6F591
:10C63000B87594F83830032B50D8DFE803F0022E99
:10C64000363FD5F894212261FFF704FCE3681844D3
:10C65000E060FFF77DFB1044C5F89401FFF7FAFB9B
:10C66000D5F87831181AC5F87801FFF7F3FBD5F83B
:10C670007C31181AC5F87C012263FFF769FBE36A75
:10C680001044606323B96262012384F83830D0E734
:10C69000FFF75EFB101A2063F6E700213046FFF734
:10C6A00097FE01280ED10223EFE7626B3946012085
:10C6B000FFF794FD012805D10323E6E7002120467A
:10C6C000FFF786FE431EDBB2012B06D894F8283014
:10C6D000062B04BF002384F82830F8BD0220F1E7C0
:10C6E000346100202DE9F743454D0029044614BF6D
:10C6F0000226002605F5805794F83C30042B71D8AB
:10C70000DFE803F0290336406300DFF8FC802B7874
:10C71000206B032B53D1404594BF4FF000094FF0DD
:10C720000109B9F1000F48D101A949F0EBFE012838
:10C7300063D1206B4946FFF72FFD01285DD1019B96
:10C740002363D7F81422013B934294BFC7F81432F5
:10C75000C7F81422DBE731462046FFF739FE0128EF
:10C76000034648D1626B02B1022384F83C30C3E730
:10C77000626B04F130010020FFF730FD01283AD14F
:10C780000323F2E7E26AD7F89431C7F894219B1AA1
:10C79000D7F810221B485343D7F8782102EB4322E5
:10C7A000C7F87821D7F87C21002102EB4323C7F892
:10C7B0007C31FFF70DFE01281DD10423D5E71FFAB8
:10C7C00080F94FF6F7739945A6E794F82830042BC3
:10C7D00004BF002384F82830A36B0BB12046984790
:10C7E00001200AE0022094F82830042B05D1002310
:10C7F00084F8283001E00228F5D003B0BDE8F083CA
:10C80000C44F002034610020F7FFFF0F70B503789C
:10C81000023B012B04461CD8237E990623D42046D4
:10C82000FFF7EAFA237E1A070AD51F4D95F89801FB
:10C83000C31F584258414CF013FC002385F898312F
:10C840000023237084F82830E36A5BB1BDE87040B0
:10C850001847037E13F0060FDED00121FFF7B8FD65
:10C860000128D9D070BDE269104900231801405851
:10C87000824211D10E4903F5817201EB0213DB797B
:10C88000C3F34503012B0BD8002301EB0212D1792E
:10C8900063F34601D171C2E70133082BE6D1BEE74D
:10C8A000013B03F03F03F0E7C45F0020DC5F0020A2
:10C8B000C44F002010B580B1027872B190F82820E2
:10C8C0006AB9D0E9012494422CBF846082600322BB
:10C8D00080F82820C162FFF799FF012010BD0020D9
:10C8E000FCE7B1F904300F2B2DE9F34104460D4666
:10C8F00016460BD14FF40071FFF7DCFA18B900208F
:10C9000002B0BDE8F0814FF6FF73AB802046FFF721
:10C9100043FA94F91B20531C074611D01E4B41F2D9
:10C92000180103EB021041588F4230D0FFF71DFB76
:10C930002046FFF79BFA0028E1D00023336024E073
:10C940002046FFF793FA80460028F1D1381E18BF21
:10C9500001204CF085FB4346112201A93846FFF720
:10C9600025FB0128E4D10198FFF70EFBE076019A40
:10C97000002ADDD0AB8801331BB2AB8002EB43133E
:10C9800033602046FFF708FA28600120B8E7183323
:10C9900003EB42230193EAE7C44F00202DE9F04165
:10C9A0004FF0FF31304A314C0D46002310780428F7
:10C9B0000ED103F5817004EB0010C079C70707D4CE
:10C9C0006E1C52F80A0C01D0884201D21D46014665
:10C9D0000133082B02F11002E8D16B1C42D0234C2A
:10C9E000234E05F5817704EB0713998849B1D6F8F2
:10C9F000283933B104EB051041F218029B688058C6
:10CA00009847D6F828399BB11A4ED3F80C801A4AA9
:10CA100004EB051C41F2180000235CF8000006EB53
:10CA20004521C04720B1022810D00020BDE8F08188
:10CA3000124BD3F89C2004EB0714013AC3F89C2056
:10CA40000322A271012283F8A020EEE706F6E87621
:10CA500004EB0714D6F89C30013BC6F89C30012348
:10CA6000A371E2E70120E1E7EA5F0020C44F002064
:10CA7000F8180020DC4F00206D950008C45F0020EE
:10CA800008B500214422104854F038F80F4B03F544
:10CA900080501B784FF6FF72A0F8D221022B4FF086
:10CAA000030218BF134680F8B831D0F81C32C0F822
:10CAB000DC31102380F8D02180F8D13100F5DC7012
:10CAC00049F00EFF012008BD7C610020C44F00200A
:10CAD00070B5124D124BC5F8BC3840F2011200235C
:10CAE00085F81132A0F84421C0F85C3105F6BC028B
:10CAF0000D23C0E95422044685F8C818C0F85831FF
:10CB000000F5A2714CF0DBFC05F5F87220461F23FE
:10CB1000BDE8704001214CF06BBD00BFF029002042
:10CB20005553425310B5074B93F8FD1104464CF092
:10CB30007DFD002804DA20460121BDE81040C7E74A
:10CB400010BD00BFF0290020F8B50B7813F0600588
:10CB500006460C4638D0202D74D14A78FE2A05D0DE
:10CB6000FF2A1CD04CF0ACFB02252BE04D88A5B968
:10CB7000CF88012F11D11A060FD5334CD4F81C32AF
:10CB80009B699847C0B284F8CC0830B13A4604F6A5
:10CB9000CC0130464CF068FC14E03046E2E74A88AD
:10CBA000002AFAD1CD88002DF7D11B06F5D4264AEC
:10CBB000012182F8115282F810121F2302F5F87237
:10CBC0004CF016FD2846F8BD4B780A2B24D00B2BD1
:10CBD00025D0012BF6D194F904308988C068002B48
:10CBE00022DA01F07F014CF063FF2179164F3046C5
:10CBF0004CF074FB02232179402230464CF097FB25
:10CC000097F81032022B12D1812130464CF026FBCE
:10CC1000002387F81032D5E70C490122BAE70A4B06
:10CC20004A8883F8CD28CDE74CF02CFFDDE794F956
:10CC30000420002AC6DA012BC4D001213046FFF7B8
:10CC400047FFBFE70025BDE7F0290020BD320020E7
:10CC500008B5084B93F81132022B07D0033B012B88
:10CC600002D80021FFF734FF002008BDFFF75AFF6C
:10CC7000FAE700BFF029002070B52F4C94F811623C
:10CC800005461EB1012E54D0002070BDD4F8F431F9
:10CC9000C4F8C038D4F8F831C4F8C438B0F8B433A4
:10CCA0001F2B0DD1D4F8F021244B9A4208D194F8CF
:10CCB000FD11012904D894F8FE31013B0F2B0AD94C
:10CCC0002021052049F06CFB022384F8103228460D
:10CCD000FCF7A8F9D8E74CF0A9FC0028F7DB94F89A
:10CCE0001132013B022BCFD9B4F8CE18E9B1D4F8F8
:10CCF000F83184F8C868994228BF1946D4F8C43876
:10CD00005B1AC4F8C438042384F8113240F20113CA
:10CD1000A5F844310A4BC5E95616C5E9543305F563
:10CD2000A27128464CF0CBFBAEE72846FFF7D0FEB9
:10CD3000AAE7FFF7F7FEA7E7F02900205553424383
:10CD4000C43F0020F0B59C0827010E46154600EBB5
:10CD50000414A04206F1100605F1100508D103F0F5
:10CD6000030339443A4404EB83039C4223D1F0BDCE
:10CD700084469CED006A16ED045AD0ED016A56ED2A
:10CD8000037A90ED027A56ED025A26EE056A66EEB7
:10CD9000A76AD0ED037A05ED046A16ED016A45ED48
:10CDA000036A27EE257A67EE867A103005ED027A5F
:10CDB00045ED017ACDE7F4EC017AB1EC017A67EE4A
:10CDC000877AE2EC017AD0E74A09012301F01F01DA
:10CDD00003FA01F150F82230194214BF012000205B
:10CDE00070474A09012301F01F0103FA01F150F8CD
:10CDF00022300B4340F8223070474A09012301F0EA
:10CE00001F0103FA01F150F8223023EA010340F830
:10CE10002230704780EA0120082341F2210210F4F9
:10CE2000004F4FEA400018BF5040013B80B2F6D19E
:10CE3000704738B50C468D18AC4200D138BD14F897
:10CE4000011BFFF7E7FFF7E74840082310F0800FCA
:10CE50004FEA400018BF80F0D500013BC0B2F5D1C9
:10CE6000704710B50A440C46944200D110BD14F826
:10CE7000011BFFF7E9FFF7E738B50A4605680446E6
:10CE80000020AA4203D36B1C2360287038BD12F81F
:10CE9000011BFFF7D9FFF4E7DFED0A7AC0ED020AC4
:10CEA00020EE270AB7EE007AC7EE007A002303606F
:10CEB000C0ED017A70EEA77A80EEA77A80ED037A52
:10CEC000704700BFDB0FC94090ED017AD0ED007ACA
:10CED000C0ED020A30EE877AC0EE876A30EE677ADC
:10CEE000E6EE877AB0EE670AC0ED007A704701235C
:10CEF00003700023C3648364036503644364436570
:10CF0000836283657047DFED157A80ED010AF4EEE8
:10CF1000E70AF1EE10FAC0ED020A80ED031AC0ED47
:10CF2000051A18DDB4EEE70AF1EE10FA10DD81EE15
:10CF3000007AC0EE207AF0EE006A77EE877A86EE0D
:10CF4000A77A80ED047A80ED0F2AC0ED0E2ACEE795
:10CF500000230361F7E700238360FAE7BD378635D6
:10CF6000FDEEC07A17EE903A2033402B43D8DFED28
:10CF7000237A9FED237AB4EEE70AF1EE10FA28DC6B
:10CF8000DFED207A9FED1E7AB4EEE70AF1EE10FA9B
:10CF900022D4DFED1D7AB4EEE70AF1EE10FA1EDDC1
:10CFA00030EE670A37EEC00A60EE007ADFED176AEE
:10CFB0009FED177AA7EEA67ADFED166AE7EE876A8D
:10CFC0009FED157AA7EEA67A20EE276AA6EE070A4D
:10CFD000704730EE470ACEE730EE070AD4E79FED00
:10CFE0000F7AB4EEC70AF1EE10FA44BF30EE270A0A
:10CFF00037EE400AD8E79FED0A0A7047DB0F494039
:10D00000DB0FC940DB0F49C0DB0FC93F9A7C2E36CE
:10D01000FAAF4FB93587083CA4AA2ABEDB0FC9BFB7
:10D0200000000000DFED027A30EE270A98E700BF2B
:10D03000DB0FC93F38B51D46304BB3FBF2F39942C5
:10D04000B0EE405AF7EE005A4FF000044FD207EE10
:10D05000901A9FED2B7ADFED2B6AF8EE677A67EE78
:10D06000877A07EE102AB8EE477A27EE267AC5EEC1
:10D07000876A87EEA64AB0EE440AFFF771FFF0EE2A
:10D08000404AB0EE440AFFF7CDFF35EE055A012DB8
:10D0900084EE854AF0EE407A1CBF35EEE76AF6EE84
:10D0A000006AB8EE000A34EE257A12BF66EE266AF0
:10D0B00027EE806AF0EE656A86EE875AC6EE076A4A
:10D0C00067EE807A75EEC45AC0ED016AC7EE876AD2
:10D0D000C5EE877A80ED005A80ED025AC0ED036AF2
:10D0E000C0ED047A846144610462C46138BDC0ED5E
:10D0F000005A44608460C4600461F3E720A1070023
:10D10000DB0FC940BD3786359FED010A002391E74B
:10D11000F304353F2DE9F041FCEEC07A13460A4690
:10D1200017EE901AD0F814808769C669056AB0EEC8
:10D13000600A89B2FFF77EFFC0F814808761C6617C
:10D140000562BDE8F081F0EEE06AB0EEC07AF4EE80
:10D15000C76AF1EE10FAD4BFB0EE476AB0EE666A65
:10D16000B5EE406AF1EE10FAF0EE405A46D0F4EE19
:10D17000C76AF1EE10FA54BFB0EE475AB0EE665AE5
:10D18000C5EE067A9FED1F6A9FED1F5ADFED1F4A1D
:10D19000A7EE865A9FED1E6AA5EE276A9FED1D5ADF
:10D1A000A6EE275A9FED1C6AA5EE276A9FED1B5A33
:10D1B000E7EE854AB7EE005AA4EEA75AF1EE467A9A
:10D1C00087EE850AF4EEC76AF1EE10FA48BFDFED8C
:10D1D000147AF5EEC00A48BF37EEC00AF1EE10FA35
:10D1E00048BFDFED107AF5EEC05A48BF37EEC00AEF
:10D1F000F1EE10FA48BFB1EE400A7047DFED0A7A4F
:10D20000C0E700BF39094E3DE3B59EBE69A2163E98
:10D2100088FA16BE45FE7FBFA7DFA8B499FB243F5E
:10D22000DB0FC93FDB0F49400000000044F25063B0
:10D23000984203DDA0F50C40A0387047034B98429C
:10D24000BCBF00F50C40A030704700BFB0B9FFFF75
:10D2500048F69F43984203DDA0F50C40A038704784
:10D260000028BCBF00F50C40A030704791ED005A7B
:10D2700008B5B0EE450AFFF7D5FEF0EE405AB0EE25
:10D28000450AFFF76DFE91ED015AF0EE404AB0EE0F
:10D29000450AFFF7C7FEF0EE403AB0EE450AFFF749
:10D2A0005FFE91ED023AB0EE405AB0EE430AFFF74E
:10D2B000B9FEB0EE404AB0EE430AFFF751FE25EE4C
:10D2C000806A63EEC07A24EE847AC0ED017AF0EED3
:10D2D000467AE5EE077A25EE843A64EE806AC0ED80
:10D2E000037AF0EE437AE5EE667AA5EE067AE5EE8D
:10D2F000436A23EE844A64EEE34A65EEA35A80ED66
:10D30000004A80ED025AC0ED047AC0ED054AC0ED36
:10D31000066A80ED077AC0ED085A08BD034600F1A1
:10D32000400100221A615A619A61DA611033994210
:10D33000F8D11022002153F0E1BB91ED007AD0ED3D
:10D34000047AE7EE077AC0ED047AD1ED006A91ED38
:10D35000017AD0ED057AE6EE877AC0ED057AD1ED57
:10D36000006A91ED027AD0ED067AE6EE877AC0ED9A
:10D37000067A91ED007AD0ED077A77EE877AC0EDE4
:10D38000077AD1ED016A91ED007AD0ED087AE6EEE8
:10D39000877AC0ED087A91ED017AD0ED097AE7EE4F
:10D3A000077AC0ED097AD1ED016A91ED027AD0EDEC
:10D3B0000A7AE6EE877AC0ED0A7A91ED017AD0ED2D
:10D3C0000B7A77EE877AC0ED0B7A91ED007AD1ED8A
:10D3D000026AD0ED0C7AE6EE877AC0ED0C7AD1EDD8
:10D3E000026A91ED017AD0ED0D7AE6EE877AC0ED12
:10D3F0000D7A91ED027AD0ED0E7AE7EE077AC0ED64
:10D400000E7A91ED027AD0ED0F7A77EE877AC0ED41
:10D410000F7A91ED007AD0ED107A77EE877AC0ED31
:10D42000107A91ED017AD0ED117A77EE877AC0ED1E
:10D43000117A91ED027AD0ED127A77EE877AB7EE13
:10D44000007AC0ED127AD0ED137A77EE877AC0EDCC
:10D45000137AD1ED017AD1ED006A91ED027A67EE8F
:10D46000A77AE6EEA67AE7EE077A90ED007AA6EEC6
:10D47000A77A80ED007AD1ED016A90ED017AA6EEEF
:10D48000A77A80ED017AD1ED026A90ED027AA6EEDC
:10D49000A77A80ED027A90ED037A77EE277AC0EDD5
:10D4A000037A70472DE9F043034685B000F1100779
:10D4B000054600261C46AC4612E0F8EC016A1EED5B
:10D4C000047AD4ED007AE6EEC77AC4ED007A984586
:10D4D0000EF1100EF1D10434BC420CF1040C03D057
:10D4E000A7F11008E646F2E701361C46B646BEF143
:10D4F000040F1FD000EB0E1CA84604F1100909E030
:10D50000FCEC016A18ED047AD4ED047AE6EEC77AF1
:10D51000C4ED047ACC4508F11008F1D1D4ED046AC9
:10D5200093ED007AC6EE877A0EF1010EC4ED047A0F
:10D530006446DCE7042E03F1140305F1040507F14A
:10D540001007B7D1002300930193029303936C4615
:10D550000023142752F8045B44F8045B07FB030C18
:10D5600000EB03156E4665451FD10133042BF1D145
:10D5700004AD103100F1400255F8044D0E4600EBA9
:10D58000031741F8044D1446A742D1ED007A17D194
:10D5900052ED016A87EEA67A013BA2F1140281EDF9
:10D5A000007AE9D105B0BDE8F083B6EC017A54ED1C
:10D5B000017AF5EC016AE6EEC77A44ED017AD2E72A
:10D5C000F4EC016AB6EC017AE6EEC77AC1ED007AB6
:10D5D000DAE79FED0C7A00F10C03F0EC017AF4EE3F
:10D5E000677AF1EE10FA06D7F0EEE77AF4EE477AB2
:10D5F000F1EE10FA03DC9842EFD1012070470020D1
:10D60000704700BFFFFF7F7F1FB50C46024669468B
:10D610001030FFF747FFDDED007AB6EE007A67EED7
:10D62000877A2046C4ED007ADDED017A67EE877ACD
:10D63000C4ED017ADDED027A67EE877AC4ED027AF5
:10D64000FFF7C7FF04B010BDB5EEC00AF1EE10FA47
:10D6500008B506DB4EF0B4FBB4EE400AF1EE10FA6A
:10D6600001D79FED010A08BD00000000F8B52DEDBF
:10D67000028B044625461C3004F1640250ED017A09
:10D68000B1EC010A77EE807A40ED017AFBF782F87F
:10D6900018309042F2D123692D4E62680133236124
:10D6A000D6F894319B1AA26893422DD99FED298A0E
:10D6B00004F13007EB6A012BC1BF03F1FF3307EE22
:10D6C000903A95ED0A7AF8EEE77AD4BFB0EE480AC0
:10D6D00087EE270AFFF7B8FFBD42D4ED057A16D0D2
:10D6E000F4EEC07AF1EE10FA05F11805E2D5237BCD
:10D6F00053BBD6F89421626000222361A261E362E9
:10D7000022636364A264E365BDEC028BF8BDF4EEB2
:10D71000C07AF1EE10FAEAD4D4ED047AD4ED066AB8
:10D72000F8EE677A022386EEA77AD4ED0C6A84EDD0
:10D73000067A86EEA77AD4ED126A84ED0C7A86EE2C
:10D74000A77A84ED127A00E003232370DCE700BFA0
:10D75000F02900200000000038B50378012B0446B2
:10D760003CD10369254D23B9426812B9D5F89421FB
:10D770004260D4ED067A77EE807A01332361C4EDFE
:10D78000067A04F11C00FBF705F86268D5F89431BD
:10D790009B1AA268934221D9E36A012BC3BF03F10C
:10D7A000FF3307EE903A94ED0A7A9FED150AC4BF55
:10D7B000F8EEE77A87EE270AFFF746FFD4ED057A01
:10D7C000F4EEC07AF1EE10FA0CD5237B3BB9D5F814
:10D7D0009421626000222361A261E36238BD0323C9
:10D7E0002370FBE7D4ED047AD4ED066AF8EE677A8D
:10D7F000022386EEA77A84ED067AF1E7F02900206D
:10D800000000000008B52DED028BF0EEC08AB0EEEE
:10D81000408AB7EE000A30EE680AFFF715FF9FED69
:10D820000E7ADFED0E7AE8EE877A9FED0D7AA7EE9D
:10D83000A87ADFED0C7AE7EE287AB5EEC08ABDEC67
:10D84000028BF1EE10FA20EE270A44BFDFED067AD4
:10D8500037EEC00A08BD00BF306E99BC2716983D50
:10D86000843459BEA40DC93FDB0F494060EEA00AC5
:10D87000E0EE000AB0EE600AE6E660EEA00AE0EE36
:10D88000000AE1EE010AB0EE600ADDE62DE9F74F8D
:10D8900090469DF83020002A14BF4FF030094FF019
:10D8A00020090D9A1C1E05460F46BABF644201238B
:10D8B000002312F8011B01B12CB9A24663B1002468
:10D8C0000D9EA41B12E0013CF3E7BD4204D2494681
:10D8D00028460193C047019BBAF1010AF5D2EFE750
:10D8E000BD4203D228460193C047019B06EB040BBF
:10D8F00016F8011B0029F3D133B15446002C07DC84
:10D90000BAF1000FA8BFD344584603B0BDE8F08F6A
:10D91000BD4202D249462846C047013CEEE70FB45B
:10D9200037B50C4D06ABD5F8D41853F8042BD5F801
:10D93000D00801934CF01DFB0446D5F8200203F0FB
:10D9400058FD0028F9D0204603B0BDE8304004B0AF
:10D95000704700BFF02900200EB403B503AB08499F
:10D9600053F8042BCDE9003001A84CF002FB019BD9
:10D9700000221A7002B05DF804EB03B0704700BFDC
:10D98000E38700080CB430B52C4CD4F8D838A5B0D7
:10D990001BB9D4F8DC38002B39D094F8E038994220
:10D9A00006D9012303FA00F0D4F8E43818422ED047
:10D9B000D4F894114FF47A7304A8B1FBF3F203FB8B
:10D9C00012131F49FFF7C8FF04AB0344289A1D49EF
:10D9D0000393054629AB03A802934CF0CAFA039BB4
:10D9E000591C03910A211970039B0246591CD4F853
:10D9F000D80803910021197090B103681B6A03B124
:10DA00009847D4F8D85804AC14F8011B21B925B0B4
:10DA1000BDE8304002B07047284603F0C0FCF3E791
:10DA2000D4F8DC38002BF2D002212A4400910A44B9
:10DA3000FD2004A928F0EAF8E9E700BFF02900205A
:10DA4000C3CA06088B87000810B54FF4004086B0A3
:10DA500026F0B6F9044690B34FF4004126F012FBCD
:10DA600002281AD1226848F201039A4227D14FF4C2
:10DA7000004048F0A9F810B31F4BD3F8E8288242C1
:10DA80001FD0D3F8C429904230D0D3F8A02A9042B6
:10DA90002FD00022C3F8DC2811E00023022294F9E1
:10DAA0000400CDE901234FF4612200924FF40041BC
:10DAB0001A4626F037FB104BC3F8D80828B906B031
:10DAC00010BD03F6E802C3F8DC280C4B04930C4BA2
:10DAD00003930C4B02930C4B01930C4B00930C4A99
:10DAE0000C4B02210020FFF74DFFE8E703F6C412BC
:10DAF000E9E703F52A62E6E7F0290020CFCA060825
:10DB0000D8CA0608E1CA0608EDCA06082CCA0608E3
:10DB100031D606083FCA0608174A38B5D2F87C4BFA
:10DB2000033004EB9003B3F5007F19D802F5386594
:10DB3000C2F87C3B114A02EB810120F00300D1F8CE
:10DB40008822C3F500731044C1F888020C4A9B0078
:10DB50000421002005EB8404FFF714FF204638BDA4
:10DB60000021084A0846FFF70DFF074A136843F0F3
:10DB7000007313600024F1E7F0290020E83A002048
:10DB8000F3CA060817CB0608505501202DE9F047C7
:10DB900006460068FBF799FF0D28054608DD1F4A79
:10DBA00000210520FFF7EEFE00242046BDE8F087A7
:10DBB0001B4F07EB80094FEA8008D9F824A2BAF17D
:10DBC000000F1CD107216420FFF7A6FF0446C9F807
:10DBD000240228B90146134A0520FFF7D3FEE4E7E3
:10DBE0006422514652F08AFF0F48D9F824322DB2F0
:10DBF00000EBC505C3E90053DB615B63DB644744AD
:10DC00007179D7F82442182000FB014300221C46FA
:10DC1000C3E903229E601A750434C6E725CB0608C3
:10DC2000F02900204ACB0608AC2B060803685A1CD2
:10DC3000026019700368090A5A1C02601970704763
:10DC400003685A1C0260197003685A1C02600A0AB1
:10DC50001A7003685A1C02600A0C1A700368090ED5
:10DC60005A1C02601970704703685A1C02600A0A45
:10DC70001A7003685A1C02601970704738B5044660
:10DC80000068154652F03AFF23682B44236038BDE4
:10DC900038B504460068154650F092FD23682B44C1
:10DCA000236038BD03685A1C026018787047036807
:10DCB0005A1C02601A4612F8021B0260587841EAA8
:10DCC0000020704710B502681146531C036011F81C
:10DCD000024B0160D31C5178036093781B0443EA24
:10DCE0000123111D0160D078234343EA006010BD79
:10DCF000D1E900329A4206D05A1C0A6008B11B785A
:10DD000003700120704700207047D1E900239B1A5F
:10DD1000012B10B50446084604DDFFF7C8FF20803C
:10DD2000012010BD0020FCE7A0F16103192B98BF72
:10DD30002038704730B50A440446914201D1002092
:10DD400011E014F8013BA3F14100192811F8010B6F
:10DD5000A0F1410598BF2033192D98BF20301B1A20
:10DD600002D10028E9D130BD1846FCE76FF000422F
:10DD7000E0E710B50288C378A2F5FA62910840F294
:10DD8000B554013B04FB013381780C24013902F0C6
:10DD9000030204FB02120D49847901EB42021821AF
:10DDA000B2F8D2201344027901FB0322437900899F
:10DDB0003C2101FB0233064A224401FB03224FF4BB
:10DDC0007A730021C2FB030110BD00BF542B06086B
:10DDD00080436D382DE9F04190461F4605464FF4CB
:10DDE0007A720023404639464DF04CF9284B3C21CD
:10DDF000034493FBF1F201FB1233AB7192FBF1F39D
:10DE000001FB13226A7140F2B551182293FBF2F420
:10DE100002FB143394FBF1F201FB1244B4F5896F59
:10DE20002B714FEA82032EDA40F2DA2294422CDC84
:10DE3000B4F5B77FB4BF00210121164A182000FBBA
:10DE400001220B2632F81600A04201DD013EF9D175
:10DE500003F5FA630B442B80731CAB700C2303FB9C
:10DE600001660D4B03EB46060134B6F8D230E41AD6
:10DE7000EC704FF47A720023404639464DF002F9B7
:10DE80002A81BDE8F0810321D7E70221D5E700BF51
:10DE900080BC92C7262C0608542B0608F0B5274DE7
:10DEA00006460F460FCD8DB06C460FC40FCD0FC484
:10DEB00095E80F0084E80F0016F003033AD16421BF
:10DEC00096FBF1F201FB126242B94FF4C87296FB65
:10DED000F2F302FB1363003B18BF0123721EC3F170
:10DEE0001D03002A019340F26D13104606FB03F355
:10DEF000B8BFB01C03EBA0006FF0630392FBF3F319
:10DF000018444FF4C87392FBF3F21044063069468C
:10DF100000240725013F51F8042BA74202EB000320
:10DF200093FBF5F0C0EBC000A3EB000004D1101A86
:10DF30000DB0F0BD0123D1E70134ECE7882C0608D1
:10DF4000084BD3E9C41251EA020309D0064BD3F8B7
:10DF500094315B1842F10002C0E9003201207047A1
:10DF600000207047E83A0020F029002037B5054628
:10DF70006846FFF7E5FF044638B1DDE9002328468F
:10DF8000FFF728FF204603B030BD40F20113288080
:10DF90006B80A880A8712881F4E71FB50190FFF776
:10DFA000E5FF0199044648B1064B0DF10E02B3F8A6
:10DFB0001833ADF80E30084648F008FA204604B091
:10DFC00010BD00BFE83A00202DE9F043994E87B01C
:10DFD0000446A6F5DC7594F83030042B11D8DFE840
:10DFE00013F0130005005E00DE00250104F11C099A
:10DFF00001AA49463046FEF774FC01280ED00228DB
:10E000002FD007B0BDE8F083304648F069FC4FF6EA
:10E01000FF732384012384F83030DCE7019F0FB1C4
:10E020003B7863B93046FDF7E7FE237EDF061BD55C
:10E0300048F056FC4FF6FF7323840223EBE797F872
:10E040000B8018F0080FD3D10B2204F131013846B0
:10E0500052F0EEFC0028CBD1637E88EA0303D90698
:10E0600004D53046FDF7C8FE0423D4E7BA8A7B8B7B
:10E0700043EA02436362D5F81022FB69A3605202AF
:10E08000B3FBF2F102FB113109B113445B1AE360F7
:10E0900084F819803046FDF7AFFE0323BBE795F8FF
:10E0A000E031002BADD104F11C08092701AA41463B
:10E0B0003046FEF716FC012850D1019888B303784A
:10E0C000E52B01D0002BF1D1FDF75EFF5A4901EBA2
:10E0D0000010FAF71FFA01F5D070FDF78DFE20222F
:10E0E0000021019852F00AFD019BD4F831201A60FA
:10E0F000D4F835205A60B4F839201A8194F83B20BE
:10E100009A72019B627EDA7203A8FFF746FF019BB9
:10E1100038BB6FF07E021A7447225A749873D87312
:10E1200038E095F8B831022B9ED095F8E031002BFD
:10E130009AD1C5E97D33D5F8CC2185F8F03185F841
:10E14000EC31D5F8143285F8E071C5F8E421C5F852
:10E15000E8313046FEF7D4F90128A7D0022883D051
:10E160004FE79DF80E109DF80F2042EA4112BDF8CE
:10E170000C10A1F2BC7142EA41221A829DF81020D3
:10E180009DF81110D20242EA41129DF8121042EAA3
:10E190005102DA811A8A1A83DA89DA827DE7237ECC
:10E1A0009A0608D5E0690023112202A9FDF7FEFEB8
:10E1B00001287FF426AF204648F092FB2269237E97
:10E1C0008AB91B0708D51D4B93F89821002A7FF4C4
:10E1D00018AF072283F89821002384F82830E36AD7
:10E1E000204698470DE703F0F70213F00403227668
:10E1F00008D00023E26AA16884F828302046FDF7A1
:10E200009DFEFEE6122AE7D1E26AA263626A84F802
:10E210003C300421C4E90B22C4E9023384F82810FD
:10E2200063636362204648F05BFBEAE60020E36A32
:10E230002070D6E77C610020DC5F0020C45F0020F6
:10E240002DE9F34103780446002B76D090F828306E
:10E25000013B082B71D8DFE803F00509475B4C61EF
:10E2600070666B0002B0BDE8F041ADE6344B456826
:10E27000D3F81072D3F818327F021D40216B20466C
:10E28000FDF7F4FD05EB01084745064626D880B1A9
:10E29000D4E901329A422CBFA260A360002384F823
:10E2A0002830E36A002B48D0204602B0BDE8F04198
:10E2B00018472169207E01AA4AF0A6FF01283CD117
:10E2C00023696361019B236163683B445B1B63605B
:10E2D000236BDB1B1D4425633546CFE763680028AD
:10E2E000D6D119446160D3E702B0BDE8F041FEF732
:10E2F0008DBA0121FEF7F6F901281ED1216C002309
:10E30000204684F8283002B0BDE8F041FEF7D2BACA
:10E31000002102B0BDE8F041FEF7E4B902B0BDE86B
:10E32000F041FEF77FB902B0BDE8F041FEF783B8D7
:10E3300002B0BDE8F041FEF7E3B802B0BDE8F081FD
:10E34000C45F0020F0B50124B0FBF4F58D4203D288
:10E3500000261CB91C70F0BD4C43F5E7B0FBF4F58A
:10E36000B4FBF1F704FB15002EB9002D03DC8C4241
:10E370000CD33C46EDE7092D08DD002A14BF3724F5
:10E3800057242C4403F8014B0136F2E73024F8E718
:10E39000A0F13003DAB2092A01D818467047A0F17B
:10E3A0006103052B01D857387047A0F14103052BB5
:10E3B00094BF37384FF0FF30704770B50446944231
:10E3C00008461546B4FBF2F602D33046FFF7F5FFD8
:10E3D00005FB1644024B1B5D00F8013B70BD00BFFE
:10E3E0006FCB0608B5EEC00ADFED2D7AF1EE10FA1C
:10E3F000CCBF30EE270A30EE670ADFED2A7A20EE36
:10E40000270A30B5FDEEC07A87B017EE904A054670
:10E4100084EAE470002303A9A0EBE470CDE90033A3
:10E42000029348F04DFA002CACBF20232D2303A803
:10E430008DF800304BF05EFF012822D130238DF89B
:10E4400001308DF802308DF8033003A9684653F08F
:10E45000A5FA68464BF04EFF0338C4B2224669461F
:10E46000284650F0ADF900232B550F49284653F0AC
:10E4700095FA0DEB0401284653F090FA284607B0B0
:10E4800030BD022805D130238DF801308DF80230DF
:10E49000DBE7032804BF30238DF80130D5E700BF48
:10E4A0006F12033A00007A446005070830B502781D
:10E4B000202A034600F10100F9D0092AF7D02D2ABD
:10E4C0004BD10346BFEE000A9FED3C7A1A46F2EEAE
:10E4D000046A134612F8010BA0F13001CCB2092CEA
:10E4E00041D92E280BD1F2EE046A1146B0EE666ACD
:10E4F0000B4611F8012B303AD0B209283CD91A78D2
:10E5000002F0DF02452A53D15A782D2A3FD1023337
:10E510000120013B00220A2513F8011F3039CCB23B
:10E52000092C3AD9B2F59A7F1346DFED256A28BF48
:10E530004FF49A731A46F7EE007A072A30D8DA08B1
:10E540006FF0070101FB0233F2EE046A63BB88B38C
:10E55000C7EE276A20EE260A30BD2B2A08BF0346E5
:10E56000B7EE000AB0E707EE901AF8EEE77AE7EEAA
:10E57000267AB0EE677AACE707EE902AF8EEE77AF3
:10E58000C7EEA65A66EE866A37EE257AB0E72B2AE2
:10E5900014BF013302330020BBE705FB0212BBE7C7
:10E5A00067EEA67A083AC8E767EEA67A013BCDE7A0
:10E5B000F7EE007A67EE276ACCE700BF00000000A4
:10E5C00020BCBE4C70B5034610F8012B202AFAD0AF
:10E5D000092AF8D02D2A0ABF034601254FF0FF353E
:10E5E000591E00240A2611F8010FFFF7D1FE092851
:10E5F00002D905FB04F070BD06FB0404F3E710B577
:10E600000023802804D893420AD2C854581C10BD55
:10E61000934205D060F07F04CC54C0090133F0E789
:10E620004FF0FF30F3E770B51249134C134E01223F
:10E630000020FEF7FEFB228862B1A31DB34217D271
:10E64000A518B54214D2052A12D92146FEF7F1FBCE
:10E650002C46F0E721460222FEF7EBFB63880849CF
:10E66000084AC31A641A5842A2F8B444584170BD0B
:10E670000020FCE70040000801400008008000087E
:10E68000FC3F0008E83A00202DE9F04F794BDFF815
:10E69000F4818FB0A3EB0802CDE901234FF0030909
:10E6A000102200210AA852F029FA019B0993029B2B
:10E6B0000893714BCDF81C801A69002ABFBF6F4ABE
:10E6C0005A6002F188325A600124F322DA604FF076
:10E6D000000A7E23224604A907A88DF83440CDF80D
:10E6E00030A08DF81030FAF72DF9504513DA0023D9
:10E6F000B9F1010900F0B780002BD1D098F80030B3
:10E700007E2B40F0B380FFF78EFF002800F0AE8034
:10E710000FB0BDE8F08F224604A95046FEF789FBF2
:10E72000574CDFF864B1ADF812005C453CD30024CF
:10E73000022205A907A8ADF81440FAF703F9A04290
:10E74000D5DBBDF81200022205A9FEF772FB0222FA
:10E75000ADF812000DF1120107A8FAF7F3F8A04284
:10E76000C5DB0B9888B1079B089A03449342BED837
:10E770000AABC0F104022146184452F0BFF90AA9BD
:10E7800007A8FAF73CF8CDE90B400C9B002BAEDB59
:10E790009DF8342022B138490A6942F000420A61EA
:10E7A000B3FA83F35B09A3E762888DF819A0C2F37B
:10E7B0000B06B31DADF814302388C3F30B011B0BFC
:10E7C0008DF818301304ADF8161020D4062205A9D0
:10E7D00007A8FAF7B7F8002889DBBDF8120006226F
:10E7E00005A9FEF726FB6168ADF81200324607A8BE
:10E7F000FAF7A8F80028FFF67AAFBDF812006168B2
:10E800003246FEF716FBADF8120014348DE70027F0
:10E810003D460135EDB2062205A907A88DF819502D
:10E82000FAF790F80028FFF662AFBDF81200062252
:10E8300005A9FEF7FEFA6168ADF8120039443246C8
:10E8400007A80391FAF77EF80028FFF650AFBDF84D
:10E85000120003993246FEF7ECFA032DADF81200D0
:10E860003744D6D1D1E7002B7FF448AF052005F01F
:10E87000C7F800BF00800008003C02402301674544
:10E880009835070800400008C03A0708034AD2F844
:10E89000B83423EA0000C2F8B8047047E83A002010
:10E8A000034606490648884201D300207047028883
:10E8B000C2F30B029342F9D01430F4E7C03A0708D0
:10E8C0009835070813B542880B460446C2F30B027D
:10E8D00000211846019252F011F9216903460A48B5
:10E8E000814209D30948019A814205D2184602B0F3
:10E8F000BDE810404FF064BF21B1184602B0BDE83A
:10E900001040084702B010BDC03A07087B3F070817
:10E9100010B4B0F902404288002C0B4641685DF803
:10E92000044BBEBFC2F30B02DBB203FB0211C9E70B
:10E9300030B5094B094CA34200D330BDB3F90220D6
:10E940005988002A06DA5A68DD68C1F30B0100FB1A
:10E9500001222A601433EEE798350708C03A070809
:10E9600030B502460144002012F8015B082480EA19
:10E97000050313F0010F4FEA50001CBF80F08C0319
:10E98000D8B2631E13F0FF044FEA5505EFD18A4257
:10E99000EAD130BD2DE9F04F87B0CDE90212002554
:10E9A000804604930195039B404603EBC50AFAF7A2
:10E9B00007FFEC00024600286DD0002201214046EE
:10E9C000FAF7E8FE0246002865D098F80430990767
:10E9D00061D5F0214046FAF7FDFE024600285AD0E4
:10E9E000039BA4F108024FF0000B012713443C469F
:10E9F0005E460593029B002B55D0082C53D804F19A
:10EA0000FF3943FA09F909F0010949464046FAF786
:10EA100098FE024600283ED0002201214046FAF727
:10EA2000B9FE0246002836D098F8041001F0600CB8
:10EA3000BCF1600F4FEAD11016D0029B1BB1082C1D
:10EA400001D8814527D1002841D01AF80610394352
:10EA50007F00013417F0FF070AF80610E4B2C9D1AD
:10EA60000136F6B2082E1CD1402C10D90721504691
:10EA70000592FFF775FF9AF80710059A814206D1B3
:10EA80000135EDB2BBF1000F05D0CDF804B0049B09
:10EA90001B78AB4287D8049B10461D7007B0BDE8B9
:10EAA000F08F0127A6E75DB1019BA34208D9059B22
:10EAB0009A5D174214BF4FF001094FF00009A4E717
:10EAC000019B1B1BD3F1000949EB03099DE7880952
:10EAD00040EA511111F0010F1AF8061008BFA346C1
:10EAE00021EA0701B4E700BF90F83C20034602F09A
:10EAF000FF0012B1002283F83C2070474FF480538E
:10EB0000838170474FF40063838170474FF4006343
:10EB1000838170474FF40063838170474FF4006333
:10EB2000838170474FF40063838170474FF4006323
:10EB30008381704710B5064A0423002152F8044B24
:10EB4000844208BF42F8041C013BF7D110BD00BF4E
:10EB5000E86100203248F0B5C38B058AB0F928403F
:10EB6000B0F91660B0F922C0B0F93070ED1A838B9D
:10EB70006B43B0F9265004EBE334ED0295FBF4F55A
:10EB800005EBE335A5F57A6E0EFB0EF42313B0F911
:10EB90001840C5620EFB06F60EFB04FEB0F92040DD
:10EBA0005C4303FB0CFCF612241406EBEC2C04EB88
:10EBB0006E34B0F91460438B02340CEB860CA41055
:10EBC000466B04F500440CFA07FC63430CF1020C9D
:10EBD0004CF25030DC0BA6EBAC0640FA07F3734363
:10EBE00055BF5B00B3FBF4F3B3FBF4F35B0071B10F
:10EBF000181240F6DE34404360430A4C00145C4374
:10EC000000EB244000F6CF6003EB20130B6022B131
:10EC10000A235D4308352D1115600120F0BD00BFAA
:10EC2000E861002043E3FFFF0120704701207047A7
:10EC30002DE9F8435E4F1546BC6BBA8FB7F842908A
:10EC4000C2EB24135200C2EBE402B7F93E40624328
:10EC500003FB03F4B7F9403024135C43A41304EB23
:10EC6000E224B7F946307C650E46A4F5FA3181FB03
:10EC700001CE4FEAE37803FB0EF20CFB0822A3FB64
:10EC80000C389044B7F9442082FB01021B0A12039E
:10EC900043EA086342EA105200031B1842EB2822A1
:10ECA00002F50042A3FB093809FB02884FEAE8732A
:10ECB0004FEA680253EA68084FF000006CD0B7F9D9
:10ECC0004C904FEAE97809FB0EFE0CFB08EEA9FB1D
:10ECD0000C9CE644B7F94AC08CFB01814FEA414CD9
:10ECE0004FEA484111EB0909B96D4CEAD83C4EEBAB
:10ECF0000C0CC1F5801E0EF00048B7F9481048EA28
:10ED00005E0810EB09004FEACE7EBEEB00000CEB74
:10ED1000C10168EB010C40F63548A0FB080108FB77
:10ED20000C114CF0AFF9B7F952304FEA613E4FEA9F
:10ED3000503C4CEAC14C03FB0EF24FEAE3790CFB6A
:10ED40000929A3FB0C324A4403FB0EFE0CFB02EE26
:10ED5000A3FB0C3CB7F95020E6445B0E43EACE130C
:10ED600013EB000C804602FB01F34FEAE27941EB22
:10ED70006E6EA2FB082809FB00314144D00C40EA2A
:10ED800041301CEB0000B7F94E304EEBE141000A78
:10ED900040EA016000EB03100EB1000A306025B1BB
:10EDA00004EB8404803424122C600120BDE8F88335
:10EDB000E861002031B10A4BD3ED1D7AFDEEE77A10
:10EDC000C1ED007A52B1064B9FED067AD3ED1E7A63
:10EDD00067EE877AFDEEE77AC2ED007A0120704790
:10EDE000E86100200000C8422DE9F74FCDE900128C
:10EDF000554AB2F88A30D16FB2F88660B2F88C709A
:10EE00001B02C91AB2F888306EEB0E0EA3FB010488
:10EE100003FB0E44B2F88430C00940EA44601B048E
:10EE2000C018A6FB013506FB0E55B2F882604FEA0A
:10EE3000132343EA05634FEAC6364FEAE41444F16C
:10EE400000049B19A7FB012607FB0E664FEAD2526E
:10EE500042EA46224FEA252545F10005F61512F54E
:10EE6000FA6C46F1000BBCF5FA6F7BF100074CDA47
:10EE7000A2FB02784FF0050A02FB06F908EB4909EC
:10EE8000A7FB0A780AFB09884FEA570949EAC879BB
:10EE9000BF08B0EB090047EA887764EB6804DB1B26
:10EEA0002A4F65EBA805BC454FF0FF377BEB070702
:10EEB00020DA40F6AC57D21946F100065643A2FBC1
:10EEC000027202EB46064FEAC608FA00BA1A48EA8E
:10EED000577866EB0808101844EB08044FF00B084D
:10EEE000A7FB087208FB06267F0847EAC677DB1BEC
:10EEF00065EB660501FB0EFEA1FB011202EB4E0E57
:10EF0000C90F41EA4E01BCEB010C009A9AB10E4ABE
:10EF1000D2F89010A1FB032301FB0535520D42EA04
:10EF2000C522121A4FEA6555009B65EB0404D20B0B
:10EF300042EA44421A60019B0BB1C3F800C00120B1
:10EF400003B0BDE8F08F00BFE861002024FAFFFFA6
:10EF500001207047B0F90000084B4143994208DB9B
:10EF6000B1F5000F07DA0029B8BFFF31081200B26F
:10EF700070470348FBE747F6FF70F8E701FF7FFFA4
:10EF80000080FFFF064B0022C3F89420C3F89820AE
:10EF9000C3F89C200022C3F8A0200120704700BFC6
:10EFA000E8610020104B1A68104BD3F8A010521AD9
:10EFB000FA2A16D8D3ED257AFDEEE77A17EE902AD5
:10EFC000D3ED267AC286FDEEE77A17EE902AD3EDCE
:10EFD000277A0287FDEEE77A17EE903A4387012001
:10EFE00070470020704700BF842B0020E86100209C
:10EFF00090F85F3230B53BB990F85D1290F85E3210
:10F000000124DAB2914200D830BDB0F8665204FA59
:10F0100003F22A43A0F866220133F2E7437913F0A2
:10F0200001031FBFD0E90732C0689B1A00F1FF300F
:10F0300014BF184018467047437913F002031FBFEE
:10F04000D0E9093200699B1A00F1FF3014BF9843E0
:10F050001846704710B5437913F0010301460DD0EF
:10F06000FFF7DCFF60B10A6A4B69C8689B5C01323C
:10F07000B2FBF0F400FB1422DBB20A62184610BDAA
:10F080000346FBE743799B070AD5436A8269D1545B
:10F09000436A02690133B3FBF2F102FB11334362AD
:10F0A000704741717047D0E90920131A58425841FE
:10F0B0007047024BD3F8A4305B681847E861002022
:10F0C000024BD3F8A43008309B681847E861002051
:10F0D00001207047012070470120704701207047D0
:10F0E0000120704731B10C4BD3ED2A7AF8EEE77A64
:10F0F000C1ED007A7AB1084BDFED086AD3F8AC3085
:10F10000A3F5D543333B07EE903AF8EEE77A87EE66
:10F11000A67A82ED007A7047E86100200000C842BC
:10F1200001207047012070477047044B03EB8000BB
:10F13000D0F8B0300BB19B6819607047E8610020CF
:10F1400008B50246FFF7F1FFBDE80840104620F081
:10F1500037BB054B03EBC00040F2FF739942A8BFD9
:10F1600019468180704700BF503E00200C4A13783A
:10F170007BB10C4B93F8F01059B193F8F11059B1E1
:10F1800050680021FA2883F8F110A8BF4FF0FF3033
:10F1900070476FF0010070476FF00200704700BFCA
:10F1A00038100020E86100200B4B93F8F2206AB180
:10F1B00093F8F3206AB1002283F8F320074B986894
:10F1C000B0F5967FA8BF4FF0FF3070476FF0010099
:10F1D00070476FF002007047E8610020381000208F
:10F1E000024BD3F8F4305B68184700BFE861002099
:10F1F000024BD3F8F4309B68184700BFE861002049
:10F20000024BD3F8F430DB68184700BFE8610020F8
:10F21000014BD868704700BF38100020044B93F8AA
:10F22000F83013B1034B186970476FF00100704755
:10F23000E8610020381000202DE9F043062592F9FE
:10F24000007087B06B43144612F80580A0EB080EDF
:10F25000A0EB070CBEF1000FB8BFCEF1000EBCF161
:10F26000000FB8BFCCF1000CE64502EB050905F133
:10F270000605BCBF4FFA88F74C46AB421646E3D1B1
:10F280001A443378BB420CD1658873884D1BCB1A66
:10F29000002DB8BF6D42002BB8BF5B429D42C8BF76
:10F2A00034460636B242ECD1637904932379039352
:10F2B000638802932378064ACDE9001303460321AD
:10F2C0000120FEF75FFB204607B0BDE8F08300BFDA
:10F2D00019CC06084B1EDBB2062BF0B598BF1D4AB1
:10F2E0001D4C98BFD25C04F1580388BF4FF4807264
:10F2F000002808BF1C46234687B013F9087B1888EE
:10F30000C8B9164B93F8F900A3790593A388049321
:10F31000A378039323880091CDE90123104A114B70
:10F320000321002808BF13460F4A0120FEF72AFBDD
:10F33000204607B0F0BD161AD51B002EB8BF764286
:10F34000002DB8BF6D42AE42BCBF1C4647B2083369
:10F35000D5E700BF482D06084C100020E8610020CA
:10F360000F06070888E1060852CC060808B50068B1
:10F3700049F0DBFC014BD867012008BDE8610020A3
:10F3800008B5006849F0D1FC024BC3F89000012099
:10F3900008BD00BFE861002038B514460D460029BD
:10F3A00043D0344B9FED346AD3ED3F7AB3F9142147
:10F3B000F8EEE77AC7EE866A07EE902AB3F91021D5
:10F3C00007EE102AF8EEE77AB8EEC77AB3F9122101
:10F3D000A6EEA77AD3ED427AF8EEE77AE6EE877AE0
:10F3E00093ED417AB8EEC70AA6EEA70A07EE902A77
:10F3F000B3F90E2107EE102AF8EEE77AB3F90C21E3
:10F40000B8EEC77AA6EEA77A07EE902AF8EEE77A6A
:10F41000E6EE877A93ED467AB8EEC77AC7EE066ACB
:10F42000A6EEA70A4CF0BEFB28600CB3114BDFED33
:10F43000126AD3ED467AB3F90021B3F90231F8EE3E
:10F44000E77A07EE102A87EEA60A07EE903AF8EE62
:10F45000E77AB8EEC77A60EE277AF6EE006AE7EE52
:10F46000267A9FED060A27EE800A4CF09BFB20606F
:10F47000012038BDE86100200000F04A0000C842C9
:10F4800038B50B4D55F8303007EE901A04466BB185
:10F4900093ED047A93ED030AF8EEE77AA7EE870A74
:10F4A0004CF080FB55F834309B68186038BD00BFC5
:10F4B000503E002010B50C4B0C4C1B68D4F81C01BE
:10F4C0001B1AFA2B06D904201AF0BAF9002084F886
:10F4D000200110BD11B1D4F824310B6012B1D4F861
:10F4E000283113600120F4E7842B0020E86100201C
:10F4F0002DE9F0410C4DDFF834802C686B69012751
:10F500001C400CB9BDE8F081B4FA84F3C3F11F03C9
:10F5100007FA03F608EB830324EA0604D3F82C0168
:10F52000036898476E61ECE7003C0140E861002009
:10F5300010B5114CD4F86C0118B1104A6421FAF7D7
:10F540001BFBD4F86C010021FAF76EFBD4F86C3188
:10F550005B681A68B2F844306FEA43436FEA53437A
:10F560009BB2A2F8443013889BB243F0010313808E
:10F57000012384F8703110BDE8610020009F240051
:10F5800010B50B4CD4F86C0118B10A4A0321FAF7F4
:10F59000F3FAD4F86C010021FAF746FBD4F86C01B9
:10F5A0000549BDE8104040F62B4247F0A1B800BF26
:10F5B000E8610020009F2400589E002037B5836832
:10F5C0001C686379DB0724D5A57994F85C3205F0D3
:10F5D00001010D46FBB1E06B43681A68D36AC3F3BF
:10F5E0004E03536294F86D32012B07D094F86132C8
:10F5F00023B1B4F868320133A4F8683285F0010110
:10F6000046F0C4FF0023A4F866324FF08073C4F8BC
:10F610005C3203B030BD94F85F320191012B04BF1E
:10F6200094F85D3284F85E322046FFF7E1FC94F8EE
:10F630005F32019953B9012384F85F3285EA0301EF
:10F64000E06B03B0BDE8304046F0A0BF002384F873
:10F650005F32F5E7F0B52DED028B83B00E4615460F
:10F6600043F03AFC002869D0364B374C1B6894F8BD
:10F67000712103F00203002A45D0002B59D0334FEB
:10F680000DF1060023F05CFED7F8EC23BDF8063040
:10F690009FED2F7A9B1A07EE903AF8EEE77AF0EE9C
:10F6A000408A87EE870A07F58067DFED2A7A20EE29
:10F6B000270AFDF7B7FC97ED008AA0EE688A3DF0B7
:10F6C0004DFED4ED5F0AD0ED057AB0EE480A70EE3B
:10F6D000A70AFEF7CBF87EB1DFED1F7A9FED1F7A08
:10F6E00020EE000A20EE270AC0EE077A9FED1C7A72
:10F6F00077EE877AC6ED007A0DB11A4B2B6003B016
:10F70000BDEC028BF0BDA3B1B4F9A23101EE103A09
:10F71000B4F9A03100EE903AB4F99E3100EE103AFF
:10F72000B8EEC11AF8EEE00AB8EEC00AFEF7A5F886
:10F73000D1E7D4F8B83193ED340ACCE79FED0A0A4B
:10F74000C9E700BFEC550120E8610020408D002092
:10F750000000C84235FA8E3CCDCC9C3F00409C4610
:10F7600082E6C547331390430000000008B520210E
:10F7700052F023F9034620B11A78202A00F1010043
:10F78000F8D0184608BD70B50D461446FFF7EEFFD9
:10F790000646A0B1FEF716FF40F634039842A8BF14
:10F7A0001846B0F5617FB8BF4FF46170A0F5617382
:10F7B0001920B3FBF0F32B7023780133237030460C
:10F7C000FFF7D4FF0646A0B1FEF7FCFE40F6340377
:10F7D0009842A8BF1846B0F5617FB8BF4FF461707A
:10F7E000A0F561731920B3FBF0F36B70237801333C
:10F7F0002370304670BD144951F8200070B500B335
:10F800000C2202FB001292F9BD31581C1AD092F85A
:10F81000C501B0B1C8188C2590F8106292F8C441A7
:10F82000002014226B431D1901EB4505013AB5F880
:10F830001452344410FA85F0F5D11423B0FBF3F0E0
:10F8400080B270BD0020FCE7E861002038B50320DD
:10F850000D461446FFF7CFFF07EE900A8DB19FEDDE
:10F860000B7AF8EE677AF0EE006A67EE877AB8EE08
:10F87000047AA7EEA67ADFED067A67EE277AC5ED61
:10F88000007A0CB1034B236038BD00BF6740533A88
:10F8900000007A443313904310B5427A044632B1E3
:10F8A0000146406851F80A3B98470023637210BD37
:10F8B00010B4447A621C0444D2B24272A172037A38
:10F8C000934202D85DF8044BE6E75DF8044B7047BD
:10F8D000EEE710B503681A79022A044602D1987A35
:10F8E00049F014FA00232360237110BDF0B50D4BCD
:10F8F0000D4E0446B34201D30020F0BD5879884232
:10F900000DD11D79A54200D04CB9D879904206D1CD
:10F9100018680779AF4202D105689D42EDD00C33DB
:10F92000E8E700BF580300080805000873B502792E
:10F93000022A38D190F910308DF8022003241426C1
:10F9400073438DF803401A4C1A4EE35800250120EA
:10F95000B3428DF800508DF8010026D0164DAB4211
:10F9600003D0164883421ED1104601F108020DEB68
:10F9700002011A8811F8085C22F040021204120CED
:10F9800014211A8001FB00401A88C16822F0380255
:10F9900031F825101204120C0A431A801A8892B208
:10F9A00042F040021A8002B070BD2846DDE700BF79
:10F9B000B00000200030014000380040003C004012
:10F9C000C36910B5044623B909211420FEF7A4F831
:10F9D000E061E06910BD10B504460068FFF7F0FF74
:10F9E0008378DBB1B0F90A3007EE903AF8EEE77AA7
:10F9F000C4ED057AB0F90C3007EE903AF8EEE77AEC
:10FA0000F1EE677AC4ED047AB0F90E3007EE903A61
:10FA1000F8EEE77A0120C4ED067A10BD1846FCE73F
:10FA200010B504460068FFF7CBFF8378CBB1B0F97F
:10FA3000043007EE903AF8EEE77AC4ED047AB0F9B4
:10FA4000063007EE903AF8EEE77AC4ED057AB0F9A1
:10FA5000083007EE903AF8EEE77A0120C4ED067A16
:10FA600010BD1846FCE710B504460068FFF7A8FF74
:10FA70008378CBB18388DBBA07EE903AF8EEE77A69
:10FA8000C4ED047AC388DBBA07EE903AF8EEE77A61
:10FA9000C4ED057A0389DBBA07EE903AF8EEE77A0F
:10FAA0000120C4ED067A10BD1846FCE710B50068C9
:10FAB0000C46FFF785FF83784BB143892222DBBADE
:10FAC00093FBF2F303F26D132380012010BD18465F
:10FAD000FCE738B500680D461446FFF771FFD0F813
:10FAE000013007EE103ACDB1D0F80530DFED166ADF
:10FAF0009FED166A07EE903AF8EE677A77EEE67AAF
:10FB000077EEA77AC7EE866AF7EE007A76EEE77AA6
:10FB1000DFED0F6A67EEE67AC5ED007A9CB1DFEDA6
:10FB20000D7ADFED0D6AB8EEC77A27EE277AC7EEB9
:10FB3000267A9FED0A7A77EEC77A9FED097A77EEFB
:10FB4000877AC4ED007A38BD9AC9CC449AC94C462C
:10FB50000E76D7450000484300E0FF4400004842CD
:10FB60003393884337B500680D461446FFF728FFE6
:10FB7000D0F805309FED237A07EE903AF8EE677AD9
:10FB800077EEC77A9FED207A67EE877AB3EE097A2F
:10FB900067EE877AB2EE047AF4EEC77AF1EE10FAE5
:10FBA00006DCBAEE047AF4EEC77AF1EE10FA0CD560
:10FBB00017EE900A4AF00AFD144ACDE9000104212B
:10FBC0000320FDF7DFFE03B030BDD0F8013007EEB3
:10FBD000103A2DB1DFED0E6A67EEA67AC5ED007A18
:10FBE000002CF0D0B8EE477ADFED0A6ADFED0A7A32
:10FBF000E7EE267A9FED097A77EE877AC4ED007AF0
:10FC0000E1E700BF00000046000080389CCC0608F9
:10FC10000AD778430319C83D000048C2339388438C
:10FC20000379022B0DD190F9103014225343064A68
:10FC3000D3581A89920746BF1889C0F3C010012013
:10FC400070470020704700BFB00000200368DB6BE6
:10FC500013B504462BB923685B6B3BB9FF23E382E2
:10FC600002E098470028F6D102B010BD214601A855
:10FC700098470028F2D0BDF80630013B9BB2EEE772
:10FC800010B5036804469B68984701236374FF23FB
:10FC9000A37410BD036810B504461B689847236819
:10FCA00020469B689847E37C0133E37410BD0368EA
:10FCB00010B504465B689847236820469B689847C0
:10FCC000E37C013BE37410BDF0B585B004461846F3
:10FCD0000D46164603934AF00DFB2268E67328444E
:10FCE0000021A07300915769039B324629462046A4
:10FCF000B84705B0F0BD30B5046885B0E469089D2B
:10FD000034B10DB90DF10F050095A04705B030BD18
:10FD10002046FBE703685B6A184703689B6A18473D
:10FD200010B5037B04460BB1437B13B92046FFF7A4
:10FD3000F4FF23682046DB68BDE8104018470368DD
:10FD40005B6C03B11847704738B504468B68016097
:10FD50000D4698470B4B2361002323752B6B13B182
:10FD6000204698472075084B93F85C351BB1237DDE
:10FD700023F0010323750023E3822046BDE83840C9
:10FD800064E700BF0001FF00E861002003681B6812
:10FD900003B11847704703685B6803B118477047A1
:10FDA00003681B6A03B11847704703685B6A03B1B5
:10FDB0001847704730B40468A46A14B1A44630BC34
:10FDC000604730BC704730B40468E46A14B1A4469C
:10FDD00030BC604730BC704703685B6C03B11847A8
:10FDE000704703689B6C03B11847704703689B6FAB
:10FDF00003B1184770470368D3F8803003B1184740
:10FE000070470368D3F8843003B11847704703681C
:10FE1000D3F8883003B11847704721B10B68D3F885
:10FE20008C3003B118470020704738B5094B0524C2
:10FE300004FB0030A0F1A00515F8010B013C48F0CF
:10FE4000B0FC14F0FF04F7D12046BDE8384048F07C
:10FE5000A8BC00BF4F2D060810B5441E14F8010FB2
:10FE600000B910BDFFF7E1FFF8E7FFF741BBFFF76F
:10FE70003FBBFFF73DBBFFF73BBBFFF739BBFFF7CE
:10FE800037BB30B1036882881B691A4214BF012056
:10FE90000020704710B1036882881A83704710B140
:10FEA000036882885A83704737B50C46054600B30D
:10FEB0000368114A03F13F4303F57E0302EB9323EA
:10FEC00093F8AA0246F0DAFCAB88009304F003032F
:10FED0008DF80430C4F381038DF805302868C4F32D
:10FEE0000013694664098DF806308DF80740FAF76B
:10FEF000D5F903B030BD00BF482D0608F7B50C4654
:10FF000015460646A8B303681B4A03F13F4303F5B1
:10FF10007E0302EB93230F2793F8AA0246F0AEFC70
:10FF20003068B6880096B6FA86F3C3F11F0303F073
:10FF30000702C3F3CC0300EB83039200196A9740D6
:10FF400021EA07011962196A95400D431D6204F008
:10FF500003038DF80430C4F381038DF8053069463E
:10FF6000C4F3001364098DF806308DF80740FAF7E2
:10FF700095F903B0F0BD00BF482D060838B5040957
:10FF8000013C032C00F00F021AD80E4D05EB440380
:10FF9000B3F8B01241FA02F313F001000FD00123BD
:10FFA00003FA02F2013A02EA01002C4452F056FC34
:10FFB00094F8B8321844044B0C2202FB003038BDD0
:10FFC0000020FCE7482D0608486700202DE9F04F87
:10FFD0005422044693B0B948002150F08FFDB84A2E
:10FFE000601E15460334134610F8011F4E1E052EE1
:10FFF00088BF0021844245F8041BF5D1B048002198
:020000040801F1
:1000000050F8044B012C00F0508101310429F7D144
:10001000002152F8040B022800F03E81013104292E
:10002000F7D10320FEF786FD0420FEF783FD0520AF
:10003000FEF780FD0620A34EA04CDFF89882FEF765
:1000400079FD4FF01A094FF0000A06F52F77207B53
:1000500048B394F90D50FFF791FF28B10523837140
:10006000002380F8079003721321FFF71DFF227B06
:10007000002317F83310914240F0DE8006EBC303F3
:10008000D3F8C0322361182303FB0585D5F8E0308F
:1000900023755A1C0723A3750123C5F8E020637557
:1000A00085F8DC309A4409F101095FFA89F9B9F160
:1000B000200F04F10C04CAD1BAF1000F00F0B9808E
:1000C000814CDFF814924FF00008237C002B00F0E5
:1000D000A6806079794D46F0D1FB207946F0CEFBC1
:1000E000A068FAF753F80023CDE90E33CDE91033B9
:1000F000069308932368A068CDF814904C330493BA
:10010000E368039363691422534307934FF48062B7
:100110004FF40063CDE909234FF400514FF480738D
:10012000CDE90B134FF4003303A90D9346F0B6FA53
:10013000A268136843F001031360644A536823F410
:10014000733323F4477323F0030343F440335360C2
:10015000226863695168012B21F04071D4BF0020EF
:10016000012021F4807141EA0021516090685849D2
:10017000014041F002019160D16A013B21F470011C
:10018000DBB241EA0353D3624FFA88F101239C4664
:1001900001914FF01F0E697D51B395F90D10019833
:1001A000814225D1297CAE7D5F1C0929FFB249D946
:1001B000A1F10A00D2F80CA000EB40004FF0070BB1
:1001C0000BFA00FB2AEA0B0A06FA00F040EA0A00E2
:1001D000D060062B44D8013B506B03EB83030EFA2F
:1001E00003F620EA060001FA03F3034353633B4698
:1001F0000CF1010CBCF1070F05F10C05CBD1936894
:1002000043F400739360936843F48073936093683E
:1002100043F001039360936843F08043936008F1D7
:100220000108B8F1030F04F1180409F58C797FF483
:100230004CAF13B0BDE8F08F0133102B7FF419AF32
:1002400000231FE7106901EB410A4FF0070B0BFA7F
:100250000AFB20EA0B0006FA0AF630431061B8E701
:100260000C2B0CD8073B106B03EB83030EFA03F641
:1002700020EA060001FA03F303431363B7E70D3BDB
:10028000D06A03EB83030EFA03F620EA060001FAB4
:1002900003F30343D362AAE7212283F8D42193F81E
:1002A0001022013283F81022BBE6112183F8C81115
:1002B00093F81012013183F81012A9E6A46300200C
:1002C000E8610020482D06080411002000230140A9
:1002D000FDF7FFC038100020FC6300202DE9F04737
:1002E0009846AB4DAB4B9D4221D26C798C4240F08D
:1002F00063812C79844202D0002840F05D81EC7942
:10030000944240F059812C68DCB11C220021201D50
:1003100050F0F4FB25602B79237195F806A0C4F802
:1003200008A02A7AE260012B03D0022B0CD0002413
:1003300007E0E87AFFF722FE6B7A2374AB7AA061BC
:1003400063742046BDE8F087E87AFFF717FE95F959
:100350000960A0612674A87AFFF710FE606100288A
:1003600000F0128114238C4D7343EF18EB58002BCF
:1003700000F00A81BB7C002B40F0C080387A46F048
:100380007DFA3B7A03F01F025B090121023B01FA6F
:1003900002F2032B08D8DFE803F06C6602607F49A5
:1003A0000B6923EA02020A61142303FB0653771C3C
:1003B0005879FFF7E3FDFFB2814618B140F60A33E2
:1003C000C3800772142303FB0653D879FFF7D6FDC9
:1003D00018B140F60A53C3800772142303FB065377
:1003E0009879FFF7CBFD18B140F60A43C380077236
:1003F000142707FB06571AF0040A7A7A3FD04A21DD
:100400004846FFF77BFDF879FFF7B8FD7A7A2A2195
:10041000FFF774FDB879FFF7B1FD7A7A142707FB6F
:1004200006570A21FFF76AFD387928B1FFF7A6FDC4
:100430007A7A0921FFF762FD14237343EA58584B77
:100440009A4226D103F58433596A41F480515962A6
:10045000596A21F48051596228E050494B6923EAD6
:1004600002024A61A0E74D490B6A23EA02020A62CE
:100470009AE74A494B6A23EA02024A6294E70A2150
:100480004846FFF73BFDF879FFF778FD7A7A0A21B5
:10049000BEE7444B9A4240D103F50033196A41F458
:1004A00080411962196A21F480411962BAF1000F82
:1004B00067D0002318461188034301F441510B43D0
:1004C00043F445731380938B23F400631B041B0CCC
:1004D00093830723138213889BB243F04003138056
:1004E000142303FB0653187918B1FFF747FDFFF7F4
:1004F000D1FC142303FB06550123AB74606928B1BA
:100500000E23C371002380F8068003720921FFF7D0
:10051000CBFC6069FFF7BEFC13E7234B9A4209D17D
:1005200003F5FE33196A41F400411962196A21F496
:100530000041BAE71D4B9A4209D103F58233596A4B
:1005400041F400515962596A21F4005183E7184B74
:100550009A4209D103F56843596A41F480115962FE
:10056000596A21F4801176E7124B9A429ED103F525
:100570006443596A41F400115962596A21F4001127
:1005800069E70123022096E72046FFF7A2F9CEE6AD
:100590005803000808050008B00000200038024099
:1005A0000030014000380040003C00400034014071
:1005B00000500140005401400C3594E6074B03EB1A
:1005C0008000D0F83C333BB19A881B6859690A42D5
:1005D00001D05A8370471A83704700BF482D060820
:1005E000094B03EB8000D0F83C3349B903B970479D
:1005F0001A689B88138370471A689B8853837047D7
:10060000002BF9D1704700BF482D06082DE9F84F9F
:100610006E4F97F87001002840F0D580D7F86C91A4
:1006200099F81030002B40F0CE8097F8AE2797F85D
:10063000AF3797F8B057A7F8AC0707F2B2788646FD
:100640003C2698F8021098F803C0C1F1FF0189B266
:10065000002900F0B480C1F1FF010CFB01F1B8F8F2
:100660000040B4FBF6FB0912BBF1050F21D8DFE80F
:100670000BF0030E65748695ACEB01036343B3FB8B
:10068000F6F353FA81F3CDB2DBB2624610E0B4FB6D
:10069000F6F206FB124292B2C2F13C02ACEB01044C
:1006A0006243B2FBF6F252FA81F2CDB2D2B26346A5
:1006B00001204FEA022C4CEA034C4CEA050C4FF0A7
:1006C000000A0121CAF1170B01FA0BFB0EEB0A0419
:1006D0001BEA0C0F04F12A0408BF8B46A4B23C4964
:1006E0000AF1010A18BF4FF0020BBAF1180F41F8D6
:1006F00024B0E6D10EF1180E1FFA8EFEBEF5406F43
:1007000008F104089DD1A7F8B2E928B187F8AE270F
:1007100087F8AF3787F8B0578023A7F8AC3797F83A
:10072000B439002B4FD0484640F62B41F9F7BAFBBD
:10073000D7F86C01BDE8F84FF9F7E6BBB4FBF6F368
:1007400006FB1344ACEB0105A4B2CAB26543B5FB8A
:10075000F6F555FA81F1CDB2A9E7B4FBF6F306FB45
:1007600013439BB2C3F13C03ACEB01046343B3FB03
:10077000F6F353FA81F3CAB2DBB2654698E7B4FBED
:10078000F6F006FB1044ACEB0102A4B26243B2FBEC
:10079000F6F252FA81F2CBB2D2B2EEE7B4FBF6F542
:1007A00006FB1545ADB2C5F13C05ACEB0104654354
:1007B000B5FBF6F555FA81F5CBB2EDB265E76546C6
:1007C0006346624674E7BDE8F88F00BFE861002029
:1007D000589E002070B500212520F9F7B3F9064690
:1007E00000B3FDF7D3F9214C0546C4F86C01C8B13C
:1007F0002520FFF7C3FBC4F8B80920B140F2152348
:10080000C38000230372327A4A21FFF777FB94F802
:10081000BC39022B07D1FEF78BFE2846F9F714FBF3
:100820000023036070BD032B06D1FEF781FE28462E
:10083000F9F70AFB6423F4E7FEF7A2FE10B984F887
:10084000B409EFE743F2AC020948002150F056F931
:1008500094F8BC39012B02BF064BFF22C3F8A82035
:10086000012384F8B439BDE87040CFE6E861002088
:10087000589E002058CE0020F8B5134BD3F86C4199
:10088000054604B393F87011C9B9E06866688268D8
:10089000136823F001031360326877790B4E938954
:1008A00036F817609BB223EA0603938121741388FC
:1008B0009BB243F0010313800177FEF739FE204617
:1008C000F9F7C2FA0560F8BDE8610020542B06086C
:1008D00038B5104CD4F86C0150B194F870313BB17C
:1008E00094F8BC39032B04D1F9F7AEFA6423036002
:1008F00038BD022B4FF0000503D1F9F7A5FA0560CA
:10090000F6E784F87051FEF73BFE0028F0D184F83A
:10091000B409EDE7E86100208379806BDB0748BF0D
:1009200081F0010109B1FFF7B5BAFFF7B8BA10B508
:10093000837913F0010F03F020020446C36B12D039
:100940005B68002A1A7A14BF02214221606BFFF70C
:10095000D5FA0121E06B84F86012A4F85C12BDE8BE
:100960001040F9F787BA5B68002A18BF02211A7A8B
:1009700008BF2221EAE7036C806B23B15B68012189
:100980001A7AFFF7BBBA0121FFF78EBA70B58368F8
:100990001C6863799A0731D594F86152D5B194F9FE
:1009A00062329BB1B4F864124B08A4F8643220465A
:1009B00001F00101FFF7B0FF94F86232A279013B28
:1009C0005BB2500684F8623218D5BBB9002384F8B4
:1009D000613213E0A36A626A94F860129A4226D1E7
:1009E00061B9A3791B0709D5236CA06BDBB15B68E8
:1009F0001A7AFFF783FA2046FFF799FF6379D90740
:100A000040F1818094F85C32002B7CD194F85D3207
:100A10000133DBB2092B84F85D3235D12046BDE8C5
:100A20007040FEF7E5BA1946FFF73EFAE3E75A1CB5
:100A3000A069A262C35C26695B0043F40073A4F85A
:100A400064320A23B24234BF1046284684F8623228
:100A50000123A06284F8613291B1A3791E070FD5FA
:100A6000E06B2946F9F706FAE36B606B5B68294691
:100A70001A7AFFF743FA84F860522046FFF77BFFAB
:100A8000A3795D068BD4B9E70A2B3CD194F85F3289
:100A90002BB9B4F8663243F00103A4F86632B4F817
:100AA0006602820501D4C3071AD4B4F86A3201334E
:100AB000A4F86A3294F85F5201239D42A4F85C3294
:100AC00021D1A179E06B002384F85F3201F00101AC
:100AD00045F05CFDE06B2946BDE87040F9F7CAB906
:100AE000E36AC0F3470013B1216B9847E2E7E3697B
:100AF0006269D054E369E2680133B3FBF2F102FBAF
:100B00001133E361D6E770BD234B1A6810B5134665
:100B10000446B3FBF1F0B0F5803F03D3012BFAD9C3
:100B20005B08F6E781B22046F9F726F823681B68D0
:100B3000587990B1032140B2F8F711FF23681B6880
:100B40005A7993F90530002B07DB02F01F010122CF
:100B50008A405B09114941F8232023681B68987972
:100B600090B1032140B2F8F7FAFE23681B689A7926
:100B700093F90630002B07DB02F01F0101228A40A7
:100B80005B09064941F8232063681A6813889BB201
:100B900043F00103138010BD6006002000E100E077
:100BA0008160C06BB0E7002ABCBF80185242002BA6
:100BB000BCBFC9185B420028BCBF121A0020F0B5A8
:100BC00084180029A4F11D04BCBF5B180021002C6F
:100BD000C8BF121BCC180F3C002CC8BF1B1B0B4EF0
:100BE00002440B443C274FF0200C90420CDC06EBF7
:100BF00040050C4604E007FB04FE013425F80EC056
:100C00009C42F8DD0130F0E7F0BD00BFA86B00208A
:100C100008B5114B1A6C42F080521A640F4A012138
:100C200011620F4AFF215162CA2151625321516260
:100C30005B6FDB0005D50020FAF772F9094B98428B
:100C400009D000210120FAF75BF9BDE80840054909
:100C50000020FAF755B908BD0038024000000E42E6
:100C60000028004076614E6970B50446012023F0EB
:100C700013FA58B103684BB11A4A237992F83C1021
:100C800092F83D209A422BD08B4229D0164B5E68B9
:100C9000710612D500212720F8F754FF00210546E0
:100CA0002620F8F74FFF1DB12A6823689A4217D013
:100CB00018B1026823689A4212D0F20308D50021C5
:100CC0002520F8F73FFF18B1226803689A4207D041
:100CD0002079112804D0A0F121035842584170BD59
:100CE0000120FCE74C030020EC550120094A30B5F7
:100CF00005460A2400201368AB4205D1D3688B4215
:100D00001EBF431CD160D8B2013C02F11402F2D1E3
:100D100030BD00BF980500202DE9F74F384DDFF8B2
:100D2000E880DFF8E8904FF0000B06462F465C465F
:100D3000AA463A68002358F833108A4243D1DBB2FE
:100D40004B4493F8803D012B42D0022B49D03846CA
:100D50000192FFF789FF78B9142303FB0BA3019AD3
:100D6000D96801F00C03042B06D11046FFF7BEFF33
:100D70000134E4B20444E4B20BF1010BBBF10A0FFD
:100D800007F11407D5D11F4F2846FFF76DFFA0B913
:100D9000E9684B0711D501F00C03042B0DD0A642D6
:100DA00027D921F0080141F004012868E960FFF724
:100DB0009DFF0134E4B20444E4B21435AF42E3D100
:100DC00003B0BDE8F08F01330E2BB4D1FF23B7E79A
:100DD000FB681807BBD523F0080343F00403FB604E
:100DE000B5E7FB685907B2D523F0040343F00803C5
:100DF000F5E721F004012868E960FFF777FFDCE7F9
:100E00009805002060060020AC2B0608E861002051
:100E100010B5044608462060194608B1F8F7ACFE44
:100E2000BDF808102068F8F7FFFE206843681A68CC
:100E3000B2F844306FEA43436FEA53439BB2A2F8DF
:100E4000443013889BB243F001031380F8F7FCFF92
:100E50000023A060036010BD2DE9F04F85B09946D6
:100E60009DF83C30039307468A469046FCF78EFE79
:100E7000054650B1224B93F88E1D072909D9214A06
:100E800000210420FCF77EFD0025284605B0BDE8C2
:100E9000F08F4A1C5C205FFA82FB83F88EBD03F55D
:100EA000596600FB013301FB00660021C3F8901D69
:100EB00083F8941D3879FFF761F8044628B10223BE
:100EC00080F806A0C37180F808B0039B7BB13A7A22
:100ED00002212046FFF712F8BDF83830009329466A
:100EE0004B4642463046FFF793FF3546CDE7204656
:100EF0001121FEF7D9FF2046FEF7D1FFECE700BF36
:100F0000E8610020BECC06082DE9F347394C14F8FF
:100F1000883C0746002B6BD014F8876C14F8863C8D
:100F20000136F61A102E0DDD022304F8853C324AF4
:100F300010230093002133460420FCF723FD02B068
:100F4000BDE8F08714F87C3C012B11D0022B13D0A4
:100F50002A4B14F87C1C44F8783C11F0FD010FD0AA
:100F6000274A0221042002B0BDE8F047FCF70ABD81
:100F700047F030F8234BECE747F02CF8224BE8E73A
:100F80007B68B34229DBDFF89480DFF88090DFF8DC
:100F900090A028370D46B542D1DADAF8042034F8AB
:100FA000823CB9FBF3F3C2F30072019234F8842C53
:100FB00000920321154A57F8040B9BB2FFF74CFF30
:100FC000014688B90523124A04F8853C04202B46C3
:100FD00002B0BDE8F047FCF7D5BC042000930D4AF1
:100FE00004F8850C3346A8E748F8040B0135D2E72E
:100FF000094AB6E7E0720020F9CC06082BF1000898
:1010000025CD0608C1F7020841F1000840420F0053
:1010100097CD060861CD0608BCCD06089862002071
:10102000EC55012030B51E4B2DED028B1C68B4FB36
:10103000F1F303F57F4383B0FF331B0CB4FBF3F4F0
:101040000023B4FBF1F5019200932246ABB20221DA
:10105000F0EE408AB0EE608AFFF7FEFEE0B107EEE8
:10106000904AB5EE408AF1EE10FAF8EE677A0ABFC0
:1010700007EE105A67EE880AF8EE470A9FED097AE4
:10108000C0EE876A0123037127EE667AC0ED046A19
:10109000A7EEA87A80ED037A03B0BDEC028B30BDD9
:1010A0006006002000007A440023064910B51C4663
:1010B000984200DC10BD51F833200AB192681460E8
:1010C0000133F5E7503E002013B50F4C8DF80700B3
:1010D000D4E90423A16853438B4212D06368E068CB
:1010E0000DF1070118444DF06BFB6368226913444E
:1010F000A268B3FBF2F102FB113363606369013351
:10110000636102B010BD00BF283E00200F4B1B786A
:10111000062B14D8DFE803F0161304070A0D10009D
:101120004FF4FA6070470A4B988870474FF47A6022
:1011300070474FF4FA5070474FF47A5070474FF4AD
:101140007A7070474FF4C870704700BF043E0020AB
:10115000903F00202DE9F04F2DED028B6A4B6B4E36
:101160001F780C2F85B081460FDD012306F8853CE2
:10117000674A0C2300933B4600210420FCF702FC45
:1011800005B0BDEC028BBDE8F08F624B9C79624BE1
:10119000032C1C7013D9231F022B12D95F4B46F866
:1011A000743C5F4B13F81430F3B95E4A02210420FB
:1011B00005B0BDEC028BBDE8F04FFCF7E3BB5A4B2A
:1011C000EDE7FFF7A3FF594A594B80B2B3FBF0F0AC
:1011D00000235360574B10604FF0000A4FF0000B94
:1011E000C3E900AB544BDAE7D9F80030BB421ADB55
:1011F000524CDFF874B19FED528A09F108094FF0A3
:101200000008B845BCDA444BDBF804201B7859F8D9
:10121000045BC2F30072062B6FD8DFE803F0642989
:10122000310B3B3B3B00032206F8852C0093454ADB
:101230003B46A1E70392FFF769FFDFED430A039AFC
:101240000146B0EE600A2846FFF7ECFE206054F835
:10125000081B002954D105233C4A06F8853C04208C
:10126000434605B0BDEC028BBDE8F04FFCF78ABBEE
:101270000392FFF74BFFDFED360A039A0146E0E7E2
:101280000392FFF743FFDFED330A039A9FED320A23
:101290000146D8E7052B24D030493148062B08BF3A
:1012A00001464FF0000A019228460A46CDF800A0F8
:1012B00014230221FFF7D0FD054680B100F114038D
:1012C000194600680393122245F012FA039B30B1CD
:1012D0001846482251464FF011FC01232B7125601E
:1012E000B5E72049DDE70392FFF710FF9FED140AF1
:1012F000039A0146F0EE480AA5E700232360A6E71B
:1013000008F101087DE700BFE8550120E0720020E8
:10131000D6CD0608903F0020043E002029F10008A9
:10132000B82C060802CE060881F40008103E002002
:1013300040420F00183E002053F10008503E0020AC
:101340006F12833A20CE06080000000059CE06082E
:101350006F120339ACC5A737ACC5A736C0C62D0080
:10136000001BB700808D5B00EC550120034A52F84A
:10137000782C12B10F2800D810477047E072002077
:1013800050B10138002330F0FF019AB203F101039C
:1013900003D140EA022080B270474008F3E70368B7
:1013A0001B68184703685B68184703689B68184701
:1013B0000368DB6970B506460C46154683B1BDE887
:1013C000704018473046FFF7F0FF0028FAD014F8B5
:1013D000011B3046FFF7E3FF2B1B002BF2DC70BD37
:1013E0000D44F9E7E4E70368DB68184703681B6905
:1013F000184703685B69184703689B6A03B118477D
:1014000070470368DB6A03B118477047164B1B68C7
:1014100013F0100F154B05D033F8702C12F0040F99
:1014200018BF002013F8562C72B153F8542CCAB1CF
:10143000926838B133F8501C0D4BB3FBF1F35B10DD
:10144000136070471060704753F84C2C13F8483CF9
:101450000BB980F001002AB11368928808B11A8391
:1014600070475A83704700BF50550120E07200203A
:1014700040420F00BFF34F8F0549064BCA6802F484
:10148000E0621343CB60BFF34F8F00BFFDE700BFA7
:1014900000ED00E00400FA0508B572B600224FF036
:1014A000FF31930003F1604303F561430132082AE1
:1014B000C3F88010C3F88011F3D1FFF7DBFF0121DF
:1014C00008B50846F9F71CFDFFF7E6FF08B501204F
:1014D000F9F726FD012809D10021F9F711FD044B88
:1014E0001A6882F308885B689847FEE708BD00BF6A
:1014F0000000FF1FEFF31183102282F312880949C5
:101500000A6801320A604FF0E0220749906941F809
:10151000440C002041F8400C1269DBB283F31188BF
:10152000704700BF842B0020E0720020064A074B62
:1015300051681B6858434FF47A73B0FBF3F053685B
:101540005B1A8342FBD97047001000E0B42C0020E6
:1015500010B504464FF4FA70FFF7E8FF6069BDE884
:101560001040FEF797BC90F9103073B51546142261
:1015700053430D4AD65883689A07044604D44069F9
:10158000019147F0BBFB0199304648F0D9FC294650
:10159000304648F0D5FCA3689B0702D42046FFF7ED
:1015A000D7FF012002B070BDB00000207FB50379E5
:1015B000012B0D460AD0022B19D18368DB0758BFD7
:1015C00001F07F0104B0BDE87040CCE781688DF880
:1015D0000F2001F001010DF10F0200920191417CF9
:1015E00090F910002A46F9F72FFB04B070BD0020D7
:1015F000FBE700682E22F421D8E7044B00681A8E1E
:101600009201343202F0FC02F421CFE7E8610020BD
:1016100008B53122F4210068FFF7C8FF012008BD9A
:10162000006801225821C1E7006801224821BDE776
:10163000006802220821B9E7006801220821B5E705
:1016400010B50446002221210068FFF7AFFF206893
:10165000FC222021FFF7AAFF206840222421FFF767
:10166000A5FF20680C222321FFF7A0FF206800229D
:101670002221FFF79BFF012010BD10B50122044677
:101680000B210068FFF792FF20B120681D2209217D
:10169000FFF78CFF00F0010010BD044B024653F829
:1016A0003C0C08B1802181E7704700BFE072002048
:1016B00010B5B020FFF7F1FF4020FFF7EEFF00204C
:1016C000FFF7EBFF1020FFF7E8FF4FF48064013CC9
:1016D0000020A4B247F065F8002CF8D110BD5039B5
:1016E00010B50446C8B2FFF7D8FF04EB4400400031
:1016F00004EB440400F00E00FFF7CFFFC4F3C30077
:101700001030BDE81040C8E708B55038C0B2FFF748
:10171000C4FF0020FFF7C1FFBDE808401020BCE770
:1017200038B500221F2333210120FEF7D7FD3D4BA2
:1017300043F83C0C10B90024204638BDAE20FFF71A
:10174000ACFF04460028F6D0D420FFF7A6FF802087
:10175000FFF7A3FFA820FFF7A0FF3F20FFF79DFFA3
:10176000D320FFF79AFF0020FFF797FF4020FFF7F5
:1017700094FF8D20FFF791FF1420FFF78EFFA1202B
:10178000FFF78BFFC820FFF788FFDA20FFF785FF00
:101790001220FFF782FF8120FFF77FFFCF20FFF7A6
:1017A0007CFFD920FFF779FFF120FFF776FFDB20E0
:1017B000FFF773FF4020FFF770FFA420FFF76DFFD6
:1017C000A620FFF76AFFAF20FFF767FFA620FFF70D
:1017D00064FFAE20FFF761FF2020FFF75EFF0020CF
:1017E000FFF75BFFB020FFF758FF4020FFF755FFE2
:1017F0000020FFF752FF1020FFF74FFF4FF48065E6
:10180000013D0020ADB246F0CCFF002DF8D1812083
:10181000FFF743FFC820FFF740FFAF20FFF73DFF72
:101820008AE700BFE072002008B5FFF7BFFE014B5A
:10183000187008BD38100020F7B51E4690F910301A
:101840001546142253430E4AD75883689A07044614
:1018500004D44069019147F051FA0199384648F0A3
:101860006FFB33462A460021384648F001FBA36847
:101870009B0702D42046FFF76BFE012003B0F0BDAA
:10188000B0000020F7B50779012F16460AD0022FC5
:1018900015D18468E40758BF41F0800103B0BDE86A
:1018A000F040C9E7826802F00102CDE900620A4611
:1018B000417C90F91000F9F7C7F903B0F0BD0020A2
:1018C000FBE707B5130A8DF804308DF805200223D5
:1018D00001AAFFF7D7FF024B187003B05DF804FBB5
:1018E0003810002010B50A4C002304F8383C04F8E6
:1018F000371C04F8362C0323A4F13802FF21FFF72C
:10190000C1FF00280CBF6FF00C00002010BD00BF0D
:10191000E072002010B50B4C002304F8383C130A89
:1019200004F8371C04F8363C04F8352C0423A4F1E1
:101930003802FF21FFF7A6FF00280CBF6FF00C0054
:10194000002010BDE0720020024A006800235121EF
:1019500098E700BFA8730020F7B51E4690F9103035
:101960001546142253430E4AD75883689A070446F3
:1019700004D44069019147F0C1F90199384648F013
:10198000DFFA334600222946384648F071FAA36848
:101990009B0702D42046FFF7DBFD012003B0F0BD1A
:1019A000B0000020F7B50779012F16460AD0022FA4
:1019B00015D18468E40758BF41F0800103B0BDE849
:1019C000F040C9E7826802F00102CDE900620A46F0
:1019D000417C90F91000F9F75DF903B0F0BD0020EB
:1019E000FBE713B5062304466A4600680221FFF7A9
:1019F000D9FFB8B1BDF9003007EE903ABDF9023019
:101A0000F8EEE77AC4ED077A07EE903ABDF90430B4
:101A1000F8EEE77AC4ED087A07EE903AF8EEE77A46
:101A2000C4ED097A02B010BD13B5022304466A461C
:101A300000680321FFF7B6FF10B9002002B010BD07
:101A40009DF90130002BF8DA206807236A4612213D
:101A5000FFF7A8FF0028F0D09DF902209DF8013083
:101A600043EA022313EB430348BF03339B1007EE03
:101A7000903A9DF904209DF8033043EA022313EBCA
:101A80004303F8EEE77A48BF03339B109DF9062025
:101A9000C4ED047A07EE903A9DF8053043EA02233C
:101AA00013EB4303F8EEE77A48BF03339B10C4ED12
:101AB000057A07EE903AF8EEE77AC4ED067ABDE7CC
:101AC00038B504460068FDF77BFF0C230546021D70
:101AD00019462068FFF766FFA870B8B1B5F9043061
:101AE00007EE903AF8EEE77AC4ED077AB5F90630DA
:101AF00007EE903AF8EEE77AC4ED087AB5F90830C7
:101B000007EE903AF8EEE77AC4ED097A38BD38B5B9
:101B100004460068FDF754FF0D230546C21C0C2146
:101B20002068FFF73FFFA870B8B1B5F90A3007EE9B
:101B3000903AF8EEE77AC4ED077AB5F90C3007EE83
:101B4000903AF8EEE77AC4ED087AB5F90E3007EE70
:101B5000903AF8EEE77AC4ED097A38BD13B503235D
:101B60000C46006801AA2221FFF71CFF30B1BDF925
:101B7000053003EB83031B12E633238002B010BD54
:101B800013B5062304466A4600681F21FFF70AFFC3
:101B9000D0B1BDF80030DBBA07EE903ABDF80230A4
:101BA000F8EEE77ADBBAC4ED047A07EE903ABDF8B6
:101BB0000430F8EEE77ADBBAC4ED057A07EE903A26
:101BC000F8EEE77AC4ED067A02B010BD13B506232D
:101BD00004466A4600682521FFF7E4FED0B1BDF84F
:101BE0000030DBBA07EE903ABDF80230F8EEE77A43
:101BF000DBBAC4ED077A07EE903ABDF80430F8EE90
:101C0000E77ADBBAC4ED087A07EE903AF8EEE77AA5
:101C1000C4ED097A02B010BD70B5066805463046BD
:101C2000FDF7CEFE0E230446021D3B213046FFF792
:101C3000B9FEA070B8B1A389DBBA07EE903AF8EE0E
:101C4000E77AC5ED077AE389DBBA07EE903AF8EE5A
:101C5000E77AC5ED087A238ADBBA07EE903AF8EE08
:101C6000E77AC5ED097A70BD07B50223006801AABD
:101C7000F621FFF797FE20B1BDF80430024A5BBAA7
:101C8000138203B05DF804FBE861002007B503236D
:101C9000006801AAF621FFF785FE80B19DF80530A6
:101CA0009DF8042007491B0243EA02439DF80620E1
:101CB0001343B1F93020C2F10802D3404B6303B0A3
:101CC0005DF804FBE861002037B50623F7210068C2
:101CD000144C6A46FFF766FE1349D8B19DF80120FF
:101CE0009DF800309DF80350120142EA03329DF83E
:101CF000023042EA13129DF804308A651B0143EA60
:101D000005339DF8055043EA1513C4E932238B636C
:101D100003B030BDD4F8C8308B65D4F8CC308B63B9
:101D2000F6E700BFE0720020E861002007B503235A
:101D3000006801AA1946FFF735FEA0B19DF80430EE
:101D40009DF805109DF904201B0443EA01239DF82A
:101D50000610002AB4BF4FF07F4200220B4313430A
:101D6000024AC2F8183103B05DF804FBE8610020B4
:101D700007B50323006801AA0021FFF713FEA0B1F5
:101D80009DF804309DF805109DF904201B0443EADA
:101D900001239DF80610002AB4BF4FF07F420022B5
:101DA0000B431343024AC2F8FC3003B05DF804FB56
:101DB000E861002013B5044600680379022B0CBFCC
:101DC0004321032106236A46FFF7ECFD18B9E0869C
:101DD000A06302B010BDBDF800305BBAE386BDF869
:101DE00002305BBA6387BDF804305BBA2387F0E743
:101DF00013B50023C38683630446062300686A463E
:101E00000321FFF7CFFD78B1BDF8003003EB4303AA
:101E1000E386BDF902305B4203EB43032387BDF841
:101E2000043003EB4303638702B010BD07B5012301
:101E300001AAFF210068FFF7B5FD03B05DF804FBC0
:101E4000F7B505460068FDF7BBFD002303700423CA
:101E500004460DEB03022868FF21FFF7A3FD10B92C
:101E6000002003B0F0BD286804236A46FF21FFF775
:101E700099FD0028F4D09DF804108A09023A012A3D
:101E8000EED99DF8053003EB012343F6FF75C3F34C
:101E90000D03AB42E4D0002BE2D09DF806109DF874
:101EA000072040F2FF7702EB0122B7EB521F4FEA07
:101EB0006211D5D00029D3D09DF800609DF8012093
:101EC00002EB0622C2F30D02AA42C9D0002AC7D0F3
:101ED0009DF802609DF8035005EB0625B7EB551FF2
:101EE0004FEA6516BCD0002EBAD09D1A002DB8BF9F
:101EF0006D42FF2DB4DC8D1B002DB8BF6D42FF2D50
:101F0000AEDC0125134431442B4129412570C4F82E
:101F10000530C4F80110A4E773B505460068FDF765
:101F20004FFD00260423044606700DEB03022868CB
:101F3000FF21FFF737FD48B19DF804108B0907D04A
:101F400003200D4A0421FBF71DFD304602B070BD91
:101F50009DF805209DF8073002EB01229DF8061040
:101F600003EB012392B25B1101212170C4F805201B
:101F7000C4F80130EAE700BF7ECE060807B50223A9
:101F800001AAFFF70FFD044B1870BDF8040040BA1A
:101F900080B203B05DF804FB3810002038B5154658
:101FA0000C4A0B0A02F8383C02F8371C0223383A74
:101FB000FF210446FFF766FC10B96FF00C0038BD36
:101FC00001232A46FF212046FFF7ECFC0028F4D02D
:101FD0000020F4E7E0720020F8B5124D164605F82F
:101FE000371CA5F1380200240223FF21074605F81B
:101FF000384CFFF747FCA5F1380210B96FF00C0020
:10200000F8BD0223FF213846FFF7CCFC0028F5D0AD
:1020100015F8382C15F8373C03EB022333802046A3
:10202000EEE700BFE07200202DE9F341744D046833
:10203000DFF8D8810023064685F8F2302D27B9B2A3
:1020400018F8012B20460137FFF74CFC882FF6D1FA
:10205000402287212046FFF745FC00238DF80630FB
:102060000DF10601204646F0FFFA9DF80630002BE0
:10207000F6D0012286212046FFF734FC002287217A
:102080002046FFF72FFC092208212046FFF72AFCF3
:1020900000220B212046FFF725FC002852D137688B
:1020A0000DF106025E213846FFF796FFBDF80630B7
:1020B000B3F5D77F00F0A08054D8512B00F09A8060
:1020C00048D81D2B6BD01E2B00F094803068212146
:1020D00046F039FA34680DF10602DE212046FFF79A
:1020E0007BFFBDF806309FED477AC3F30903282232
:1020F000ADF80630534307EE903AF8EEE77A424ADD
:1021000067EE877A0021FCEEE77A02F8381C17EEBA
:10211000903A6C2102F8371C190E02F8361C190C83
:1021200002F8351C190A02F8341C02F8333CFF216E
:10213000383A06232046FFF7A5FB30684022872166
:10214000FFF7D0FBB0FA80F0400985F8F20002B04A
:10215000BDE8F081AD2B4FD0D62B01D0602BB5D18F
:1021600021241DE040F2E132934247D00CD840F2E6
:10217000D922934242D040F2E122934202D0B3F5F9
:10218000E67FA3D164240BE040F28F42934203D058
:1021900040F29152934299D14FF4FA7400E00F2427
:1021A000002893D10A224B213846FFF79BFB0F22D0
:1021B00060213846FFF796FB0D2263213846FFF772
:1021C00091FBB82269213846FFF78CFB40F60D726F
:1021D00078213846FFF79EFB40F60E627A2138469A
:1021E000FFF798FB00287FF471AF2146384646F090
:1021F000AAF96BE71424D3E73224D1E7C824CFE748
:10220000E86100209A99893FE0720020903006082A
:1022100037B5124D95F8F2300446E3B100680DF180
:10222000050146F021FA9DF805307BB10DF106025B
:1022300020689621FFF7D0FE0A22BDF80630B3FBD6
:10224000F2F3074A9360012385F8F33020680122F6
:102250008621FFF747FB03B030BD00BFE8610020D7
:102260003810002013B5022301AA0446512100684A
:10227000FFF798FB114AE8B1BDF804305BBA9BB296
:10228000D360D368B3F5C87F02DD4FF0FF33D3606E
:102290000B4B0C4A1968D2F8D03032338B4207D23C
:1022A000C2F8D01020680023C8325121FFF7EAFAA3
:1022B00002B010BD6FF00103E9E700BF3810002045
:1022C000842B0020E072002007B50223006801AAD9
:1022D0000021FFF767FB0F4B83F8F800B0B1BDF8A2
:1022E00004300D4A5BBA9BB2B3F5FA6F3FBF0A21C7
:1022F000B3FBF1F307EE903AF8EEE77A2BBF4FF01D
:10230000FF33FDEEE77A1361C2ED047A03B05DF8A6
:1023100004FB00BFE86100203810002013B5022341
:102320000C46006801AA0021FFF73CFB60B15CB1DC
:102330009DF805309DF90420DB0903EB830302EBD4
:10234000820203EB4203238002B010BD90F91030EB
:1023500073B51546142253430E4AD65883689A071C
:10236000044604D44069019146F0C8FC0199304606
:1023700047F0E6FD012300222946304647F078FD6C
:10238000A3689B0702D42046FFF7E2F8012002B0C1
:1023900070BD00BFB000002073B50379012B164655
:1023A0000AD0022B15D18368DB0758BF41F08001AA
:1023B00002B0BDE87040C9E7826802F00102CDE9D1
:1023C00000620A46417C90F91000F8F763FC02B005
:1023D00070BD0020FBE7F7B515460DF107021C465E
:1023E00006460F46FFF7D8FF9DF8073005EA0302BF
:1023F000A24209D023EA050222433946304603B0FF
:10240000BDE8F040FFF7D2B803B0F0BD13B5044605
:102410006A4600680821FFF7BFFF9DF8003013F0FF
:1024200010037ED0206806236A460021FFF7BAFA1F
:10243000002874D09DF801309DF800209FED3A6A85
:102440009DF804101B0203EB02439DF802201C02BE
:102450001A4448BF02F17F4207EE902AF8EEE77A6D
:102460009DF80330C7EE866A090201EB03419DF82F
:1024700005300B44090248BF03F17F4307EE903A51
:102480002A4BB3F97020B8EEE77A07EE902AB3F939
:102490006C20C7EE065A06EE102AF8EEE77AB8EE80
:1024A000C66AB3F96820A6EEA76AD3ED197AB8EE2A
:1024B000E77AD3ED187AA6EE867AF8EEE77A26EE7A
:1024C000A55AE6EE877A07EE102AB3F96E20B8EE29
:1024D000C77A06EE102AB3F96A20E5EE877A07EE8E
:1024E000102AB8EEC66AB8EEC77AB3F95C20A6EE39
:1024F000867AF6EE006AE5EE077A07EE102AB3F95F
:102500005E20C3ED1D7A07EE902AF8EEE77AB8EE6A
:10251000C77A67EEA57AE7EE267AC3ED1E7A02B097
:1025200010BD1846FBE700BF00007848E8610020B6
:102530001FB50446002300688DF807300DF107022F
:102540002721FFF729FF68B19DF8073013F0080332
:1025500020D02068062302AA2821FFF723FA18B901
:10256000E086A06304B010BDBDF90830002BB8BFF1
:1025700003339B10E386BDF90A30002BB8BF033349
:102580009B102387BDF90C30002BB8BF03339B1081
:102590006387E7E71846E5E71FB500210446C186D3
:1025A00081630DF107020068FFF7F6FEC0B19DF8E8
:1025B000073013F0080315D02068062302AA012172
:1025C000FFF7F0F960B1BDF808305BBAE386BDF8FB
:1025D0000A305BBA2387BDF80C305BBA5B42638775
:1025E00004B010BD1846FBE730B5002585B00446A1
:1025F000C58685630DF1070200680621FFF7CCFE52
:10260000A0B19DF8073013F0040311D02068062311
:1026100002AA2946FFF7C6F940B1BDF80830E386A3
:10262000BDF80A302387BDF80C30638705B030BD94
:102630001846FBE707B50DF10702FFF7ADFE034BA8
:1026400018709DF8070003B05DF804FB38100020F7
:10265000F8B5144E144F41F0010200210446FFF773
:10266000E3F83568C7F8D45013212046FFF7E2FF9E
:1026700010F007000BD001220B212046FFF7D4F801
:10268000002220461146FFF7CFF8012008E0D7F8D6
:10269000D820002AE8D033689BB25B1B9A42E3D271
:1026A000F8BD00BF842B0020E072002010B50C465E
:1026B0000121FFF7BFFFC0F300132370C0F3C00375
:1026C000A370C0F380036370C0F38013C0F3C01025
:1026D000E370207110BD2DE9F04788465021144663
:1026E0000646FFF7A7FF01304000C0B22080462118
:1026F0003046FFF79FFF2D4F2378013080B27B4398
:102700004FF47A79A08003F5FA734FF4FA6AB3FBB9
:10271000F9F25121B3FBFAF300FB02333046B3FB6D
:10272000F9F3E360FFF72AFCC3B2C0F30F22257868
:1027300003FA02F2013293B27D43E38005F5FA72A7
:102740003046B2FBF9F1B2FBFAF203FB0122702131
:10275000B2FBF9F22282FFF76DFF01304000C0B2F8
:10276000608071213046FFF709FCC3B2C0F30F202F
:102770008340013398F803209BB2238112B1E28891
:102780009B1A2381A37820897B4303F5FA734FF4C6
:102790007A724FF4FA65B3FBF2F1B3FBF5F300FB89
:1027A0000133B3FBF2F36382BDE8F087002F3A00F8
:1027B0002DE9F047DB4FDFF87483DFF874934FF4B3
:1027C000FA738CB00446002689210068C7F8D83017
:1027D00088F8F060FFF72EFF40F00100C2B28921B7
:1027E0002068FFF721F8324620688821FFF71CF89F
:1027F000206801228021FFF717F820680122FF21BD
:10280000FFF712F8324631462068FFF70DF89121A4
:102810002068FFF70FFF314687F8DC0001222068AF
:10282000FFF702F832462068FF21FEF7FDFF32462F
:1028300020688021FEF7F8FF60212068FFF7FAFE8C
:1028400040F01200C2B260212068FEF7EDFF206860
:1028500020224421FFF735F82068FF220121FEF7EE
:10286000E3FF2568012280212846FEF7DDFF0122D3
:10287000FF212846FEF7D8FF324631462846FEF7AC
:10288000D3FF0622FF212846FEF7CEFF83212846EC
:10289000FFF7D0FE40F00400C2B283212846FEF7C5
:1028A000C3FF0722FF212846FEF7BEFF0122812138
:1028B0002846FEF7B9FF012280212846FEF7B4FF23
:1028C0006B2294212846FEF7AFFF3246832128462B
:1028D000FEF7AAFFD9F80060C7F8D4608321284624
:1028E000FFF7A8FE002800F052830122284683212A
:1028F000FEF79AFF92212846FFF79CFE0022C0F3C4
:10290000C716814681212846FEF78EFF06222846FB
:10291000FF21FEF789FF83212846FFF78BFE8321E5
:1029200000F0FB022846FEF77FFF28460122FF2128
:10293000FEF77AFF284601220021FEF775FF2846A0
:102940000022FF21FEF770FF284600228021FEF7BB
:102950006BFF062305AAB0212068FFF723F8206843
:102960000122FF21FEF760FF206800224F21FEF7C1
:102970005BFF20682C224E21FEF756FF20680022C4
:10298000FF21FEF751FFB4222068B621FEF74CFF6D
:102990000025002E18BF0C2609F07F092A464FF0AB
:1029A000010CC5F3C40000F130035FFA85FE0DEBA6
:1029B0000300764510F81C3C05F0070102D891454C
:1029C00040F0F0820CFA01F123EA010300F81C3C0C
:1029D0000135302DE5D1062305AAB0212068FEF788
:1029E00051FF514B01221870FF212068FEF71CFF98
:1029F000002211462068FEF717FF20680022FF2101
:102A0000FEF712FF206800220921FEF70DFF206863
:102A100000221021FEF708FF206800221121FEF796
:102A200003FF206801222421FEF7FEFE2068FF221A
:102A30002521FEF7F9FE206800227521FEF7F4FE3D
:102A400020680122FF21FEF7EFFE20682C224E2194
:102A5000FEF7EAFE206800224821FEF7E5FE29463F
:102A600020682022FEF7E0FE20680022FF21FEF70A
:102A7000DBFE294620680922FEF7D6FE20680022E8
:102A80005421FEF7D1FE206804223121FEF7CCFE4E
:102A9000206803223221FEF7C7FE206883224021EE
:102AA000FEF7C2FE206825224621FEF7BDFE206803
:102AB00000226021FEF7B8FE206800222721FEF7E1
:102AC000B3FE206806225021FEF7AEFE20680022E9
:102AD0005121FEF7A9FE206896225221FEF7A4FE9E
:102AE000206808225621FEF79FFE2A4620685721BB
:102AF000FEF79AFE206800226121FEF795FE20680D
:102B000000226221FEF790FE206800226421FEF779
:102B10008BFE206800226521FEF786FE2068A02239
:102B2000662107E0E072002038100020E8610020F4
:102B3000842B0020FEF778FE20680122FF21FEF79B
:102B400073FE206832222221FEF76EFE20681422D6
:102B50004721FEF769FE2068FF224921FEF764FE47
:102B6000206800224A21FEF75FFE20680022FF2134
:102B7000FEF75AFE20680A227A21FEF755FE2068E9
:102B800000227B21FEF750FE206821227821FEF7EB
:102B90004BFE20680122FF21FEF746FE206834220A
:102BA0002321FEF741FE206800224221FEF73CFE71
:102BB0002068FF224421FEF737FE206826224521A7
:102BC000FEF732FE206805224621FEF72DFE402248
:102BD00011462068FEF728FE206806220E21FEF727
:102BE00023FE20681A222021FEF71EFE20684022C4
:102BF0004321FEF719FE20680022FF21FEF714FE94
:102C0000206803223421FEF70FFE2068442235217C
:102C1000FEF70AFE20680122FF21FEF705FE20686C
:102C200004223121FEF700FE206809224B21FEF725
:102C3000FBFD206805224C21FEF7F6FD20680422EA
:102C40004D21FEF7F1FD20680022FF21FEF7ECFD8B
:102C5000206800224421FEF7E7FD2068202245215C
:102C6000FEF7E2FD206808224721FEF7DDFD20681F
:102C700028224821FEF7D8FD206800226721FEF7B0
:102C8000D3FD206804227021FEF7CEFD20680122CA
:102C90007121FEF7C9FD2068FE227221FEF7C4FDF6
:102CA000206800227621FEF7BFFD206800227721F0
:102CB000FEF7BAFD20680122FF21FEF7B5FD20686E
:102CC00001220D21FEF7B0FD20680022FF21FEF752
:102CD000ABFD206801228021FEF7A6FD2068F822C6
:102CE0000121FEF7A1FD20680122FF21FEF79CFDD6
:102CF000206801228E21FEF797FD20680122002125
:102D0000FEF792FD20680022FF21FEF78DFD20686E
:102D100000228021FEF788FD042220680A21FEF7A8
:102D200083FD256884212846FFF784FC842100F078
:102D3000EF022846FEF778FD012220680B21FEF7FE
:102D400073FD2068019003A9FFF7B0FC019807AA62
:102D500003A9FFF7C0FC9DF80C30002B00F0288180
:102D60000A9D05F684559DF80E30002B00F0238156
:102D70000A9B03F2B22305EB43059DF80F3023B104
:102D8000BDF82C3003F525731D449DF8103023B198
:102D9000BDF82E3003F226231D442068C7F8E0500A
:102DA000E8220121FEF740FD44F61F639D4203D94E
:102DB0002068294645F078FC012220681146FEF77C
:102DC00033FD20684021FFF743FC002800F0E78036
:102DD000206801210222FEF727FD20680021FFF76D
:102DE00037FC002800F0DB802068DFF8E491E8225F
:102DF0000121FEF719FD202220684421FEF761FD24
:102E0000256803A92846FFF751FC07AA03A928460D
:102E1000FFF761FC502257212846FEF705FD0822E6
:102E200056212846FEF700FD082250212846FEF7CD
:102E3000FBFCBDF82C004FF47A7A48F20E660AFBD0
:102E40000060B0FBF9F080B2FEF79AFA5121024619
:102E50002846FEF736FD0A9A5C4B0AFB02669E4244
:102E60009DBFB6FBF9F202F1FF32D2B2FF2246213A
:102E70002846FEF7D9FCD7F8E01044F61F639942C4
:102E800002D9284645F010FC01212846FFF7D2FB65
:102E90000222064601212846FEF7C6FC00212846EC
:102EA000FFF7D6FB324601212846FEF7BDFC246819
:102EB00003A92046FFF7FAFB07AA03A92046FFF75C
:102EC0000AFC482211462046FEF7AEFC08224721A4
:102ED0002046FEF7A9FC032232212046FEF7A4FC7F
:102EE000072230212046FEF79FFC0122FF212046C9
:102EF000FEF79AFC202230212046FEF795FC0022A6
:102F0000FF212046FEF790FC062220467021FEF7A6
:102F10008BFCBDF82E304FF47A7246F6440002FB6B
:102F200003004DF28803B0FBF3F09DF80F3080B240
:102F30001BB1BDF82230184480B2FEF721FA71218E
:102F400002462046FEF7BDFCD7F8E01044F61F63AA
:102F5000994202D9204645F0A7FB01212046FFF700
:102F600069FB0222054601212046FEF75DFC002197
:102F70002046FFF76DFB2A4601212046FEF754FC50
:102F80006423C7F8D830012388F8F03007E0D9F877
:102F900000309BB29B1BB3F5FA7F7FF69FAC0CB061
:102FA000BDE8F0870B41DB0744BF0132D2B20FE529
:102FB00040F63635D7E69DF80D30002B3FF4DDAEF8
:102FC0000A9B03F525731D44D7E600BF1B280D019E
:102FD0001C0C0100F8B53B4F97F8F0300446002B6D
:102FE00037D0394D95F8E460012E33D0022E4FD002
:102FF0007EBB006801228021FEF716FC20680122BA
:10300000FF21FEF711FC206832463146FEF70CFC2A
:1030100095F8DC2020689121FEF706FC206801224B
:103020003146FEF701FC20683246FF21FEF7FCFB2B
:10303000206832468021FEF7F7FB206801223146E6
:10304000FEF7F2FB214B1B68C5F8D430012385F84D
:10305000E430F8BD00680021FFF7ECFAC20711D593
:10306000D5F8D820002AF4D0184BD5F8D4101B6816
:103070009BB25B1A9A42ECD2154B4FF0FF325A606A
:103080000023E4E7114B1B68C5F8D4300223DEE7C8
:1030900000681321FFF7CEFA4307E1D01E21206814
:1030A000FEF76CFF012206460B212068FEF7BCFBF1
:1030B000074B0A20B6FBF0F6B6B25E60012387F834
:1030C000F130DDE7E8610020E0720020842B002071
:1030D0003810002010B5EFF31182102383F312880B
:1030E0004FF0E023D2B29C69196911F4803F0D4979
:1030F0001EBF012041F8400C9C690B4B186851F829
:10310000403C82F31188094A11684FF47A720344F3
:1031100002FB01F0001BB0FBF1F00021E3FB020118
:1031200010BD00BFE0720020842B0020B42C0020D2
:10313000124B5B68C3F3080330B4EBB9EFF31183B0
:10314000D3B90F4B0F484FF0E0251968AC691A68E6
:103150008A42FAD150F8441CA142F6D30A4B1968AE
:103160004FF47A7303FB01F0001BB0FBF1F0002178
:10317000E2FB030130BC704730BCABE700ED00E080
:10318000842B0020E0720020B42C002010B5074CE6
:1031900094F8E90040B1FFF7CBFFD4F8F030C01A43
:1031A000C0F5FA5020EAE07010BD00BFE0720020C8
:1031B000F8B506460D46FFF7BBFF04460F46FFF77E
:1031C000B7FF031B61EB0702B34272EB0503F6D3B3
:1031D000F8BD38B50D460446FFF7D8FF011E02DDE5
:1031E000C917FFF7E5FF064B2068002283F8E920A6
:1031F000492193F8EA302A46FEF7D4FB012038BD76
:10320000E07200202DE9F341364CD4F8F830C0F8D4
:103210003630B4F8FC30438794F8E830012B05468B
:1032200000F1360704F1F8060AD0022B23D08BBB3D
:103230000122022143F039FF012384F8E83002E043
:10324000FFF7A4FF28B194F8FE20104602B0BDE8B5
:10325000F08169462846FFF7BCFF18B19DF80030A1
:103260009B0701D10023E8E707220321284643F00A
:103270001CFF0223E1E7FFF789FF0028E3D169463D
:103280002846FFF7A6FF9DF80630024610B113F05E
:10329000080805D0002284F8E82084F8FE20D4E74E
:1032A000B4F900116846FBF755FE4042B4F902112B
:1032B000E8860DF10200FBF74DFEB4F904112887F2
:1032C00001A8FBF747FED5F83630C4F8F830404285
:1032D0006887BB88B380012384F8E88084F8FE30D7
:1032E000B3E700BFE072002010B50446013C00D2F5
:1032F00010BD4FF47A700021FFF75AFFF6E710B5C2
:10330000044600210068FCF711FBB6221421206856
:10331000FEF74CF96420FFF7E7FF812210212068B7
:10332000FEF744F90120FFF7DFFF15212068802216
:10333000FEF73CF90120FFF7D7FF20680321BDE825
:103340001040FCF7F3BA10B5044600210068FCF702
:10335000EDFAB6227E212068FEF728F96420FFF7F7
:10336000C3FF00227C212068FEF720F96420FFF7CC
:10337000BBFF04227D212068FEF718F96420FFF7C7
:10338000B3FF8C2240212068FEF710F90120FFF7DF
:10339000ABFF022241212068FEF708F90120FFF768
:1033A000A3FF20680221FCF7C1FA4FF40063A38158
:1033B00010BD10B504464069FCF771FD0120FFF710
:1033C00093FF6069FCF766FDBDE810400A208BE7BB
:1033D00073B50468B6227E2105462046FEF7E6F85E
:1033E0006420FFF781FF02212046FCF79FFA204668
:1033F000FFF7DFFF00227C212046FEF7D7F80120EF
:10340000FFF772FF002259212046FEF7CFF8012076
:10341000FFF76AFF5E238DF8073094F9103014220D
:1034200053433D4AD658A3689A0702D4606945F0D1
:1034300065FC01230DF107020021304646F018FD1E
:103440004FF4A473354A0021304646F011FDA368BD
:103450009B0702D42046FEF77BF80A20FFF744FFC3
:10346000012259212046FEF7A1F80120FFF73CFF79
:103470008C2240212046FEF799F80120FFF734FF07
:10348000032241212046FEF791F80120FFF72CFF8F
:10349000234EA96B234A95F83500B6FBF1F10923B9
:1034A00089B2FBF7C9FE4388B6FBF3F62E640279B6
:1034B000422142F0C0022046FEF778F80120FFF7D3
:1034C00013FF082243212046FEF770F80120FFF782
:1034D0000BFF042258212046FEF768F80120FFF771
:1034E00003FF0A2253212046FEF760F80120FFF770
:1034F000FBFE00227C212046FEF758F80120FFF752
:10350000F3FE06227D212046FEF750F8012002B08E
:10351000BDE87040E8E600BFB0000020EB300608D0
:1035200040420F0034320608F8B5816B0468294A1E
:10353000294FB7FBF1F10546102389B290F8350009
:10354000FBF77AFE00214388B7FBF3F706462F64AA
:103550002046FCF7EBF980226B212046FEF726F887
:103560006420FFF7C1FE032268212046FEF71EF803
:103570006420FFF7B9FE01226B212046FEF716F802
:103580000F20FFF7B1FE18221B212046FEF70EF890
:103590000F20FFF7A9FE18221C212046FEF706F88F
:1035A0000F20FFF7A1FE32791A212046FDF7FEFF1A
:1035B0000F20FFF799FE727919212046FDF7F6FFDB
:1035C0006420FFF791FE20460321BDE8F840FCF798
:1035D000ADB900BF6A32060840420F00F7B50F23AD
:1035E0000468816B654A664FB7FBF1F1054689B205
:1035F00090F83500FBF720FE00214388B7FBF3F776
:1036000006462F642046FCF791F9002276212046D9
:10361000FDF7CCFF0F224E212046FDF7C7FF0F20FC
:10362000FFF762FE72794F2102F00F022046FDF78C
:10363000BDFF0F20FFF758FE7279502102F00F02F4
:103640002046FDF7B3FF0F20FFF74EFE5221FF2269
:103650002046FDF7ABFF0F20FFF746FE95F835102B
:10366000072941D0474E96F8F900FBF733FE05468F
:10367000012276212046FDF799FFAA780C212046E9
:10368000FDF794FF2A790D212046FDF78FFFAA79D7
:10369000AB88120142EA1322D2B20E212046FDF776
:1036A00085FF4FF4807196F8F900FBF713FE05468D
:1036B000022276212046FDF779FFAA78520002F017
:1036C000FE0203212046FDF771FF2A7904212046DE
:1036D000FDF76CFFAA79AB88120142EA1322D2B23D
:1036E00005212046FDF762FF002276212046FDF7E6
:1036F0005DFF032214212046FDF758FF0F20FFF73E
:10370000F3FD002263212046FDF750FF6420FFF700
:10371000EBFD082265212046FDF748FF0DF1070269
:1037200064212046FEF738FE9DF8072022F01002A3
:1037300042F06002642120468DF80720FDF736FF35
:103740000F20FFF7D1FD0DF106024D212046FEF7B7
:1037500023FE9DF8062002F03F0242F040024D2178
:1037600020468DF80620FDF721FF0F20FFF7BCFD56
:1037700003212046FCF7DAF803B0F0BDCA32060890
:1037800040420F00E8610020F8B5816B04682D4AC3
:103790002D4FB7FBF1F10546102389B290F83500A3
:1037A000FBF74AFD00214388B7FBF3F706462F6479
:1037B0002046FCF7BBF880226B212046FDF7F6FE81
:1037C0006420FFF791FD072268212046FDF7EEFEF9
:1037D0006420FFF789FD00226B212046FDF7E6FEFD
:1037E0006420FFF781FD01226B212046FDF7DEFEFC
:1037F0000F20FFF779FD18221B212046FDF7D6FE8A
:103800000F20FFF771FD18221C212046FDF7CEFE88
:103810000F20FFF769FD32791A212046FDF7C6FE19
:103820000F20FFF761FD727919212046FDF7BEFEDA
:103830006420FFF759FD20460321BDE8F840FCF75E
:1038400075B800BF6A32060840420F009CE710B509
:103850007822044600210068FDF7A8FE0520FFF746
:1038600043FD202201212068FDF7A0FE0520FFF77F
:103870003BFD002202212068FDF798FE6420FFF73F
:1038800033FD012010BD10B5072204460A2100684F
:10389000FDF78CFE0520FFF727FD2422412120683B
:1038A000FDF784FE0520FFF71FFDC022422120689E
:1038B000FDF77CFE0520FFF717FD012010BD10B5B8
:1038C0000122044610210068FDF770FE48B1142063
:1038D000FFF70AFD2068A022BDE810401121FDF786
:1038E00065BE10BD13B5044600210068FCF71EF844
:1038F0000021204643F0C0FB1420FFF7F5FC0F2108
:10390000204643F0B9FB0A20FFF7EEFC01AA03238F
:103910001021204642F089F90A20FFF7E5FC9DF8C6
:103920000420174B8032A3F800219DF80520803237
:10393000A3F802219DF806208032A3F8042100217B
:10394000204643F099FB0A20FFF7CEFC0DF103025D
:1039500001230221204642F068F901230DF1030200
:103960000921204642F061F92046122143F084FBF0
:1039700020680321FBF7DAFF012002B010BD00BF71
:10398000E07200200023F7B51A4636210120FCF72B
:10399000A5FC154E0446C6F8080140B996F80C314E
:1039A0000C2B02D10123C6F81031254618E005275B
:1039B0009620FFF799FC0DF1070200212046FEF743
:1039C000EBFC054660B9013FF2D196F80C310C2BA7
:1039D00008BF0223204608BFC6F81031FBF779FF65
:1039E000284603B0F0BD00BFE072002008B50068B3
:1039F00001220921FDF7DAFDBDE80840642073E4E7
:103A000080B506460B25013D01D1FDF758FD01218A
:103A10000846FCF7E5FD00210846FCF7E1FD771CB0
:103A20004FF0320805240120FCF7C8FD0020FCF708
:103A3000C5FD0120FDF7EAFC4046FFF755FC0120DB
:103A4000FCF7BCFD0020FCF7B9FD0020FDF7DEFC13
:103A50004046FFF749FC7CB1013C05D14FF4FA70B8
:103A6000FFF742FC4FF0FA0854EA0703DBD14FF4AA
:103A70007A70FFF739FCC6E7013FF5E737B5044632
:103A800000210068FBF752FF15227E212068FDF718
:103A90008DFD6420FFF728FC11227E212068FDF7B0
:103AA00085FD0520FFF720FC20680DF107020321AA
:103AB000FEF772FC9DF8073003F03C03142B02D094
:103AC0000620FFF79DFF0C2240212068244DFDF7C2
:103AD0006DFD0120FFF708FCA16B224A94F8350028
:103AE000B5FBF1F1092389B2FBF7A6FB4388B5FBCF
:103AF000F3F52564027920684221FDF757FD012086
:103B0000FFF7F2FB082241212068FDF74FFD01205D
:103B1000FFF7EAFB002243212068FDF747FD012063
:103B2000FFF7E2FB102251212068FDF73FFD012045
:103B3000FFF7DAFB0A2253212068FDF737FD012049
:103B4000FFF7D2FB802256212068FDF72FFD0120D0
:103B5000FFF7CAFB20680321FBF7E8FE03B030BD86
:103B600040420F0024330608F0B5816B0568514AC6
:103B7000514FB7FBF1F185B00446102389B290F89C
:103B80003500FBF759FB00214388B7FBF3F70646E6
:103B900027642846FBF7CAFE80226B212846FDF7E2
:103BA00005FD9620FFF7A0FB032268212846FDF7BC
:103BB000FDFC9620FFF798FB03226B212846FDF7BA
:103BC000F5FC0F200021FFF7F3FA10226A212846A6
:103BD000FDF7ECFC0F200021FFF7EAFA00226C2130
:103BE0002846FDF7E3FC0F200021FFF7E1FA727988
:103BF00019212846FDF7DAFC0F200021FFF7D8FA3B
:103C000018221B212846FDF7D1FC0F200021FFF7C9
:103C1000CFFA18221C212846FDF7C8FC0F200021EE
:103C2000FFF7C6FA32791A212846FDF7BFFC0120BA
:103C30000021FFF7BDFA03212846FBF777FE206835
:103C4000062302AA4321FDF7ADFED0B1BDF808302E
:103C5000DBBA07EE903ABDF80A30F8EEE77ADBBA45
:103C6000C4ED077A07EE903ABDF80C30F8EEE77A2B
:103C7000DBBAC4ED087A07EE903AF8EEE77AC4EDC5
:103C8000097AD4ED087AFDEEE77ACDED017A9DF957
:103C9000043001330CD1D4ED077AFDEEE77ACDED97
:103CA000017A9DF90430013302D10620FFF7A8FE06
:103CB00005B0F0BD6A32060840420F0018B1036833
:103CC0005B6803B11847FF20704718B103689B6811
:103CD00003B118470020704770B450B106798E4286
:103CE00007D34579954204D30368DB680BB170BCF8
:103CF000184770BC704710B440B184798C4205D32A
:103D000003681B6913B15DF8044B18475DF8044B59
:103D1000704718B103685B6903B11847704718B161
:103D20000368DB6903B118470020704718B10368C6
:103D30001B6A03B118470020704730B560B1041DFD
:103D40000A4600F1140320686168154603C508346B
:103D50009C422A46F7D1012030BD10B50C4670B9FF
:103D60002D23002023750A4B2061C4E90000C4E91B
:103D70000200C4E90633302384F8203010BD036804
:103D8000DB6A002BECD098470028E9D0F6E700BFAB
:103D9000A206070838B5054D441E14F8011F01B9E5
:103DA00038BDD5F83001FBF783FDF6E7E07200205F
:103DB00013B50C4C01900C480091FFF7EBFFDDE9C7
:103DC00000320A49D4F8300146F0D3F8D4F8300173
:103DD000FBF762FD94F8343113B1012384F83531D7
:103DE00002B010BDE0720020A1CE0608D1F8000894
:103DF00008B50648FFF7CEFF054BB3F8360118B1FA
:103E0000BDE80840FFF770BA08BD00BF242B0708C3
:103E1000E072002010B5074C02460B46D4F8300182
:103E2000054946F0A6F8D4F83001FBF735FDBDE8AA
:103E30001040DDE7E0720020D1F8000808B5FFF778
:103E4000A9FFBDE80840D3E710B504460648FFF7D0
:103E5000A1FF2046FFF79EFF044B93F8342112B1D7
:103E6000012283F8352110BDA1CE0608E0720020A2
:103E700010B504460348FFF78DFF2046BDE810400B
:103E8000DCE700BFADCE06080CB4830607B500D54D
:103E900051B9049805A90191FFF7BCFF012003B0B7
:103EA0005DF804EB02B070470020F8E7024B0146D2
:103EB000D3F83001FBF7FCBCE07200200CB407B56E
:103EC00010F0400009D069B92320FFF7EFFF0498F4
:103ED00005A90191FFF79EFF012003B05DF804EBF7
:103EE00002B070470020F8E70FB413B5094C0A4937
:103EF000D4F8300104AB53F8042B019346F039F8A1
:103F0000D4F83001FBF7C8FC02B0BDE8104004B0A3
:103F1000704700BFE0720020D1F800080FB407B569
:103F200004A951F8040B0191FFF774FF03B05DF889
:103F300004EB04B070470FB407B504A951F8040BA3
:103F40000191FFF735FFFFF753FF03B05DF804EB76
:103F500004B0704770B58379164603F007028EB03F
:103F60000446062A50D8DFE802F0041417191C1E74
:103F70004A000D7813F0C00348D0402B3DD12946AC
:103F8000204615F043FE00285BD00EB0BDE870401F
:103F9000AAE791F90050EDE70D88EBE7B1F9005081
:103FA000E8E70D68E6E791ED000A02A8FAF71AFAC9
:103FB00001462948FFF798FFFEB1A37913F0C00F1F
:103FC0001BD1204615F071FD00EE100A02A8B8EED4
:103FD000C00AFAF707FA01462048FFF785FF204696
:103FE00015F074FD00EE100A02A8B8EE400AFAF7C8
:103FF000F9F901461948FFF777FF0EB070BD164872
:104000000EB0BDE870406FE70025B3E7042A0CBF8F
:10401000134814482946FFF767FF002EEDD0A37917
:1040200013F0C00FE9D1204615F03FFD0190204666
:1040300015F04CFD019902460B480EB0BDE87040EA
:1040400052E702A9204615F043FC084802AA294677
:10405000FFF771FFD1E700BFB2D40608C7D6060844
:10406000FECE0608F9050708502C0708B2CE060850
:104070002DE9F04F8FB001F020034D4C00938146A5
:104080000F464FF000084B4BD3F83001FBF704FC10
:1040900094F806B00BF038034B454BD1204615F091
:1040A00091FCFAF7FDFB0646204615F0ADFCD6F86C
:1040B00008A005460AEB0006204615F0E9FC0BF0C7
:1040C0000702062A6BD8DFE802F0043F44484D514E
:1040D0005D001AF805200078111A4A424A41009BF7
:1040E00003B13ABB02A92046019215F0F1FB7B0611
:1040F00015D5019A9AB9304802A9FFF7F5FE2F4964
:1041000002A846F0EDF800284BD11AF80530202B14
:1041100047D12B483146FFF7E7FEFFF769FE2948F4
:1041200002A9FFF7E1FE002231462046FFF712FF09
:10413000FFF75EFE08F10108B8F5197F04F10B04E2
:10414000A1D10FB0BDE8F08F1AF9052090F9000059
:10415000C2E73AF805200088BEE73AF90520B0F931
:104160000000B9E75AF805200068B5E796ED007A37
:10417000D0ED007AB4EE677AF1EE10FA0CBF0122AE
:104180000022ACE70190204615F0A0FC0199421CEA
:1041900030464CF04DFCB0FA80F252099FE7002205
:1041A0009DE7002231462046FFF7D4FEB5E700BF69
:1041B0004A350608E0720020CFCE0608222C0708F8
:1041C000AAD40608D0CE060813B50446019115F00E
:1041D0005FFC019A0146204602B0BDE81040B9E6F6
:1041E000F7B5847914F0C003054603D0402B18D0EE
:1041F00003B0F0BD04F0070415F068FC062C05D1EF
:104200000146164803B0BDE8F04087E60190284615
:1042100015F04BFC019A0146114803B0BDE8F0408F
:104220007CE615F0E3FC05460E480F4E0F4FFFF7F6
:10423000B1FD00242B79A34203D803B0BDE8F040C0
:10424000D6E514B13046FFF7A5FD2B68384653F884
:104250002410FFF749FE0134ECE700BFDACE060870
:10426000EACE060801CF060811CF0608C7D6060811
:1042700008B50548FFF78EFD044BD3F83001BDE8C3
:104280000840FBF709BB00BFADCE0608E072002076
:10429000004850E613CF060813460A460146014877
:1042A00049E600BF1FCF060820B10078B0FA80F0C1
:1042B00040097047012070472DE9F04F87B0034651
:1042C000FFF7F2FF064618B107B0BDE8F04FDFE791
:1042D0004649DFF84091DFF840A1DFF840B105AA78
:1042E00018464BF07BFA34460546B0464FF0FF3790
:1042F0008DB97EB230461FF04FFD10B14568002DDC
:104300005AD1B8F1000F36D139483946F9F707FBD1
:1043100007B0BDE8F08F012E0ED0022E11D01EB9CD
:104320002846FAF74FF90746304905AA00204BF016
:1043300055FA01360546DBE72846FAF743F9804689
:10434000F2E7494628464DF092FB20B92949284614
:104350004DF08DFB08B144F00104514628464DF064
:1043600086FB28B9594628464DF081FB0028DBD052
:1043700044F00204D8E7002C08BF03240023E4B271
:10438000CDE9008402931A46194630461FF0CAFE52
:10439000054610B918483946B8E718484246394624
:1043A000F9F7BDFA39461648F9F7B9FA154B294617
:1043B000D3F8380140F014FE13483946F9F7AFFA44
:1043C0005CB16979A14208D010482246F9F7A7FAF2
:1043D0002B68E1B29B6928469847EB6A002BE1D035
:1043E0000B48F9F79CFA0023EB62DBE75824070837
:1043F0003FCF0608FE0B070867CF060886CF0608E2
:10440000F1CF0608E0720020A3CF0608BBCF060854
:10441000DBCF060834E206083CCF060811EA06089E
:104420002DE9F04F85B00546FFF73EFF044630B159
:104430000021012005B0BDE8F04F40F02BBE8549BA
:104440002846F9F793FC20B905B0BDE8F04F3AF0E3
:10445000BDBB81492846F9F789FC28B9012005B080
:10446000BDE8F04F3AF01EBD7C492846F9F77EFCC6
:10447000034688BB7A4A92F9271E82F8200E10461E
:1044800092F8D254012D08D0033D052D05D9002CFA
:1044900000F0D28080F8271ECEE092F8D354A52DEC
:1044A00003F1010313D101290ED16E4A80F8213E98
:1044B000002380F8201E82F83C3180F8273E05B0AA
:1044C000BDE8F04F3AF03ABD013949B20124782BEA
:1044D00002F11402D4D1DAE72846FAF773F8614BF7
:1044E00093F93C31009303FA80F6772E834600F26D
:1044F000A7802846FBF73AF90746002800F0898094
:10450000FAF760F80124C5B23846FBF72FF90746E1
:10451000002800F08180FAF755F801340190E4B2E8
:104520003846FBF723F98046002877D0FAF74AF897
:1045300001340746E4B24046FBF718F981460028EB
:104540006ED0FAF73FF801340290E4B24846FBF728
:104550000DF98246002865D0FAF734F801340FFAD5
:1045600080F9E4B25046FBF701F9824600285BD09F
:10457000FAF728F801340FFA80F8E4B25046FBF756
:10458000F5F8002852D00390FAF71CF803990FFAB7
:1045900080FA0846FBF7EAF80346002857D004F0F3
:1045A000FD04FAF70FF8042C46D1C3B2012D02D94D
:1045B000E91E052940D81BB1A52B01D0482B3BD1C2
:1045C000274C0EB984F8276E142101FB0646019A88
:1045D000C6F8C024A52B029A86F8D254C6F8C47433
:1045E000C6F8C824A6F8CC94A6F8CE84A6F8D0A421
:1045F00086F8D3340AD100981A4B0130584483F816
:104600003C0194F8273E013384F8273E05B0BDE80D
:10461000F08F0446054677E7019081E707468AE771
:10462000029093E781469DE78046A7E75FFA88F30B
:1046300082468046062CB9D005B0BDE8F04F27E68B
:1046400009487722214605B0BDE8F04F24E6013441
:10465000E4B2EFE71FD0060825D0060824E00608DC
:10466000408D0020E07200202AD0060810B50346D5
:10467000FFF71AFE30B1FCF72BF9BDE810400748F0
:10468000FFF7DCBB1846F9F79DFF044680B2FCF744
:10469000F3F821460248BDE810403FE433D0060855
:1046A0003FD0060808B50346FFF7FEFD40B10C4BAE
:1046B0000C480022A3F83621BDE80840FFF7BEBB36
:1046C0001846F9F77FFF014630B1054BA3F83601D4
:1046D000BDE80840044821E4BDE80840D8E500BF33
:1046E000E072002051D0060867D006082DE9F04F8F
:1046F000DFF8B8A087B0074616460C4615464FF0BF
:10470000000B4FF019094FF46178002E4BD023783D
:1047100028788342EB7844D161786A78914240D11D
:10472000A178AA7891423CD1E178CA1A514251410C
:10473000CDE9041314F0FAF9059B049919FB0383DE
:104740000393AB7819FB038302936B78019343794E
:10475000009352465B463846FFF7B0FB0499207839
:10476000049114F0E3F9E378049919FB03830393AC
:10477000A37819FB03830293637801934379009331
:1047800052465B4638460BF1010BFFF77DFBBBF150
:10479000280F04F1040405F10405B6D107B0BDE803
:1047A000F08F0021C4E73146D9E700BF7ED006086C
:1047B000F7B50746FFF778FD044630B12E490022D1
:1047C000012003B0BDE8F04090E73846F9F7FAFE63
:1047D000272806463DDC8500781C8DF80740FAF74F
:1047E000C5FF074690B1F9F7EDFE031E0EDB234A25
:1047F0002146DBB202F2146404EBC10CC8009CF841
:1048000005C09C452CD001313929F5D13846FAF73D
:10481000ADFF044660B1F9F7D5FE0D2808D8184B56
:104820002B4483F83E019DF8073001338DF80730A3
:10483000114FA91C0DF1070239442046FAF7A3FFD6
:104840009DF80730042B02D0002347F8263003B030
:10485000F0BD0C482722214603B0BDE8F0401BE51F
:10486000074B02442B4492F8182683F83D2101237C
:104870008DF80730CAE700BF1D740020482D0608D8
:10488000E072002094D106082DE9F04F89B0374E30
:10489000DFF8E090069280460C46154602F1300B98
:1048A00094F9041000230C22314F02FB03F0C0578F
:1048B000884255D00133042BF6D10C355D4504F107
:1048C0000C04EDD109B0BDE8F08F95F904302A68E9
:1048D000687995F806C095F808E095F807A0994220
:1048E0003CD12168914239D16179814236D1A17997
:1048F000614533D1217A714530D1E179A1EB0A07C5
:104900007942794156F82A7056F82000049756F8F3
:104910002E70039756F82C700297CDE900204A4676
:1049200040460791FFF7CAFA0799E27994F90430F3
:1049300056F822200492227A56F822200392A27975
:1049400056F822200292627956F8222001922268BB
:10495000009240464A46FFF797FAAEE70021D1E7BA
:10496000069B002BB1D11946DFE700BF002D0608DA
:10497000C074002091D00608F0B585B00346FFF75B
:1049800093FC30B13F490022012005B0BDE8F04062
:104990007AE718465E1CF9F715FE044640B21FF090
:1049A0007BFB054630B93848214605B0BDE8F040EC
:1049B000FFF7C1BA0068696801AB03C3A868186053
:1049C0003046FAF7D3FE044600284BD003782B2B51
:1049D00005D02D2B3BD0F9F7F5FD019009E001340E
:1049E0002046F9F7EFFD019B012202FA00F0034394
:1049F0000193022600272046FAF7B8FE044600B3CA
:104A0000F9F7E0FD214900228C4651F804EB70458E
:104A1000D3B203D00132112AF7D100235CF823204E
:104A200090420ED1022F1FD0032F20D0012F14BF90
:104A30008DF809308DF80A3001370136042FF6B2AF
:104A4000D9D1012E16D805B0BDE8F04020E40134DC
:104A50002046F9F7B7FD019B012202FA00F023EA94
:104A60000003C5E70126C5E78DF80C30E4E78DF8B3
:104A70000B30E1E701AB03CB286018686960A860E0
:104A800005B0F0BDF0740020AED00608002D060879
:104A90002DE9F04FDFF8C0B089B0804617460C46CC
:104AA000154600264FF0190A4FF46179002F51D0B6
:104AB0006979A8780791A1782B786A7895F803C06E
:104AC00095F804E00693814242D1217899423FD182
:104AD000617891423CD1E178614539D121797145C4
:104AE00036D16179079BCB1A59425941069B0691F1
:104AF0001AFB0393CDE901031AFB0292079B039271
:104B00000093CDE904CE33465A464046FFF7D6F926
:104B1000069923790593E378049363781AFB03934A
:104B2000039323781AFB03930293A3780193637989
:104B300000935A46334640460136FFF7A5F9142E36
:104B400004F1060405F10605B0D109B0BDE8F08F07
:104B50000021CBE73946DCE7C1D006082DE9F34751
:104B60008246FFF7A1FB064630B13C4900220120F6
:104B700002B0BDE8F0478BE75046F9F723FD132854
:104B8000054663DC062747430AF101008DF80760FC
:104B9000334CFAF7EBFD04F5117909EB07080646EB
:104BA00048B1F9F70FFD03289FBFE31983F84902C5
:104BB00001238DF807303046FAF7D8FD064668B174
:104BC000F9F700FD0D2809D8062303FB054383F8F8
:104BD00046029DF8073001338DF807300DF10702CA
:104BE00041463046FAF7CFFDFAF7C0FD064668B1F8
:104BF000F9F7E8FC3B2809D89DF80730062202FBAC
:104C00000542013382F847028DF807303046FAF743
:104C1000ADFD68B1F9F7D6FC0D2809D89DF807302D
:104C2000062202FB0544013384F848028DF8073060
:104C30009DF80730062B06D0002349F80730A8F866
:104C40000430FFF725FB02B0BDE8F08705481322CA
:104C5000314602B0BDE8F047FFF71EBB24750020C7
:104C6000E072002094D106082DE9F04F2DED088B5D
:104C7000DFF814A197B0074690460C46154600266B
:104C800094ED008AB5EE408AF1EE10FA73D0D4EDBF
:104C9000019A94ED029AD4ED038AB8F1000F40D046
:104CA00095ED000A95ED01BAD5ED02AA95ED03AA9E
:104CB000B4EE408AF1EE10FA62D1F4EE4B9AF1EEC6
:104CC00010FA5DD1B4EE6A9AF1EE10FA58D1F4EE12
:104CD0004A8AF1EE10FA0CBF4FF001094FF00009BB
:104CE00012A8F9F77FFBB0EE4B0A83460EA8F9F73E
:104CF00079FBB0EE6A0A05900AA8F9F773FBB0EEEB
:104D00004A0A049006A8F9F76DFB059B049A0390E4
:104D1000CDE900B302923346524649463846FFF782
:104D2000CDF8B0EE480A12A8F9F75CFBB0EE690ABC
:104D300081460EA8F9F756FBB0EE490A83460AA849
:104D4000F9F750FBB0EE680A049006A8F9F74AFBA1
:104D5000049B0390CDE901B3CDF800903346524651
:104D6000002138460136FFF78FF80C2E04F11004AD
:104D700005F1100584D117B0BDEC088BBDE8F08FAC
:104D80004FF00009ACE700BFDFD00608F8B50546D4
:104D9000FFF78AFA064668B1414991F84E344FF45C
:104DA000C87202FB0311BDE8F840002201F533711F
:104DB000012059E73B4905222846F8F7BBFF78B99F
:104DC000374A02F52F7392F84E244FF4C87101FB55
:104DD0000233002201300C2843F8102FFAD1F8BD1D
:104DE0002846F9F7EFFB0B28044652D82846FAF775
:104DF000BDFC0646C0B3F9F759FB294B93F84E2486
:104E0000192101FB024203EB021383EDB30A0125D2
:104E10003046FAF7ABFC064660B1F9F747FB204B8A
:104E200093F84E24192101FB024203EB021383ED98
:104E3000B40A01353046FAF799FC064660B1F9F735
:104E400035FB174B93F84E24192101FB024203EB6B
:104E5000021383EDB50A01353046FAF787FC28B90D
:104E6000BDE8F840FFF714BA0546D1E70C4E96F8B6
:104E70004E74F9F71BFB192000FB074406EB0414E2
:104E8000032D84EDB60AEBD14FF4C87101FB076125
:104E900089E731460448BDE8F8400B22FFF7FCB92A
:104EA000E07200201FD0060894D106082DE9F043D7
:104EB000DFF8649085B080460D4616460227002430
:104EC00046B336F8242035F82430F05B93421FD1E6
:104ED000EB5B191A4B424B411946CDE900202346A2
:104EE0004A4640460391FEF7E9FF0399EB5B0193C5
:104EF00035F8243000934A46234640460134FEF7F5
:104F0000C3FF042C07F10407DAD105B0BDE8F08334
:104F10000023E1E73146E9E7F3D00608F8B5044697
:104F2000FFF7C2F9054628B1BDE8F840294900223B
:104F30000120BBE728492046F8F718FFA8B9274BFE
:104F40004FF47A714FF4FA62A3F87414A3F876243C
:104F5000A3F87814A3F87A24A3F87C14A3F87E2489
:104F6000A3F88014A3F88224F8BD2046F9F72AFBA1
:104F70000328074627D82046FAF7F8FB044670B105
:104F8000F9F720FB012506462046FAF7EFFB10B1A2
:104F9000F9F718FB2DB9BDE8F840FFF779B90546D8
:104FA000F2E7A6F2EE2240F2DC539A42F3D8A0F2E6
:104FB000EE229A42EFD8094B03EB8703A3F87464FF
:104FC000A3F87604D0E729460548BDE8F840032257
:104FD000FFF762B9547700201FD00608E072002066
:104FE00004D106082DE9F04FDFF800A191B0834607
:104FF00091460C461546002604F115080422414648
:1050000009A84CF011FD00238DF82830D4E90232B4
:10501000082B72F100010BAF56D230491A463846C0
:10502000F8F79AFCB9F1000F55D02B780793079A3F
:10503000237893424DD1D4E90202D5E902139A4272
:1050400008BF884245D1227D2B7D9A4241D104225E
:1050500005F1150140464CF091FC002839D1216939
:105060002B69CB1A594259411D4B059300230493D8
:10507000B5F912300393B5F910300293194B01932F
:10508000079B00935246334658460791FEF716FF9A
:10509000079909AB0593237D0493B4F91230039368
:1050A000B4F91030CDE9017314F8203B0093524657
:1050B000334658460136FEF7E7FE082E05F1200577
:1050C0009AD111B0BDE8F08F07493846F8F744FC93
:1050D000A8E70021C8E74946DBE700BFF905070854
:1050E000F5EE06082E1007080CD1060817D10608A1
:1050F0002DE9F74F0446FFF7D7F8074630B172495C
:105100000022012003B0BDE8F04F6BE76F49204655
:10511000F8F72CFE014638B96B484FF4807203B0A3
:10512000BDE8F04F4BF0EABC2046F9F74BFA83B2EA
:10513000072B054600F2C0802046FAF717FB82468F
:1051400000284CD0F9F73EFA01240FFA80F95046B6
:10515000FAF70CFB68B14FF00008411E00F1100C8B
:10516000464611F8013F13F0DF0F3BD10127013410
:10517000E4B2FAF7FBFA824600284CD0F9F722FA9B
:1051800001340FFA80FBE4B25046FAF7EFFA034617
:10519000002842D00190F9F715FA0134019B0FFA6B
:1051A00080FAE4B21846FAF7E1FA0346002836D04E
:1051B0000190F9F707FA0134019B42B2E4B21846B4
:1051C0000192FAF7D3FA019A034650B30134E4B2DC
:1051D000032C28D803B0BDE8F04FFFF759B80446B8
:1051E0008146B4E76145C2D0A3F13002D2B2092AA8
:1051F00005D9A3F16102052A07D8573BDAB2360177
:1052000046EA187642EA0818ABE7A3F14102052AFC
:10521000ADD8373BF2E78346B6E78246C2E702469F
:10522000CDE72B4BD4E71FFA89F10229D2D80BF234
:10523000262189B2B1F5E16FCCD80AF2262189B2D4
:10524000B1F5E16FC6D8D4B2062CC3D81846019385
:1052500045F050F80428BDD8002FBBD01D4A019B53
:105260002DB202F5926002EB45114FEA451C00EBAE
:10527000451702EB4512184D40F80C8081F88894D0
:10528000A1F898B4A1F89AA481F89C447E60591EB4
:1052900002F29D42033311F8010F445D04F0030450
:1052A000022C08BF203802F8010B087808B18B42A5
:1052B000F1D103B0BDE8F08F08480722394603B0AA
:1052C000BDE8F04FFEF7E8BF687700201FD0060862
:1052D000F5EE0608E07200206131070838D10608B3
:1052E0002DE9F04FDFF8A89089B0804617460C46AC
:1052F00015460026002F49D0687A627AB5F90AC0AF
:10530000B5F90CE095F808A08242D5E900B33BD18D
:1053100022685A4538D162689A4235D1B4F90A20D8
:10532000624531D1B4F90C2072452DD1217AA1EB1F
:105330000A0251425141CDE9020CCDE900B3CDE959
:1053400004EA33464A4640460791FEF7B7FD0799FF
:10535000237A0593B4F90C300493B4F90A3003931B
:10536000637A02936368019354F8103B00934A46B2
:10537000334640460136FEF787FD112E05F1100534
:10538000B8D109B0BDE8F08F0021D4E73946DFE796
:1053900045D106082DE9F74F0446FEF785FF05467F
:1053A00030B14F490022012003B0BDE8F04F97E72C
:1053B0004C492046F8F7DAFC30B94FF0FF3003B023
:1053C000BDE8F04F3BF010BC2046F9F7FBF8C3B244
:1053D000102B834607D944481022294603B0BDE864
:1053E000F04FFEF759BF2046FAF7C0F90646E8B17C
:1053F000F9F7E8F8012482463046FAF7B7F906468D
:10540000B8B1F9F7DFF801348146E4B23046FAF773
:10541000ADF9064600285CD0F9F7D4F8012880469B
:1054200009D903B0BDE8F04FFEF732BF044682460B
:10543000E2E78146EAE70134E4B23046FAF796F94A
:105440000646002847D0F9F7BDF800F5B473B3F568
:10545000347F0746E5D80134E4B23046FAF786F9DE
:105460000346002839D00190F9F7ACF800F5B47282
:10547000B2F5347F0646D4D80134019BE4B2184615
:10548000FAF774F9034640B10190F9F79BF801343B
:10549000051E019B18BF0125E4B21846FAF766F90C
:1054A00008B10134E4B2062CBBD1104B4FFA8BFB90
:1054B00003EB0B13C3F888A5C3F88C9583F891858B
:1054C000A3F89275A3F8946583F8905503B0BDE8EE
:1054D000F08F8046B1E70746BFE70646CFE700BF3B
:1054E000687800201FD0060865D10608E072002009
:1054F0002DE9F047DFF874A086B0814690460D464E
:1055000017460026B8F1000F2ED03B782A789A4231
:10551000D7E9010C26D16A68824223D1AC68A4EB9A
:105520000C0254425441CDE9010C214600935246ED
:10553000334648460594FEF7C1FC0599AB680293D3
:105540006B68019315F80C3B00935246334648466E
:105550000136FEF799FC082E07F10C07D2D106B0F0
:10556000BDE8F0870024DEE74146E7E776D106088C
:105570002DE9F8430446FEF797FE054628B1BDE83D
:10558000F8432E4900220120B2E72D492046F8F7C2
:10559000EDFB014628B9BDE8F843284860224BF0EE
:1055A000ADBA2046F9F70EF8C3B2072B064606D966
:1055B00029462448BDE8F8430722FEF76DBE204681
:1055C000FAF7D4F8074628B3F8F7FCFF051E18BF12
:1055D000012501243846FAF7C9F80746E0B1F8F783
:1055E000F1FF01348046E4B23846FAF7BFF80746C7
:1055F000A0B1F8F7E7FF01348146E4B23846FAF784
:10560000B5F808B10134E4B2032C09D0BDE8F84381
:10561000FEF73EBE0446DDE78046E5E78146EDE75E
:10562000094B76B20C2000FB063686F89856C6F871
:105630009C86C6F8A096BDE8F88300BF7879002064
:105640001FD006088BD10608E07200202DE9F04F2C
:10565000DFF8849091B007468846164600240DF185
:105660002C0A04EB840508EB050358F805001B79A8
:105670000290514602A88DF80C303FF05FFC4EB30B
:10568000731970591B790490052204A902A88DF89A
:1056900014304CF073F90DF1180BB0FA80F559463F
:1056A00004A86D093FF04AFCCDF800B023464A46F5
:1056B00029463846FEF702FC2346CDF800A04A46AC
:1056C000294638460134FEF7DFFB802CC9D111B0E2
:1056D000BDE8F08F3546EFE79AD106082DE9F04F87
:1056E00089B00546FEF7E0FD044630B16849002266
:1056F000012009B0BDE8F04FA8E72846F8F762FF9F
:105700007F28074600F3BB802846FAF72FF8604A47
:105710000194BB00039307EB8703D118D4505D4B72
:105720000C71064602932546A246A346A046A14612
:10573000029B05AA13F801CB02939646002330463C
:1057400016F8011B19B18C4501D00A2B0CD120335E
:105750006B444FF000068C4503F80C6C08D009B080
:10576000BDE8F04FFEF794BD0EF8011B0133E6E7EC
:1057700009F1FF33461C032B03D8DFE803F02E4565
:105780006E7705A8F8F71EFF019009F101095FFA8D
:1057900089F9B9F1050FCBD1039A3F4B01993A44EE
:1057A00017469A1803F5DF631F4405F00F0004F055
:1057B0000F0444EA081440EA01104FEA281882F85E
:1057C000F80682F8F9B682F8FAA6FC7087F8048029
:1057D00009B0BDE8F04F2CF0D5BE05A8F8F7F2FEF1
:1057E0000546D2E74E2B14D0452B14D0532B14D0A2
:1057F000572B14D0552B14D0442B05D10523012150
:1058000001FA03F348EA030812F8013B002BE9D13F
:10581000BBE70023F3E70123F1E70223EFE70323CC
:10582000EDE70423EBE7DFF878C0002319461CF806
:10583000013B834204D0072901F10103F6D1594607
:10584000DFF860C000231CF801EB70450AD101208D
:1058500000FA03F34AEA030A8B4612F8010B002808
:10586000E1D192E70133072BEDD1F5E705A8F8F771
:10587000A9FE10280446B4BF0446002485E7074863
:105880007F22214609B0BDE8F04FFEF705BD00BFFD
:10589000D879002024350608E072002094D106084B
:1058A00029350608313506082DE9F047DFF870A0E4
:1058B00086B0814690460D4616460027B8F1000F87
:1058C0002BD033882A889A4225D16C887188621A35
:1058D00054425441F2780292B2780594CDE90032F4
:1058E00021463B4652464846FEF7E8FA0599EB78D2
:1058F0000293AB78019335F8043B009352463B4644
:1059000048460137FEF7C0FA102F06F10406D5D13C
:1059100006B0BDE8F0870024DCE74146E7E700BFBA
:10592000A4D106082DE9F8430546FEF7BDFC044660
:1059300028B1BDE8F843254900220120B4E72846F4
:10594000F8F740FE0F28064630DC2846F9F70EFF30
:10595000A0361F4FDFF8848005464FEA86092846A7
:10596000F8F730FE37F8023B984226DC012C08EBB2
:10597000090311D0022C12D0A3F8F80628462C21D6
:105980004CF01BF8054668B1013501230134A3B181
:10599000032CE4D1BDE8F88383F8FA06EEE783F838
:1059A000FB06EBE7A21E53425341EFE721460948AD
:1059B000BDE8F8430F22FEF76FBC074B002243F807
:1059C0002620BDE8F843FEF763BC00BF587C0020EA
:1059D0003835060894D10608D8790020E0720020F6
:1059E0002DE9F04F14462C4A85B00646894600271B
:1059F0004FF0060B0BFB07F505F530754FF000086F
:105A000019F805A0002C43D0635DAAEB03004142C6
:105A10004141CDE9008330463B460391FEF74EFA03
:105A200003991D4ACDE9008A3B46304608F101083A
:105A3000FEF72AFAB8F1060F174A05F10105DFD182
:105A40000137062FD6D1144F4FF4397519F805A038
:105A5000A5F53978F4B1635DAAEB030251425141D7
:105A6000CDE900833A46062330460391FEF726FA35
:105A700003990623CDE9008A3A463046FEF704FA38
:105A8000013540F2ED239D42E0D105B0BDE8F08F35
:105A90002146C7E72146ECE7B6D1060870B586B0C7
:105AA0000346FEF701FC044630B11A4900220120EA
:105AB00006B0BDE8704093E71749174E02AA184692
:105AC00049F08CFE03AD80B1032C03D1FEF7E0FB5F
:105AD00006B070BDF8F776FD02AA45F8040B314612
:105AE0000020013449F07AFEEDE7032CEED1DDE928
:105AF0000345059B01931A462946E0B22CF0A0FE0F
:105B00000028E3D0019B05482A462146FEF706FA05
:105B1000DEE700BFD879002058240708B6D1060870
:105B20002DE9F043DFF8989087B0804617460C4681
:105B300015460026002F41D0B5F90030B4F9001009
:105B4000B5F90220B5F9040095F906C0994233D1A0
:105B5000B4F9021091422FD1B4F9041081422BD133
:105B600094F90610A1EB0C0EDEF1000141EB0E01E1
:105B7000CDE90032CDE9020C33464A464046059154
:105B8000FEF79CF9059994F906300393B4F90430B3
:105B90000293B4F90230019334F9083B00934A466A
:105BA000334640460136FEF76FF9102E05F1080521
:105BB000C0D107B0BDE8F0830021D9E73946E2E75C
:105BC000CAD106087FB50546FEF76EFB00285ED0F9
:105BD00030490022012004B0BDE87040A0E72D2B21
:105BE00003D0A3F13002092A4CD8042C04DD04B000
:105BF000BDE87040FEF74CBB2846F8F7E3FC04AB69
:105C0000621C03EB440424F80C0C15F8013F303BF4
:105C1000092BFAD914462B78002BE0D1052CE6D1BC
:105C2000BDF80430BDF904600F2BE0D8BDF90610B3
:105C3000A1F5FA7292B2B2F5FA6FD8D8BDF9082080
:105C4000A2F5FA7080B2B0F5FA6FD0D8BDF90A00AB
:105C50008142CCDC8242CADB9142C8DCBDF90C50E7
:105C600005F17D04A4B2FA2CC1D80B4B03EBC6039B
:105C7000A3F8E619A3F8E829A3F8EA0983F8EC5990
:105C800004B070BD202BB2D101352246C2E70446D4
:105C9000C1E700BFC67C0020E07200202DE9F04F74
:105CA000DFF8B8B08FB0804617460C461546002680
:105CB000A388ADF82C3023780893B4F90290637868
:105CC00020680693237994F905A00A900793B9F107
:105CD000000F3CD0002F3FD02868BDF828100C9052
:105CE00080B2AB88ADF8343081422A7895F801C093
:105CF000B5F9023095F804E02CD14B452AD1BDF816
:105D00002C10BDF83400081A41424141CDE901C3CD
:105D10000092CDE903EA33465A4640460991FEF720
:105D2000CDF80999079BCDF810A0CDE90293069B09
:105D30000193089B00935A46334640460136FEF7CE
:105D4000A3F8202E04F1060405F10605B0D10FB02A
:105D5000BDE8F08F0021D9E73946E3E7DFD1060837
:105D6000F0B589B0044644F0C5FA10F0FF020DD139
:105D70003C4991F84E344FF4C87000FB031101F513
:105D80006371012009B0BDE8F04087E7364905227C
:105D90002046F7F7CFFFB0B9324B93F84E244FF4BB
:105DA000C87101FB0233314A1568948803F56373A7
:105DB000062606FB00F29918013020289D508C80A1
:105DC000F7D109B0F0BD20462949294E01AA49F072
:105DD00005FD4FF0FF33079302AD002478B1062C88
:105DE00002D1FEF755FAECE7F8F7ECFB01AA45F80B
:105DF000040B31460020013449F0F0FCEEE7042C9E
:105E0000EFDD029F1F2FECD8039E0F2EE9D8049DD3
:105E1000262DE6D8059C04F57A73B3F5FA6FE0D821
:105E20000698FF28DDD807994B1C402BD9D80D4B7D
:105E300093F84E244FF4C87C0CFB02F24FF0060C92
:105E40000CFB0722134483F8900383F88C63094802
:105E500083F88D53A3F88E4383F89113FFF780FFE7
:105E6000AFE700BFE07200201FD006083E350608ED
:105E700058240708F5EE06082DE9F04F9BB0DFF82F
:105E800014A10E93074693460C46154600260E9B1A
:105E90005A1C01D0B3426FD1A646BEE80F000DF1E7
:105EA000400CACE80F00DEF80030CCF80030237B6B
:105EB0000A93237C0B9394F911300C93A37C94F8F0
:105EC000048094F81390089009920D93BBF1000F91
:105ED0005ED0AE46BEE80F000DF1540CACE80F00EA
:105EE000DEF80030149ACCF8003022F07F4223F024
:105EF0007F439A420F9095F804E0A86895F80CC08B
:105F0000E97C43D1F04541D1089B0F9A93423DD1A2
:105F10000A9B63453AD1099B834237D1A9EB010320
:105F200059425941099B06930A9B0593089BCDF85A
:105F30001C90CDE903830D9B02930C9B01930B9B5B
:105F400000935246334638460F91FDF7B7FF0F993D
:105F5000099B06930A9B0593089BCDF81C90CDE9FD
:105F600003830D9B02930C9B01930B9B0093524662
:105F700033463846FDF788FF0136402E04F11404FD
:105F800005F1140583D11BB0BDE8F08F0021C9E7EE
:105F90005946DDE7F6D10608034B9A780021101A1E
:105FA000997018BF012070472C77002010B5114B55
:105FB000014603F1180253F8044B41F8044B934295
:105FC000F9D11B880B800B4900F11A0351F8044BDF
:105FD00043F8044B9142F9D111881980054B3430B4
:105FE00053F8041B40F8041B9342F9D11B8803802B
:105FF00010BD00BF9C4F0608104A117A537A0B431C
:10600000D17C0B4351780B4391780B43D1780B43F0
:1060100011790B43917B0B43917E0B4392F8231034
:106020000B4392F82F100B4305D192F83D00013835
:1060300018BF012070470120704700BF08CF002023
:1060400070B5244C94F84C3005460E4643B1D4E963
:106050001423904271EB030324BF002384F84C30D7
:10606000E36E1D48984710F0010321D080F0020331
:10607000C3F3400384F84C30D4E918315B1946EB84
:106080000106C4E91436012384F880304307D4F8AC
:10609000880048BF0123A5EB000548BF84F8813084
:1060A000002D0EDD012084F8800000F0010070BD9D
:1060B0008207EBD594F84C20002AE7D084F84C30C6
:1060C000E4E794F8803013B994F88100EDE70120FB
:1060D000EBE700BF08CF002060CF00202DE9F041A2
:1060E0008AB004460D4644F005F910F0FF0210D1C5
:1060F0003F4B197849B94FF0FF330A463D4901201B
:106100000AB0BDE8F041FFF7B7BE6B1C6CD02B4660
:10611000F4E7394905222046F7F70CFE38B935482F
:106120004FF47E710AB0BDE8F04142F011BE204646
:106130003249324E6A4649F051FB01AD002478B134
:10614000092C02D1FEF7A4F84EE0F8F73BFA6A46B4
:1061500045F8040B31460020013449F03FFBEEE7DF
:10616000092CEFD101993F29ECD8DDF808E0BEF108
:10617000010FE7D8DDF80CC00CF10103402BE1D88A
:10618000049F342FDED8059E072EDBD8069D1C4ABF
:1061900005F5742303F510739342D3D8079C072C9D
:1061A000D0D8089800F5742303F510739342C9D82A
:1061B000099AFF2AC6D8134B4FF0140808FB013385
:1061C00009B2C3F8980083F8A0E00F4883F8A1C093
:1061D00083F8A27083F89460C3F8905083F89C40D1
:1061E00083F8A320FFF77AFF0AB0BDE8F08100BF73
:1061F0001474002098CF00201FD0060858240708E8
:1062000080841E0008CF0020F5EE06084FF0FF3115
:1062100064E737B505460846019144F06BF80199EB
:10622000044602462846F7F785FD68B92B5DA3F1C1
:106230003002092A06D923F02003413B192B01D94A
:106240000134281903B030BD0020FBE72DE9F04FE1
:10625000164615461C4A87B007460C464FF0000B01
:10626000D4E9009AD4F8088066B3AB689845D5E9BC
:10627000000125D1814523D1AAEB0103594259419F
:10628000CDE9019ACDF800805B4638460591FDF7CF
:1062900015FE05990C4ACDF800805B46CDE9019AC0
:1062A00038460BF1010BFDF7EFFDBBF1080F064A75
:1062B00004F10C0405F10C05D2D107B0BDE8F08F54
:1062C0000021DDE73146E6E730D4060870B586B038
:1062D000044644F00FF810F0FF0205D121490120D7
:1062E00006B0BDE87040B1E71F4905222046F7F728
:1062F00021FD38B91B4840F2FF3106B0BDE87040BF
:1063000042F026BD20461949184E01AA49F066FA06
:1063100002AD002478B1042C02D1FDF7B9FF1FE0D3
:10632000F8F750F901AA45F8040B31460020013472
:1063300049F054FAEEE7042CEFD1029A072AECD880
:106340000B4B0C480C2101FB0233039AC3F8982530
:10635000049AC3F89025059AC3F89425FFF7B6FF71
:1063600006B070BD98D400201FD006085824070836
:1063700008CF0020F5EE06082DE9F04FDFF808B150
:10638000A1B0804617460C4615460026A646BEE834
:106390000F000DF1480CACE80F0023680C93237933
:1063A0000A93A3680B939EE80700238A0D93638AE0
:1063B0000E93A38A0F93E38A94F80C9094F818A094
:1063C00010938CE80700002F5CD0AE46BEE80F00AB
:1063D0000DF1640CACE80F009EE807002B7E5345DE
:1063E0008CE807004CD12B790A9A934248D12B684C
:1063F0000C9A9A4244D12B7B4B4541D1AB680B9A06
:106400009A423DD1169A82423AD117991E9BCB1AD5
:1064100059425941109B08930F9B07930E9B06937B
:106420000D9B05930B9B1191CDE903930C9B02935C
:106430000A9B5A46CDE900A340463346FDF73EFD90
:106440001199109B08930F9B07930E9B06930D9B2E
:1064500005930B9BCDE903930C9B02930A9B5A4631
:10646000CDE900A3404633460136FDF70DFD042E6D
:1064700004F11C0405F11C0588D121B0BDE8F08FA2
:106480000021C7E73946DCE741D406082DE9F0438F
:106490008DB0044643F02EFF10F0FF0205D13E49B7
:1064A00001200DB0BDE8F04366E73C4905222046D7
:1064B000F7F740FC38B938484FF47E710DB0BDE8AD
:1064C000F04342F045BC20463549354E01AA49F01B
:1064D00085F902AD002478B10A2C02D1FDF7D8FE6F
:1064E00057E0F8F76FF801AA45F8040B3146002091
:1064F000013449F073F9EEE70A2CEFD1DDF808809A
:10650000B8F1030FEAD8DDF80CE0BEF1010FE5D8D1
:10651000DDF810C0BCF1070FE0D8059F214B07F54F
:10652000742202F510729A42D8D8069E072ED5D84A
:10653000079D05F5742202F510729A42CED8089C88
:10654000B4F5004FCAD20998B0F5004FC6D20A99E7
:10655000B1F5004FC2D20B9AB2F5004FBED2124B2A
:106560004FF01C0909FB0833A3F8020683F808E67C
:106570000E4883F8F4C5C3F8F07583F8FC65C3F8DA
:10658000F855A3F80046A3F80416A3F80626FFF76B
:106590007DFF0DB0BDE8F083F8D400201FD00608C1
:1065A0005824070880841E0008CF0020F5EE060856
:1065B0002DE9F04FDFF864A0DFF864B085B006463F
:1065C000894615461F460024002F01DBA7421CD137
:1065D00019F80480FDB12B5DA8EB03020AEB8303DD
:1065E0005142DB690093514123465A46304603919C
:1065F000FDF764FC03990AEB88085A46D8F81C306A
:10660000009330462346FDF73FFC01340E2CDBD1CE
:1066100005B0BDE8F08F2946EDE700BF9C4F0608A6
:1066200063D406082DE9F04FA1B0DFF848810D9141
:1066300006461546002414AF0D9A02EB441263017E
:106640000DF1400E02F1200910685168F446ACE8E3
:10665000030008324A45E646F6D1002D00F0888056
:106660002B440DF1600C03F1200E18685968624646
:1066700003C2083373459446F7D19DF840300A931E
:106680009DF860100A98BDF842300B9381429DF846
:1066900044300C93BDF846909DF848A0BDF84AB030
:1066A0009DF84C30BDF84E2060D1BDF862100B98BB
:1066B00081425BD19DF864100C98814256D1BDF89F
:1066C0006610494552D19DF8681051454ED1BDF82C
:1066D0006A1059454AD19DF86C10994246D1BDF8CF
:1066E0006E10914242D11CA93846CDE90E3243F0DA
:1066F000F7FDDDE90E32B0FA80F14909CDE905B3C5
:106700000C9B02930B9B01930A9B0093CDE90727F7
:10671000CDE9039A2346424630460A91FDF7CEFB67
:106720000A99BDF84E3007939DF84C300693BDF89A
:106730004A3005939DF848300493BDF846300393E2
:106740009DF844300293BDF8423001939DF84030EB
:10675000009308972346424630460134FDF794FBE8
:10676000032C7FF469AF21B0BDE8F08F0021C5E7AD
:106770002946D6E77BD406082DE9F04190B00446BF
:1067800043F0B8FD10F0FF0205D14549012010B0DB
:10679000BDE8F04146E74349434F01AA204649F08E
:1067A0001DF841496A4649F019F806AE00243546FD
:1067B00000286ED0092C61D13A4901AA002049F085
:1067C0000DF80646002869D043F094FD0F280446D2
:1067D00028BF0F2420B12246314602A847F0F0FF1F
:1067E00004F14003DDF818800DEB0304B8F1020F4B
:1067F0004FF0000304F8383C4DD8DDF81CE0BEF142
:10680000070F48D8DDF820C0BCF1FF0F43D8099F1F
:10681000072F40D80A9EFF2E3DD80B9C072C3AD854
:106820000C98FF2837D80D99022934D80E9AFF2AE0
:1068300031D81E4B03EB481303F5CE6303F8084C25
:1068400003F810EC23F80ECC03F80C7C23F80A6C48
:1068500023F8060C03F8041C23F8022C02AC224691
:1068600003CAAA4218605960144603F10803F6D11E
:106870000F48FFF781FF10B0BDE8F081F7F7A2FEE7
:106880006A4646F8040B39460020013448F0A6FF5A
:106890008EE7092C90D0FDF7FBFCECE704469FE760
:1068A00068D500200AF006085824070808CF002001
:1068B000F5EE0608F8B50C4C0C4E0D4F332520684C
:1068C000FDF768FA616811B13046FDF70DFBA1686C
:1068D00011B13846FDF708FBFDF78AFA013D04F1D6
:1068E0001004ECD1F8BD00BFC84F060883F00608BD
:1068F000AFD4060830B5274885B0FDF74BFAF4F75A
:1069000003FF28B9244805B0BDE83040FDF796BA2A
:10691000F5F7FEF908B92148F5E7F5F703FA02683B
:10692000037D81790446407C0290207C0190608A3E
:10693000009052081A48FDF7D7FAE51D0C3415F8F7
:10694000010BFDF7B3FAA542F9D1164C1648FDF735
:1069500021FA6378022B06D007D9032B10D11348F4
:10696000FDF718FA0CE01248FAE704F580541148D4
:10697000FDF710FA94F8B431022B06D0032B06D0A1
:1069800005B0BDE83040FDF733BA0B48E8E70B48E7
:10699000E6E700BFB5D40608BFD40608CDD4060884
:1069A000DCD40608C44F00200AD506081AD506080C
:1069B00020D506082DD5060833D506084CD506087F
:1069C0002DE9F3473649DFF8D89001AA48F006FFD1
:1069D0004FF0000A4FF0FF3557465446D0462E463A
:1069E00068B9BAF1040F50D03ADCBAF1020F13DCE7
:1069F0002C492B46324601203EF0D6FB0EE0BAF180
:106A0000040F09D8DFE80AF0030D12171C00F7F78E
:106A1000D9FD064603281BD9FDF73AFC02B0BDE8B4
:106A2000F087F7F7CFFD05469528F4E7F7F7CAFD9D
:106A300080463F28EFE7F7F7C5FD04463F28EAE721
:106A40000378482B03D0562BE6D1012700E000271E
:106A500001AA494600200AF1010A48F0BFFEBFE73B
:106A6000BAF1050FD8D1962303FB0655A4010E4EAB
:106A700004F47C6408F03F0844EA080406EB45058A
:106A800044EA4734A5F8C046C8E7962303FB0652FC
:106A9000054B03EB4203B3F8C076C7F34037E2E798
:106AA00058240708C8D5002008CF00202DE9F0435E
:106AB00085B003AA2549264E264FDFF8A08048F06E
:106AC0008DFE0024024625464FF0FF3942B9012DC4
:106AD00035DD022D07D120494B4601F8094030E051
:106AE00035B1012D12D0FDF7D3FB05B0BDE8F08321
:106AF0001046F7F767FD0D288146F4D803AA13491D
:106B0000002048F06BFE01350246DFE711463046B3
:106B10000192F7F72BF9019A04460028EED01146AE
:106B20003846F7F723F9019A38B111464046F7F78E
:106B30001DF90028D7D10224E0E72C46DEE70649FC
:106B40004B460120FFF734FDCFE700BF582407086C
:106B50005ED5060866EE0608686F0020D0180708A4
:106B60002DE9F04F2DED028B4D484E4D9FED4E8A95
:106B70008BB0FDF7D3F90027B946BA464B4B4C4AC8
:106B8000196800238B4227DB01371A2F05F14805CE
:106B9000F4D14849484BD1E90021520942EAC16287
:106BA0004649186809684FF47A73B0FBF3F3444818
:106BB000FDF7B4F90A2299FBF2F302FB139000905F
:106BC0009AFBF2F13F4802FB11A2FDF7A7F90BB0C7
:106BD000BDEC028BBDE8F08F52F8040BA84201D047
:106BE0000133CFE7AC6A4CB107EE904AB8EEE77AD2
:106BF000C8EE077AFDEEE77A17EE904AD5E90C6108
:106C0000AB6B08934A09EB6B0992089A4FEAE47B55
:106C100063437609A4FB020C46EAC16602FB0B3112
:106C200041F28833C01841EB0C014FF47A72002313
:106C300044F078FA099A04FB02F1804606FB0B1B2C
:106C400041F28833A4FB0601C0184BEB01014FF45D
:106C50007A72002344F066FA042F2B6C01964FF4ED
:106C60007A72B3FBF2F306934FF00A0318BF814424
:106C700090FBF3F203FB1200CDE9042098FBF3F242
:106C800003FB1283CDE90223089B00932A680E4878
:106C90002346394618BFC244FDF740F974E700BFE8
:106CA00063D50608E808002000247449F85501203F
:106CB00058550120C4550120CC550120D455012040
:106CC000DFD5060801D60608AAD506081FB5094B68
:106CD0000293094B0193094B0093094A094B0A4956
:106CE0000A48FDF71BF90A490A4805B05DF804EBAC
:106CF000FDF714B9CFCA0608D8CA0608E1CA0608C3
:106D00002CCA0608EDCA06083FCA06082FD6060890
:106D100047D6060861D60608F8B50C480C4D0D4E4E
:106D20000D4FFDF7FBF800246CB93268C2F5007214
:106D3000920022B157F824100848FDF7EFF801340B
:106D4000222CF1D1F8BD55F82420F2E76AD60608C6
:106D5000703D00206C350020F852060880D60608E9
:106D60002DE9F84F054643F0C5FADFF8EC800446FC
:106D7000D8F80090C0B93048304D314FFDF70AF8CF
:106D8000012655F8041B59B10B783BB106FA04F300
:106D900013EA090F02D03846FDF7A6F80134F0E7F0
:106DA000BDE8F84FFDF724B8024626492846F6F715
:106DB000C1FF78B92448214C214DFCF7EBFF54F872
:106DC000041B0029ECD00B78002BF8D02846FDF7E7
:106DD0008BF8F4E72B78DFF864B02D2B03BF013577
:106DE00004F1FF344FF0010A4FF0000A00265BF86F
:106DF000047B1FB9BDE8F84F3EF036B9224639464C
:106E00002846F6F797FFA8B90120B040BAF1000F65
:106E10000AD0F7F73BFD0D48FCF7BCFF39460C489C
:106E2000BDE8F84FFDF77AB840EA0900C8F800005D
:106E30000848F1E70136DAE78ED6060880530608DF
:106E40001E2807088AE5060898D60608A4D606086C
:106E5000C7D60608ADD60608A03F00202DE9F84F9A
:106E6000054643F047FA354F0446D7F8786BC8B962
:106E70003348344DDFF8DC80FCF78CFF0127E3B2A8
:106E800005EB8302D2F8681441B107FA03F33342E9
:106E900002D04046FDF728F80134F0E7BDE8F84F8E
:106EA000FCF7A6BF024628492846F6F743FF60B91B
:106EB0002648274C274DFCF76DFF54F8041B00298A
:106EC000ECD02846FDF710F8F7E72B78DFF880B014
:106ED0002D2B03BF013504F1FF344FF0010A4FF0B1
:106EE000000A4FF000095BF8048BB8F1000F03D1E2
:106EF000BDE8F84F3EF0B8B8224641462846F6F7BE
:106F000019FFB8B9012303FA09F3BAF1000F0CD045
:106F100026EA03031048C7F8783BFCF73BFF4146DD
:106F20000E48BDE8F84FFCF7F9BF33430C48C7F8EB
:106F3000783BF2E709F10109D5E700BF08CF00204F
:106F40008ED606089C4F06088AE5060898D60608DD
:106F5000045406081E280708A4D60608C7D6060843
:106F6000ADD606082DE9F047814643F0C3F94D4EF2
:106F70000446376800BB4C484C4D4D4EFCF7B4FFFF
:106F80004FF00C0808FB04F35B5D5A1E012393408D
:106F90003B4206D020461CF03FFD01463046FCF740
:106FA000A3FF0134182CEDD117B94248FCF7F2FECB
:106FB000BDE8F047FCF71CBF02463F494846F6F7DC
:106FC000B9FE054678B93D48FCF7E4FE2C46384D3D
:106FD00020461CF021FD013401462846FCF784FFC1
:106FE0001A2CF5D1E4E799F800302D2B03BF09F1F5
:106FF000010904F1FF344FF0010A4FF0000A4FF08D
:10700000000840461CF008FD224605460146484659
:10701000F6F790FE00283BD1BAF1000F1FD0B8F16F
:10702000180F0BD16FF07F4333602548FCF7B2FE99
:1070300029462448BDE8F047FCF770BFB8F1190FA6
:1070400001D17368F0E7204B0C2202FB083898F856
:10705000A0345A1E012393401F433760E5E7B8F17F
:10706000180F03D1C6F800A01848DFE7B8F1190FD0
:1070700001D17760F8E7144B0C2202FB083898F82E
:10708000A0345A1E0123934027EA03073760EBE739
:1070900008F10108B8F11A0FB3D1BDE8F0473DF08F
:1070A000E3BF00BF80720020B5D606083C54060836
:1070B000C6D60608BFD606088AE50608CBD6060857
:1070C000A4D60608C7D606089C4F0608ADD6060803
:1070D000F0B585B0044643F00DF904283AD1661E98
:1070E0002546E71C16F8010FF6F71EFEBE4230706B
:1070F000F8D11B4F261D15F8011B019138464AF0A7
:107100005CFC20B1019928464AF057FC20B105B03B
:10711000BDE8F040FDF7BCB8B542ECD1204621F007
:10712000E9FA1048104CFCF735FE0D4901231A5DB1
:1071300011F8010B10326A440133052B02F8080CD8
:10714000F5D1002309488DF80C3002A9FCF7E6FEC2
:1071500005B0F0BD0028E4D0FDF79AF8E1E700BFE4
:1071600074550608D6D6060884DA0020B2D406087C
:1071700008B504460648FCF70DFE064B1868F8F7FC
:107180008BFB054B18681DF017F9204606F0F8FF39
:10719000DCD606081074002018740020034808B5D7
:1071A000FCF7F8FD0120FFF7E3FF00BFE8D6060873
:1071B0007FB5194B93F87C2B012A29D193F8813B99
:1071C0000A2B05D0154807B05DF804EBFCF7E2BDCB
:1071D0001122002101A849F091FCA6238DF800306E
:1071E00041238DF80130EB238DF803300C4B1B78D5
:1071F0008DF80430B22315218DF80530684603233D
:107200008DF802108DF8063021F0ABFC0548DAE766
:1072100007B05DF804FB00BF08CF002001D70608C7
:107220004C11002010D7060808B50A48FCF706FEE6
:10723000094B1868F8F730FB084B002483F89E4B85
:10724000C3F8E04B83F8E44B13F00EFF2046FFF742
:107250008FFF00BF2AD706081074002008CF002037
:1072600008B5214B214C1D68D4F8F00B1DF0A4F893
:1072700028461DF0A1F8D4F8F00B41798B0704D40F
:10728000036841F002019B69984700210846F9F71D
:10729000A7F900210120F9F7A3F9D4F8F00BFAF7C8
:1072A00081F878B101210020F9F79AF9D4F8F00BB0
:1072B000FAF799F801462846FAF771F800210846CE
:1072C000F9F78EF92846FAF76DF80028E5D0012184
:1072D0000846F9F785F92846FAF785F80146D4F803
:1072E000F00BFAF75CF8D4E71874002008CF002000
:1072F000F7B50546FCF7D8FF044620B103B0BDE85A
:10730000F040FCF7C5BF28461E491E4F01AA48F0B1
:1073100065FA2646254640B90B2D18D901461A486C
:107320000B22FCF7B9FF03B0F0BD44B1012C0AD029
:1073300001AA39460020013448F050FAEBE7F7F78C
:1073400041F90546F4E7F7F73DF90646F0E7022C68
:107350000ED1A6F57A73B3F57A7F05D90B484FF4B1
:10736000FA624FF47A71DCE7094B03EB45039E8028
:10737000074B084803EB45032946B3F90420FCF703
:10738000CDFDD0E75824070894D1060864F206081A
:10739000F855012054D7060870B50446FCF784FF61
:1073A000C0B11F4B5E68013630461CF035FB3446D9
:1073B0000546E8B901341A2CA8BF002420461CF069
:1073C0002BFB0546A0B9B442F4D1BDE87040154886
:1073D000FCF734BD2046F7F7F5F804461CF01CFB1B
:1073E000054628B921461048BDE87040FCF796BD17
:1073F0000B4B5C601DF094FA0C4821462A46FCF7C2
:107400008DFD192C9DBF0A480C2101FB04000020B2
:10741000BDE8704098BF90F8A0041DF099BA00BF75
:107420004C11002061D7060875D706088BD70608CF
:107430009C4F060838B51749052204464AF0D2FA8F
:1074400058B9154A13781BB901211170134A1370EA
:10745000BDE838401248FCF7F1BC1249032220462F
:107460004AF0C0FA80B90C4D0C4C2B7843B123780C
:1074700033B10D48FCF75FFD00232B70237038BD3E
:107480000A48FCF7DBFCF7E7BDE838400848FCF7A2
:1074900052BD00BFFEDD06081474002015740020E4
:1074A000A0D7060845E00608B6D70608EDD70608B7
:1074B00001D8060838B50E4D2B7863B10D4C2378F2
:1074C0004BB10D48FCF737FD0C48FCF734FD0023A9
:1074D0002B70237038BD0A48FCF75CFC21F0EEF8F5
:1074E000F7F7D2F821F0F4F80020FFF741FE00BFD3
:1074F0001474002015740020B6D7060810D80608AA
:107500002ED806082DE9F0478CB0074610F8013B4D
:10751000202BFAD000251F4CDFF88080DFF8809008
:10752000DFF880A02E466946204612F0D1F9394690
:1075300068464AF09CFAE0B169464046FCF7D4FC44
:107540004946684642F0CCFEF8B9204612F0A0FA4F
:10755000114B0146007820280CBF50461846FCF716
:10756000C3FCFCF745FC2046FCF73AFEFCF740FC68
:1075700001360135B5F5197F04F10B04D3D10EB9ED
:107580003DF072FD0CB0BDE8F08700212046FCF70D
:107590001BFEE6E74A350608B2D40608D4CE060834
:1075A000222C0708AAD406082DE9F04F2DED028BF6
:1075B0008DB00578202D064600F10100F9D0304647
:1075C00042F098FE044618B1012820D12A2D1ED180
:1075D0009248934D934FFCF731FC002628466946AC
:1075E00012F076F969463846FCF77EFC01362846EB
:1075F0002146FCF7E9FDFCF7FBFBB6F5197F05F129
:107600000B05EBD10DB0BDEC028BBDE8F08F3D2139
:1076100030464AF0D2F9002800F0F8800346994637
:1076200013F8012D202AFAD0A9EB06090130804673
:10763000074610F8013B202BF9D0794D4FF0000A96
:107640005FFA89F96946284612F042F9684642F025
:1076500051FE6946024683463046F6F76BFB704B97
:10766000044650BBCB4528D10B2202FB0A339B7941
:1076700003F00706062E38D1404642F03BFE844216
:10768000064624D36849684642F02AFE20B167497D
:10769000684642F025FE28BB98F80030222B21D105
:1076A00008EB060313F8013C222B1BD1B21E08F194
:1076B0000101284612F0B6FAA4E70AF1010ABAF568
:1076C000197F05F10B05BDD13DF0CEFC9AE718F806
:1076D0000430A3F16102192A9CBF203B08F8043052
:1076E0000134C9E732464146E3E713F0C0030AD04C
:1076F000402B5BD04E48FCF7A7FB2846FCF770FDFB
:10770000FCF776FB7EE798F80030002BF2D0494971
:1077100040464AF09CF90446404642F0EBFD844264
:10772000E8D14046F6F7C2FE2846B0EE408A12F095
:10773000BCF907EE900AF8EEE77AF4EEC87AF1EEBB
:1077400010FAD7D8284612F0C1F907EE900AF8EEE1
:10775000677AF4EEC87AF1EE10FACBDB052E0BD186
:1077600018EE104A284612F093F9052E3FD8DFE8AC
:1077700006F03D3D4747494B042E12D13A4617F8D3
:10778000013B202BFAD0092BF8D0013A00240A2122
:1077900012F8013F303BDBB2092BE3D801FB043484
:1077A000F6E74046F6F70EFF0446DBE7284612F000
:1077B0001DFA90F804B0814627462346A246BB45F1
:1077C00000D91BB1BAF1000F94D0CBE7D9F8003043
:1077D000414653F82700F6F7C9FA002805BF3C4692
:1077E000012300234FF0010A0137E8E704706946DE
:1077F0001148FCF779FB00212846FCF7E5FC01E77E
:107800000480F4E70460F2E70460F0E730460DB06E
:10781000BDEC028BBDE8F04F74E600BF35D806081A
:107820004A350608D4CE0608222C070847D8060891
:107830006BD8060852D8060860D806082DE9F04F24
:10784000A5B0C04B0293C04B0193C04BC04AC14985
:10785000C1480093C14BC24CC24DC34FFCF75EFB05
:10786000C249C348FCF75AFBC24BC34819684FF4DE
:107870007A73B1FBF3F1FCF751FB08A8F6F776FB3E
:10788000BE4B08A9B3F9002018A83FF089FB18A93E
:10789000BB48FCF743FB21F08FFC94F81D3C05EB43
:1078A00083036422D3F8E035B0FBF2F102FB11024E
:1078B0000093B44894F81C3C92B289B2FCF72EFBBA
:1078C000B14BB2481968B24BB1FBF3F1FCF70CFBBA
:1078D000D7F81C80002605F5BE6904F61E4A05F29D
:1078E0000C6B0123B34013EA080F0BD059F8263074
:1078F00043B11AF806205BF8261053F82220A54859
:10790000FCF7F2FA0136072EEBD1FCF771FAA24828
:107910009F4EFCF793FA0BA8F2F702FD0B999F48D4
:10792000B1FBF6F1FCF7FAFA0C999D48B1FBF6F1C0
:10793000FCF7F4FA0D999B48B1FBF6F1FCF7EEFA6F
:107940000E999948B1FBF6F1FCF7E8FA22F066F8D7
:1079500005EB8000D0F83416079122F069F805EBAA
:107960008000D0F83426069222F072F805EB8000F1
:10797000D0F83436059322F08FF805EB8000D0F86C
:10798000349622F0ABF8064622F0F2F8804622F058
:10799000D7F805EB800005EB8808D0F83406039093
:1079A00005EB8606D8F834060290D6F83406079917
:1079B000CDE90090DDE905327C48FCF7AFFA7C4B5D
:1079C0001B68DB031CD57B4B93F80080B8F1000FDC
:1079D00016D07948DFF83892DFF838A24146FCF734
:1079E0009DFA0026B9F90220314650460136FCF7CF
:1079F0007BFAF3B2434509F11009F3D3FCF7F8F928
:107A00000020FEF777FF6D4B6D4A1E886D4B6E4967
:107A10001B686E48DFF800A2DFF80092DFF80082F2
:107A2000DFF800B2C3F500739B00FCF777FA684AF1
:107A3000684B6948D31A694AB6B231461288FCF7D6
:107A40006DFA6748FCF7FAF904265AF8041B6548F2
:107A5000FCF74AFA6448FCF79DF919F8011B002964
:107A600040F097816148FCF795F96148FCF792F97D
:107A700058F8041B002940F090815C48FCF7DEF9BF
:107A8000013EE2D1398C5B48FCF72EFA5A490A6F65
:107A90005AB107EE902ADFED596AF8EEE77A86EEE2
:107AA000A77AFDEEC77A17EE902AD1F800315BB1C4
:107AB00007EE903ADFED516AF8EEE77A86EEA77AA4
:107AC000FDEEC77A17EE903A896A59B107EE901A1F
:107AD000DFED4A6AF8EEE77A86EEA77AFDEEC77A1E
:107AE00017EE901A46480091464FB4F82C1CDFF868
:107AF0003891FCF713FA4448FCF74CF93E6826F03D
:107B0000004626F07F064FF00108002E40F0498124
:107B1000FCF76EF93B685F0140F18C800FA811F013
:107B2000EDFF002840F086800F9BB3F5197F3DBF25
:107B300036480B2606FB0300304618A911F0C8FE94
:107B400074E000BFCFCA0608D8CA0608E1CA060812
:107B50002CCA06083FCA060831D60608EDCA060830
:107B600008CF00209C4F0608F855012047D606088C
:107B700063D60608842B0020AED80608003E0020FD
:107B8000C8D80608D9D8060860060020FED806081E
:107B900040420F000ED9060816D906082BD9060850
:107BA0003DD906084FD9060861D9060873D90608D9
:107BB000EC550120E8550120C6D90608B02C00205C
:107BC000000002206C35002000180000FAD90608D9
:107BD000008000080040000832DA06089C3F0020C0
:107BE0006CDA06087FDA060887DA0608C1D60608C6
:107BF0009DDA0608A7DA0608E80800200024744980
:107C0000B7DA060850550120F4DA06084A350608A6
:107C1000C43E0020EBD90608E05506082DDB002005
:107C2000E861002096DA0608C7D60608734818A946
:107C3000FCF781F97248FCF7ADF8D4F8301C002944
:107C400000F0C2800B7B4A7B6E488968FCF74CF9D8
:107C5000FCF7CEF86C48FCF79DF8D4F8340CFCF730
:107C600034F8002800F0B4800FA9D4F8340CFCF7E5
:107C700074F89DF850109DF85C30169A6348FCF734
:107C800033F9139911B16248FCF72EF9119911B12A
:107C90006048FCF729F9FCF7ABF85F4B1B68180646
:107CA0006AD594F8383C012B66D85C48FCF772F82A
:107CB000D4F8F43BB3F5487F00F0988000F28C8054
:107CC000B3F5167F00F09480B3F52F7F00F092801B
:107CD0005349544AB3F5FA7F08BF114694F8FB0B99
:107CE00094F8F93B94F8F82B072896BF05EB800031
:107CF0000020D0F8B40600904B48FCF7F5F8FCF7EC
:107D000077F84A48FCF70AF94948FCF797F84948D8
:107D1000FCF794F894F8443C19070AD594F84C2CD5
:107D200094F84D1C4448C2F3C002C1F3C001FCF7F3
:107D3000F5F894F8443C5A070AD594F84C2C94F87A
:107D40004D1C3E48C2F38002C1F38001FCF7E6F807
:107D500094F8443C9B070AD594F84C2C94F84D1C9D
:107D60003748C2F34002C1F34001FCF7D7F894F85A
:107D7000481C3448FCF7D2F8334B1B7833B105EB81
:107D800083053248D5F8D416FCF7C8F825B0BDE80D
:107D9000F08F5846FCF7A8F867E65846FCF7BEF89F
:107DA0006EE696FAA6F3B3FA83F308FA03F2062B0B
:107DB00026EA02067FF7A9AE05EB83034846D3F80F
:107DC0003816FCF791F8A0E62148FBF7E3FF3FE700
:107DD0002048FBF7DFFF5EE7B3F5617F0CD0104969
:107DE0001D4AB3F57A7F08BF114677E71B4975E74F
:107DF0001B4973E71B4971E71B496FE70BDB06085B
:107E00001FDB060825DB06083EDB060844DB060808
:107E100062DB06086BDB0608A03F002087DB060854
:107E20007BD8060891D806088DDB0608B4DB060867
:107E3000C9DB0608EADB0608F6DB060808DC0608EC
:107E400019DC06082BDC06085B72002042DC060801
:107E500032DB06087ADB0608A6D8060883D80608AF
:107E60008AD806089FD8060898D806082DE9F34155
:107E70001A481B4C1B4E1C4FDFF87080FCF74EF865
:107E80000025E2792168A37994F808C006EB820204
:107E900001F13F41D2F8EC06A28806EB830301F51D
:107EA0007E01B2FA82F2890AD3F85C33C2F11F0272
:107EB0004131BCF1000F0CD0CDE900C04046FCF7C9
:107EC0002DF80135312D04F10C04DAD102B0BDE8F2
:107ED000F08100903846FCF721F8F2E75CDC0608F8
:107EE000486700209C4F060888DC060878DC0608F6
:107EF00010B5F3F704FF124CD0B11248FBF7B8FFEE
:107F00001148FBF747FF2068F7F7C6FC4FF47A707B
:107F1000FBF7EAF90D4B18681CF04EFA0C4B187879
:107F2000F9F7C2F802210120F2F7EAFFF9F7B4FAF3
:107F30000848FBF72FFF2068BDE81040F7F7ACBCFE
:107F40001074002096DC0608DCD6060818740020A1
:107F5000E8550120B6DC06082DE9F0410446254E1F
:107F6000254DDFF8B0800020FEF716F82348FBF718
:107F70007FFFB17822480131FBF7D0FF2146202056
:107F8000FCF776F81F48FBF773FFB3781E4A4FF4EF
:107F9000C87707FB0353D3ED047AF5EE407AF1EE90
:107FA00010FA0CBF012100212046FBF76DFFB178CC
:107FB0007943103108EB010220462944FCF754FEB6
:107FC0001248FBF755FFB378114A07FB03532046CD
:107FD000B3F9D210B1FA81F14909FBF755FFB17835
:107FE0007943D03108EB010220462944BDE8F04135
:107FF000FDF754BE2C77002038830020E5DC06080E
:10800000F3DC060806DD060819DD060828DD06088B
:108010003BDD06089C750020A0F2DC50164BB0F545
:10802000FA7FA8BF4FF4FA70984210B5B8BF18464F
:108030000C4611463DF01FF900B207EE900A9FED85
:108040000F7AF8EEE77AE4B287EE870AFBEE096A68
:10805000E0EE006A07EE904A9FED097AF8EE677A43
:10806000A7EEA67AF3EE097A20EE070A80EE270A39
:1080700043F098FD00B210BD0CFEFFFF0000C842A7
:1080800000401C452DE9F843884D95F8550C2DED21
:10809000028BB0EE408A80B3854E864FDFF828927F
:1080A000002405F5456895F87C3C062202FB037325
:1080B000234493F86A3753B1012B0DD00134042CBB
:1080C00006F10206EFD1BDEC028BBDE8F88308EBA8
:1080D00044031B8E3380F1E7032C01D00023F9E722
:1080E000D9F80030DA0405D412F04AFF00B2724B1E
:1080F0005885E3E740F2DC50F9E76F4C20F01AFBBB
:10810000E76AD5F8886C95F88C2C17F4807714BF43
:10811000717B317AFFF780FFA084012020F00AFBF9
:10812000002F00F08480717B95F88C2CFFF774FF92
:10813000E084022020F0FEFA002F7AD0B17B95F87F
:108140008D2CFFF769FF404200B22085002F72D0CE
:10815000A28CF37BE18C13FB02F3642293FBF2F31A
:10816000A384337C13FB01F393FBF2F3E384737C6E
:1081700013FB00F090FBF2F0208511F005F995F863
:10818000543C608543B9B4F92830626AC5F8802C44
:10819000A5F8843CA5F8860CE36A5B0693D5B4F990
:1081A000343007EE103AB8EEC77AF2EE046AC7EE42
:1081B000267AB5F9983C08EE103AB8EEC88A37EE40
:1081C000C88ADFED3E7ABDEEC88A18EE103A1BB2BF
:1081D00008EE103AB8EEC88A28EE278AB0EE480AB0
:1081E000F4F720FFF0EE408AB0EE480AF4F7B8FE4C
:1081F000B4F9263007EE903AB4F9243006EE903AFE
:10820000F8EEE66AF8EEE77A26EE807AA7EEA87A2C
:1082100060EE677ABDEEC77AE6EEA87AFDEEE77A01
:1082200017EE903AA38417EE103AE3844BE7317AC5
:108230007AE7717A83E7224EB4F924003378122B5F
:1082400008BF204BB0EE480A08BF1860002112F0AA
:10825000EDFD3378122B02BF1A4BB4F926209A6039
:1082600000B208BF5860A084B0EE480A0121B4F9FA
:10827000260012F0DBFD3378122B02BF114BB4F94C
:1082800028201A6100B208BFD860E084B0EE480A26
:10829000B4F92800022112F0C9FD3378122B08BF6F
:1082A000084B00B2208508BF586166E708CF002060
:1082B0001C5601209C4F0608F855012035FA8E3CCB
:1082C000EC730020F0730020F05501202DE9F043FD
:1082D000DFF8F891774CD9F80030D3F82880764B46
:1082E0001B6813F0100F87B040F0A68094F8383068
:1082F000002B00F0A180714E06F69C45D6F8A43CF8
:1083000028469847002800F0978096F8013D002BFA
:1083100043D1022384F85830B6F9023D07EE903A73
:10832000B6F9043DF8EEE77AC5ED0A7A07EE903A21
:10833000B6F9063DF8EEE77AC5ED0B7A07EE903A0E
:10834000F8EEE77AC5ED0C7A5D4903AAA1F10C00BD
:108350003DF0EAFF03A996F8E02C084621F0DEF88C
:1083600003A821F09DF895ED060A5649554D03A83E
:108370003DF0E7FF05F178070026B5EC010AD4F8D7
:10838000243185ED020A384698470136032E05ED63
:10839000010A07F12407F0D14EE094F85830012B80
:1083A000D2D1EB6903932B6A049303A96B6A0593FB
:1083B00004F15800F5F75AF994F85830012B4FF0B2
:1083C000000772D0022B67D0039704970597DDED65
:1083D000037A9DED047ADDED056AC5ED0A7A85ED37
:1083E0000B7AC5ED0C6AFDEEE77ABDEEC77AFDEEBD
:1083F000E66A17EE903A17EE102A16EE901A1BB2A4
:1084000012B209B2A6F8023DA6F8042DA6F8061D80
:108410000120CDE9002104212B4AF5F7B3FAD9F860
:10842000003000200021C3E90C01C3E91001C3E9B9
:108430000E0127646764A764E3695B0629D51F4DB5
:1084400095F8383D2BB34FEAE8763146404642F086
:10845000D3FD05F5516307EE900AD4ED106A93ED54
:108460000F7AD5F8582DD5F85C1DA7EEA67A12EB39
:10847000080246EB0106D4ED116A83ED0F7A93ED05
:10848000107AC5F8582DA7EEA67AC5F85C6D83ED75
:10849000107A07B0BDE8F083236F0393D4F88830D7
:1084A0000493D4F8A030059391E7AF62EF622F6395
:1084B000BFE700BFF85501205055012008CF00202C
:1084C000CCDB00203856012048DD0608E4550120A9
:1084D00038B52D4B1B68580350D5D90609D42B4B02
:1084E0001A782B4B302101FB0233D3F89037DA0591
:1084F00045D4284B5D79002D40D0274AD26A930796
:108500003CD02DB212F03CFD044611F0FBFC9FED77
:10851000237AB4EEC70AF1EE10FAF7EE007A30D4FF
:10852000B4EE670AF1EE10FAC8BFB0EE670A07EEC4
:10853000105AC7EE806A184DB5F92A301B1B00216E
:10854000B8EEC77ADFED165A87EE256A76EEE76A4F
:10855000E6EE867AB0EE677A07EE903AF8EEE76AD2
:1085600007EE904AF8EEE77AE6EE877AFCEEE77AD5
:1085700017EE903A98B212F00FFF688538BD642567
:10858000C0E7B0EE470AD2E7EC550120408D00204D
:108590009C4F06082C770020F85501209A99193F26
:1085A0000000C842034B012283F8682D022283F8A1
:1085B000692D704708CF002070B50D4E35782D1A03
:1085C00018BF01250328044634BF04460024204672
:1085D000F6F7AEF9074B347003F66A501A2204FB23
:1085E0000200C3F8880C1BF0BBF8284670BD00BF22
:1085F0002C77002008CF0020022810B50C4618D890
:10860000FFF7DAFF0B48FBF733FC0B4B0B481978ED
:108610000131FBF783FC21460820FBF729FD2146A9
:108620001020FBF725FD21462820BDE81040FBF770
:108630001FBD10BDFFE406082C770020F9DC0608FA
:1086400038B5154C154DAC4213D30020F6F770F930
:10865000134820F04FF8134A136843F48003136063
:1086600000BF114B1878FFF7A7FFBDE8384029F08D
:1086700089BFB4F90230002B4FF00001204607DA21
:10868000F6F746F901212046F6F742F90221204685
:10869000F6F73EF91434D6E798350708C03A0708CC
:1086A0006FDD0608A03F00202C77002010B504469F
:1086B0000A48FBF76FFBFFF7C3FF1FF0FFFFF5F75B
:1086C000E3FF20F005F8064B0649002220461A7009
:1086D000FDF79FFD08B9FEF74BFD10BD78DD0608DC
:1086E0001574002036DE060810B5064B5C78241A97
:1086F00018BF0124032828BF0020587020F01EFD59
:10870000204610BD2C770020022810B50C4610D84A
:10871000FFF7EAFF0748FBF7ABFB074B0748597821
:108720000131FBF7FBFB21461820BDE81040FBF7A9
:108730009FBC10BD8EDD06082C7700209EDD06084C
:108740002DE9F04F0D468DB0B4490446FDF761FDAB
:108750000646002840F0B580B1492046FDF759FD96
:108760000646002840F0AF80AE492046FDF751FD97
:108770000646002840F0A980AB492046FDF749FD98
:108780000646002840F0A3802046A849FDF741FD99
:108790000028064612BF1024264601240DB144F0DD
:1087A0002004A34DA34F95F800A095F8019095F8EB
:1087B0000280DFF8F4B25F45C0F08B80FFF740FF26
:1087C0005046FFF7F9FE4846FFF78EFF4046FDF79B
:1087D000E3FB99493046FDF71CFD08B144F0400425
:1087E00014F01103009300F099829448FBF740FBCA
:1087F0000020FEF76BFA9248FBF73AFB9148FBF733
:108800001DFB04F03003302B02D18F48FBF730FB07
:108810008E48DFF89892FBF72BFB8D48FBF728FB7F
:108820004FF0FF338B4A8C492046FDF7C1FE8B4841
:10883000FBF71EFB8A4A8B492046FDF771F98A48EF
:10884000FBF716FB894A8A492046FCF751FE894806
:10885000FBF70EFB884A89492046FCF741FD884812
:10886000FBF706FB874B884A1E68884B1F6867EA40
:108870000603CB464FF0000A01935BF8043B002B44
:1088800034D01978D1B1019902934FF0010808FA58
:108890000AF811EA080F14BF012100212046FBF756
:1088A0000DFB66EA070111EA080F774A029B14BF25
:1088B000012100212046FBF7E7FA734A0AF1010A79
:1088C000DBE701246AE7022468E7042466E708245A
:1088D00064E77B88C3F30B021B04D7E9011048BF90
:1088E00002EB420245F06CFF143764E79846684A91
:1088F00067EA0603019359F804BBBBF1000F27D0C8
:108900009BF8001009B34FF0010A0AFA08FA17EAB7
:108910000A0F0BD066EA070111EA0A0F5B4614BF83
:10892000012100212046FBF7C9FA594A16EA0A0F2D
:108930000BD0019B13EA0A0F18BF01215B4608BF49
:1089400000212046FBF7A0FA514A08F10108D2E7BE
:108950005048DFF85CA1FBF78BFA4F4AD2F8009041
:108960004E4A12685E4689EA0208DFF848B16FEAAB
:1089700008080127B74018EA070F14BF012100219A
:1089800019EA070714BF52465A463046039101922E
:108990001BF042F8019A0399029003462046019188
:1089A0000136FBF78BFA002F14BF5A465246029B42
:1089B00001992046FBF768FA182EDAD13848DFF81B
:1089C000F8A0DFF8F880DFF8F890FBF751FA354BA4
:1089D000D3F8C07D0026F3B20AEB8302D2F868B464
:1089E000BBF1000F6ED00121994039405B460CD09D
:1089F0004A4600212046FBF747FA5B464A460021DB
:108A00002046FBF75BFA0136E5E742462046019136
:108A1000FBF73AFA01995B464246F1E7C8DD0608E2
:108A2000FFE406088EDD0608E5DC0608CFDD060853
:108A30002C77002098350708D3DD060828E90608BA
:108A4000E0DD0608F8DD060804DE06085AE506083B
:108A50003FDE0608686F0020548600204FDE0608BF
:108A6000C67C0020467D00205FDE06087879002065
:108A7000B480002068DE0608687800201481002099
:108A800079E30608A43F00207CDE0608A03F002012
:108A900088DE060815E206083C8600208072002069
:108AA00093DE060808CF0020C03A07088053060866
:108AB000B3DD0608BDDD06089C4F0608A8DE0608E3
:108AC0009CDE06089D489E4EFBF7D2F901239D4887
:108AD0008DF820B08DF810B08DF821B08DF811B060
:108AE0008DF822B08DF812B08DF823B08DF813B048
:108AF0001F46A6F5127E9A5D10F801CB02F13001F7
:108B0000694401F820CC13F80E1001F13008E84454
:108B100008F810CC2FB1A2EB010CDCF1000747EBF9
:108B20000C070133052BE6D13946874A002608ABEE
:108B300020468DF81460FBF7C1F904AB3946824A30
:108B40002046FBF7A1F98148FBF792F9804A814959
:108B50002046FBF799FE8048FBF78AF97F4A804957
:108B60002046FCF773FD7F48FBF782F97E4A7F4978
:108B70002046FCF799FE7E48FBF77AF9774A784958
:108B80002046FCF72DFF7B48FBF772F97A4A7B49B8
:108B90002046FBF7ABFD7A48FBF76AF9794A7A4938
:108BA0002046FBF775FF7948FBF762F9784A794967
:108BB0002046FCF77BF97848FBF75AF9774A784961
:108BC0002046FCF70FFA7748FBF752F97649204622
:108BD0003CF060FA7548FBF74BF94FF0FF331A464B
:108BE000734920463CF0E0FA7248FBF741F94FF038
:108BF000FF33714A71492046FDF73EF97048FBF793
:108C000037F9704A70492046FDF720FB6F48FBF7A3
:108C10002FF96F4A6F492046FDF7AEFB6E48FBF710
:108C200027F96E4A6E492046FDF7FCFC6D48FBF7BC
:108C30001FF921463046FBF71BFAE7065FD52046B1
:108C400095F800806F7895F80290FFF785F9214636
:108C50003046FFF7D1FC21460120FFF7CDFC21462D
:108C60000220FFF7C9FC21463046FFF74DFD2146A3
:108C70000120FFF749FD21460220FFF745FD404650
:108C8000FFF79AFC3846FFF72FFD4846FDF784F9B9
:108C90005548FBF7EDF8554809F10101FBF73EF99E
:108CA000534808F10101FBF739F95248791CFBF7E9
:108CB00035F9200704D5AB7813B92046FFF74CF9F6
:108CC000A10703D528782146FFF796FC620703D554
:108CD00068782146FFF718FD009B13B14648FBF763
:108CE000C7F82EB14548FBF7C3F84548FBF7A6F88F
:108CF000444C454DAC4213D30DB0BDE8F08FAB787A
:108D000013B92046FFF728F928782146FFF774FCAD
:108D100068782146FFF7F8FC0126CAE7009EC8E7FD
:108D20006388C3F30B021B04D4E9010148BF02EBC3
:108D3000420245F045FD1434DCE700BFB5DE06080D
:108D4000CCDC002074550608CBDE0608D2DE06080F
:108D5000F074002068850020D8DE0608D87900204D
:108D6000C67D0020DDDE0608587C002046800020FD
:108D7000E7DE0608F6DE06081D7400209C8500204C
:108D800002DF060824750020F084002019DF0608A1
:108D900054770020288300202ADF06086877002007
:108DA0002882002036DF0608F0DC002055DF0608A8
:108DB00050E6002066DF060898CF002000EB002078
:108DC00079DF060898D4002000F0002097DF06081D
:108DD000F8D4002060F00020B4DF060868D5002039
:108DE000D0F00020C8DD0608C9DF0608ECDF060861
:108DF000F2DF0608FDDF060810E0060829E0060895
:108E00003FE0060898350708C03A0708002197E4B4
:108E1000012195E42DE9F74FBF4CC04B9C42C0F0B7
:108E20006781BF4C2078FFF7C7FB6078FFF75CFCD9
:108E3000A078BC4CFDF7B0F894F8483094F849207D
:108E4000B9489A4224BF002384F84830F5F71EFD44
:108E5000B64B1A68B64B934312D100212520F0F788
:108E600071FE054660B100212720F0F76BFE38B196
:108E700002682B689A4203D14FF48030F5F706FD63
:108E80000026AC4F35464FF0FF0848F2B83957F886
:108E900026004308810801F0333103F077330B4497
:108EA000C10801F01131C31A5B1A03EB131310F060
:108EB000010203F00F33B3FBF8F1C1EB012118BF3E
:108EC0000135A3EB010318BFEDB2012B08D9022B2A
:108ED0000CD112B110EA090F02D13EF075FA28B197
:108EE00003360C2ED3D1013D022D03D991480D211B
:108EF0003FF02EFFB4F87830B4F87620643B93420C
:108F0000A8BF1346A4F8763000BF94F8E43013B934
:108F1000082384F8E430002010F0F0FD864D2B6823
:108F2000002800F0378123F080632B60834BDFF84B
:108F30002482D3F8887C12F023F8814B39781E887C
:108F400083B2361A6422009306FB01F393FBF2F31B
:108F500013FA80F0A4F8FA0097F80190C1F16E03BB
:108F600001EB810CA2EB090B9BB24A42C1F1640EEA
:108F70004FEA4C0C92B201935FFA8EFE4FF00A0A50
:108F800017B2002F40F30981704607FB07F309FB76
:108F900003F310FB00F093FBF0F0584407FB00F3E1
:108FA00093FBFAF363441BB24FF47A70734393FB61
:108FB000F0F30098034428F8023B0A32019B92B276
:108FC0009342DDD120F0D4F81AF058F93022002174
:108FD0005C4847F093FD10F0BEFB584B93F8542CBF
:108FE0004ABB93F83A00C3F8602C6421C82611FBF1
:108FF0000060C3F8580C93F83B00C3F8642C11FBD5
:109000000061C3F85C1CC3F8682C93F83D10C3F8EA
:109010006C2CC3F8702CC3F8742C83F87D2C83F867
:109020007E2C83F8552CC3F8802C4FF07A7283F88D
:109030007C1CC3F8842C2B6843499B060A6800F10A
:10904000B080E08FA38F0343B4F8400003431BB20A
:10905000002B40F0A680B4F94230B3F5805F40F0B9
:10906000A080B4F94430B3F5805F40F09A80B4F941
:109070004630B3F5805F40F0948022F400720A60BD
:109080001FF09CFFB4F82C21DFED307A304B07EE57
:10909000102AB8EEC77AB4F82E21C7EE276A07EE79
:1090A000102AB8EEC77AC3ED506AC7EE276AB4F843
:1090B000302107EE102AB8EEC77AC3ED516AC7EE29
:1090C000276AB4F8322107EE102AB8EEC77AC3ED4A
:1090D000526AC7EE276A94F8342183F85021C3ED11
:1090E000536A19F0C3F903B0BDE8F04F36F03EBC47
:1090F000B4F90230DFF86090002BADBF00270327E2
:109100004FF00108B846002608EB0601C9B28F42AD
:1091100024D2143481E600BF98350708C03A070806
:109120002C770020F8F0002020631406A03F0020D8
:1091300040000100F07400205055012008CF0020AD
:10914000903F0020F4F10020EC55012000401C4627
:10915000F85501202057012000800008234A02F121
:10916000060ACA453DD21588DDB35019484538D2A4
:10917000052D36D9B4F800C0B2F802E0CCF30B0CE0
:10918000E64505D192F805C00CF0030C8C450BD0D8
:109190000246E4E743F08063C7E614BF08460120B7
:1091A000F3E642F400726AE73146204692F804B0D2
:1091B000F5F7AEFB2188BBEB113F10D1B4F802C02C
:1091C0006068CCF30B01AA1F8A42A8BF0A461CF4B0
:1091D000004F18BF01FB0600514645F0F1FA013679
:1091E00092E731462046F5F793FBF8E70140000887
:1091F00010B5154C94F8693D022B18D11FF05EFA9A
:10920000F5F742FAFFF706FE1FF062FA01201BF0A5
:10921000DDFB0E4B0E491B6803F59C5300220833FF
:1092200084F8682DC1F83C3184F8692D10BD012BFC
:10923000FCD11FF043FAF5F727FA1FF049FA002393
:1092400084F8693DF2E700BF08CF0020842B00209E
:10925000F8F0002010B50446FFF7AEF938B11FF062
:109260002DFAF5F711FAFFF7D5FD1FF031FA601C62
:10927000C0B2BDE810401BF0A9BB38B50C4D044688
:109280002046FBF711F838B10A4B0B481978BDE8B6
:1092900038400131FAF742BE2046F5F793F901381C
:1092A000022804D8C0B2FFF7D5FF2C46E8E738BD46
:1092B000F5EE06082C770020F2DF060810B504460C
:1092C000FFF712FA38B11FF0F9F9F5F7DDF9FFF7FA
:1092D000A1FD1FF0FDF9601CC0B2BDE810401BF0FD
:1092E00075BB38B50C4D04462046FAF7DDFF38B1A2
:1092F0000A4B0B485978BDE838400131FAF70EBEE9
:109300002046F5F75FF90138022804D8C0B2FFF70C
:10931000D5FF2C46E8E738BDF5EE06082C7700208F
:10932000FDDF060810B50446FCF736FE38B11FF025
:10933000C5F9F5F7A9F9FFF76DFD1FF0C9F9601C34
:10934000C0B2BDE810401BF041BB70B50C4E0446E6
:109350002046FAF7A9FF054638B10A4B0A48997822
:10936000BDE870400131FAF7D9BD2046F5F72AF97A
:10937000012804D12846FFF7D5FF3446E8E770BD41
:10938000F5EE06082C770020ECDF060838B5144D02
:10939000EC69630702D539F0FFFCF8B1200703D56B
:1093A000104B1B68D90519D5A20602D539F094FDDA
:1093B000A0B139F067FC10B9FCF71EFE68B995F84A
:1093C0005431012B04D1A30702D5FCF715FE20B9B7
:1093D00020F04EFC80F00100C0B238BD0120FCE757
:1093E000F8550120EC5501202DE9F843964C2568ED
:1093F00015F0040705D0BDE8F84301210020F7F778
:10940000EFB8FFF7C3FF914E002800F0B38045F49A
:109410000075256086F840718D4F256897F87E3C71
:10942000012B96F8423114BF45F4802525F48025A0
:1094300025603BB90FF080FF002800F0A98025F4DB
:109440000025256037F08EF950B197F88F0C25680C
:109450000FF05AFF002800F09E8045F400052560BB
:10946000DFF80882DFF80892D8F800202368110797
:10947000B9F8202054BF43F4807323F48073632A27
:109480008CBF43F4806323F480630020236036F0B4
:10949000C1F92568002800F0818045F40065D9F8FD
:1094A0001C301A077DD5D8F80020D00579D445F4B2
:1094B00080559907256077D5D8F800309A0573D480
:1094C000FCF79AFD00286FD045F40055256020F088
:1094D00067FB256800286AD145F400451220256005
:1094E0000FF0BEFF002865D045F4803517202560B9
:1094F0000FF0B6FF002860D045F400351B20256032
:109500000FF0AEFF00285BD045F080752560F9F7BD
:109510000FFED6E95232C01A4E4B61EB02015A7A65
:10952000022A50D84C4B4D4D002A18BF2B462568B7
:10953000984271F1000397F82A3034BF45F0005586
:1095400025F00055256093B12A200FF089FF0028EF
:1095500040D096F85031002B43D0B6F8462132B1B6
:109560003F4BD6F854111B685B1A934239D225F051
:10957000805538E096F8403125F400752560002BC1
:109580007FF44AAF012086F840011BF0E1F943E780
:1095900045F4002555E725F4000560E725F400654E
:1095A0007DE725F4805584E725F400558EE725F402
:1095B000004593E725F4803598E725F400359DE7CD
:1095C00025F08075A2E7274B234D033A012A88BF77
:1095D0002B46ACE7012386F85031214B1B68C6F8B7
:1095E000543145F08055256025686B0006D5002074
:1095F0000FF036FF10B925F08045256000200FF0F0
:109600002FFF2568184A15EA020315D0B0B145F4BA
:10961000804525602368134214BF0223002386F887
:109620005831F9F785FDD6F85C31C01A002808DBFF
:10963000BDE8F8431BF058B90028F0D125F4804567
:10964000E7E7BDE8F88300BF50550120F8F000209F
:1096500008CF00208072002000171100407E050016
:10966000842B002060CC050080FFFF7FEC5501209B
:10967000F855012070B5434D2B685C0771D5424CFD
:1096800084F86001F9F754FD2B68404A23F0040385
:109690002B6013683E4D23F0006313602B68C4E910
:1096A0005A01190307D594F870310A2B5AD8082BA0
:1096B00062D8012B58D8374EF36A1A0406D5142005
:1096C000F7F702FDF36A23F40043F36294F888315C
:1096D0009BB3314BD4F88C211B689B1A42F20F725A
:1096E00093422AD94FF47A72B3FBF2F3D4F87C2177
:1096F0001344C4F87C3134F031FDD4F89031C01AF1
